
STM32F407DISCOVERY.elf:     file format elf32-littlearm

Sections:
Idx Name          Size      VMA       LMA       File off  Algn
  0 .init         0000000c  00008000  00008000  00008000  2**2
                  CONTENTS, ALLOC, LOAD, READONLY, CODE
  1 .text         0000510e  0000800c  0000800c  0000800c  2**2
                  CONTENTS, ALLOC, LOAD, READONLY, CODE
  2 .fini         0000000c  0000d11c  0000d11c  0000d11c  2**2
                  CONTENTS, ALLOC, LOAD, READONLY, CODE
  3 .rodata       00000070  0000d128  0000d128  0000d128  2**2
                  CONTENTS, ALLOC, LOAD, READONLY, DATA
  4 .ARM.exidx    00000008  0000d198  0000d198  0000d198  2**2
                  CONTENTS, ALLOC, LOAD, READONLY, DATA
  5 .eh_frame     00000004  0000d1a0  0000d1a0  0000d1a0  2**2
                  CONTENTS, ALLOC, LOAD, READONLY, DATA
  6 .init_array   00000004  0001d1a4  0001d1a4  0000d1a4  2**2
                  CONTENTS, ALLOC, LOAD, DATA
  7 .fini_array   00000004  0001d1a8  0001d1a8  0000d1a8  2**2
                  CONTENTS, ALLOC, LOAD, DATA
  8 .data         000001e0  0001d1ac  0001d1ac  0000d1ac  2**2
                  CONTENTS, ALLOC, LOAD, DATA
  9 .bss          000019c8  0001d38c  0001d38c  0000d38c  2**2
                  ALLOC
 10 .comment      0000007b  00000000  00000000  0000d38c  2**0
                  CONTENTS, READONLY
 11 .debug_aranges 000010d0  00000000  00000000  0000d407  2**0
                  CONTENTS, READONLY, DEBUGGING
 12 .debug_info   0001720e  00000000  00000000  0000e4d7  2**0
                  CONTENTS, READONLY, DEBUGGING
 13 .debug_abbrev 00003218  00000000  00000000  000256e5  2**0
                  CONTENTS, READONLY, DEBUGGING
 14 .debug_line   00010961  00000000  00000000  000288fd  2**0
                  CONTENTS, READONLY, DEBUGGING
 15 .debug_frame  00004844  00000000  00000000  00039260  2**2
                  CONTENTS, READONLY, DEBUGGING
 16 .debug_str    000c8fc9  00000000  00000000  0003daa4  2**0
                  CONTENTS, READONLY, DEBUGGING
 17 .debug_ranges 00000f80  00000000  00000000  00106a6d  2**0
                  CONTENTS, READONLY, DEBUGGING
 18 .debug_macro  00024389  00000000  00000000  001079ed  2**0
                  CONTENTS, READONLY, DEBUGGING
 19 .ARM.attributes 00000030  00000000  00000000  0012bd76  2**0
                  CONTENTS, READONLY

Disassembly of section .init:

00008000 <_init>:
    8000:	b5f8      	push	{r3, r4, r5, r6, r7, lr}
    8002:	bf00      	nop
    8004:	bcf8      	pop	{r3, r4, r5, r6, r7}
    8006:	bc08      	pop	{r3}
    8008:	469e      	mov	lr, r3
    800a:	4770      	bx	lr

Disassembly of section .text:

0000800c <exit>:
    800c:	b508      	push	{r3, lr}
    800e:	4b07      	ldr	r3, [pc, #28]	; (802c <exit+0x20>)
    8010:	4604      	mov	r4, r0
    8012:	b113      	cbz	r3, 801a <exit+0xe>
    8014:	2100      	movs	r1, #0
    8016:	f3af 8000 	nop.w
    801a:	4b05      	ldr	r3, [pc, #20]	; (8030 <exit+0x24>)
    801c:	6818      	ldr	r0, [r3, #0]
    801e:	6a83      	ldr	r3, [r0, #40]	; 0x28
    8020:	b103      	cbz	r3, 8024 <exit+0x18>
    8022:	4798      	blx	r3
    8024:	4620      	mov	r0, r4
    8026:	f005 f877 	bl	d118 <_exit>
    802a:	bf00      	nop
    802c:	00000000 	.word	0x00000000
    8030:	0000d194 	.word	0x0000d194

00008034 <__do_global_dtors_aux>:
    8034:	b510      	push	{r4, lr}
    8036:	4c05      	ldr	r4, [pc, #20]	; (804c <__do_global_dtors_aux+0x18>)
    8038:	7823      	ldrb	r3, [r4, #0]
    803a:	b933      	cbnz	r3, 804a <__do_global_dtors_aux+0x16>
    803c:	4b04      	ldr	r3, [pc, #16]	; (8050 <__do_global_dtors_aux+0x1c>)
    803e:	b113      	cbz	r3, 8046 <__do_global_dtors_aux+0x12>
    8040:	4804      	ldr	r0, [pc, #16]	; (8054 <__do_global_dtors_aux+0x20>)
    8042:	f3af 8000 	nop.w
    8046:	2301      	movs	r3, #1
    8048:	7023      	strb	r3, [r4, #0]
    804a:	bd10      	pop	{r4, pc}
    804c:	0001d38c 	.word	0x0001d38c
    8050:	00000000 	.word	0x00000000
    8054:	0000d1a0 	.word	0x0000d1a0

00008058 <frame_dummy>:
    8058:	b508      	push	{r3, lr}
    805a:	4b03      	ldr	r3, [pc, #12]	; (8068 <frame_dummy+0x10>)
    805c:	b11b      	cbz	r3, 8066 <frame_dummy+0xe>
    805e:	4903      	ldr	r1, [pc, #12]	; (806c <frame_dummy+0x14>)
    8060:	4803      	ldr	r0, [pc, #12]	; (8070 <frame_dummy+0x18>)
    8062:	f3af 8000 	nop.w
    8066:	bd08      	pop	{r3, pc}
    8068:	00000000 	.word	0x00000000
    806c:	0001d390 	.word	0x0001d390
    8070:	0000d1a0 	.word	0x0000d1a0

00008074 <_mainCRTStartup>:
    8074:	4b15      	ldr	r3, [pc, #84]	; (80cc <_mainCRTStartup+0x58>)
    8076:	2b00      	cmp	r3, #0
    8078:	bf08      	it	eq
    807a:	4b13      	ldreq	r3, [pc, #76]	; (80c8 <_mainCRTStartup+0x54>)
    807c:	469d      	mov	sp, r3
    807e:	f5a3 3a80 	sub.w	sl, r3, #65536	; 0x10000
    8082:	2100      	movs	r1, #0
    8084:	468b      	mov	fp, r1
    8086:	460f      	mov	r7, r1
    8088:	4813      	ldr	r0, [pc, #76]	; (80d8 <_mainCRTStartup+0x64>)
    808a:	4a14      	ldr	r2, [pc, #80]	; (80dc <_mainCRTStartup+0x68>)
    808c:	1a12      	subs	r2, r2, r0
    808e:	f004 fdf3 	bl	cc78 <memset>
    8092:	4b0f      	ldr	r3, [pc, #60]	; (80d0 <_mainCRTStartup+0x5c>)
    8094:	2b00      	cmp	r3, #0
    8096:	d000      	beq.n	809a <_mainCRTStartup+0x26>
    8098:	4798      	blx	r3
    809a:	4b0e      	ldr	r3, [pc, #56]	; (80d4 <_mainCRTStartup+0x60>)
    809c:	2b00      	cmp	r3, #0
    809e:	d000      	beq.n	80a2 <_mainCRTStartup+0x2e>
    80a0:	4798      	blx	r3
    80a2:	2000      	movs	r0, #0
    80a4:	2100      	movs	r1, #0
    80a6:	0004      	movs	r4, r0
    80a8:	000d      	movs	r5, r1
    80aa:	480d      	ldr	r0, [pc, #52]	; (80e0 <_mainCRTStartup+0x6c>)
    80ac:	2800      	cmp	r0, #0
    80ae:	d002      	beq.n	80b6 <_mainCRTStartup+0x42>
    80b0:	480c      	ldr	r0, [pc, #48]	; (80e4 <_mainCRTStartup+0x70>)
    80b2:	f3af 8000 	nop.w
    80b6:	f004 fdab 	bl	cc10 <__libc_init_array>
    80ba:	0020      	movs	r0, r4
    80bc:	0029      	movs	r1, r5
    80be:	f003 fe9f 	bl	be00 <main>
    80c2:	f7ff ffa3 	bl	800c <exit>
    80c6:	bf00      	nop
    80c8:	00080000 	.word	0x00080000
	...
    80d8:	0001d38c 	.word	0x0001d38c
    80dc:	0001ed54 	.word	0x0001ed54
	...

000080e8 <HAL_Init>:
  *         need to ensure that the SysTick time base is always set to 1 millisecond
  *         to have correct HAL operation.
  * @retval HAL status
  */
HAL_StatusTypeDef HAL_Init(void)
{
    80e8:	b580      	push	{r7, lr}
    80ea:	af00      	add	r7, sp, #0
  /* Configure Flash prefetch, Instruction cache, Data cache */ 
#if (INSTRUCTION_CACHE_ENABLE != 0U)
  __HAL_FLASH_INSTRUCTION_CACHE_ENABLE();
    80ec:	4b0e      	ldr	r3, [pc, #56]	; (8128 <HAL_Init+0x40>)
    80ee:	681b      	ldr	r3, [r3, #0]
    80f0:	4a0d      	ldr	r2, [pc, #52]	; (8128 <HAL_Init+0x40>)
    80f2:	f443 7300 	orr.w	r3, r3, #512	; 0x200
    80f6:	6013      	str	r3, [r2, #0]
#endif /* INSTRUCTION_CACHE_ENABLE */

#if (DATA_CACHE_ENABLE != 0U)
  __HAL_FLASH_DATA_CACHE_ENABLE();
    80f8:	4b0b      	ldr	r3, [pc, #44]	; (8128 <HAL_Init+0x40>)
    80fa:	681b      	ldr	r3, [r3, #0]
    80fc:	4a0a      	ldr	r2, [pc, #40]	; (8128 <HAL_Init+0x40>)
    80fe:	f443 6380 	orr.w	r3, r3, #1024	; 0x400
    8102:	6013      	str	r3, [r2, #0]
#endif /* DATA_CACHE_ENABLE */

#if (PREFETCH_ENABLE != 0U)
  __HAL_FLASH_PREFETCH_BUFFER_ENABLE();
    8104:	4b08      	ldr	r3, [pc, #32]	; (8128 <HAL_Init+0x40>)
    8106:	681b      	ldr	r3, [r3, #0]
    8108:	4a07      	ldr	r2, [pc, #28]	; (8128 <HAL_Init+0x40>)
    810a:	f443 7380 	orr.w	r3, r3, #256	; 0x100
    810e:	6013      	str	r3, [r2, #0]
#endif /* PREFETCH_ENABLE */

  /* Set Interrupt Group Priority */
  HAL_NVIC_SetPriorityGrouping(NVIC_PRIORITYGROUP_4);
    8110:	2003      	movs	r0, #3
    8112:	f000 f939 	bl	8388 <HAL_NVIC_SetPriorityGrouping>

  /* Use systick as time base source and configure 1ms tick (default clock after Reset is HSI) */
  HAL_InitTick(TICK_INT_PRIORITY);
    8116:	2000      	movs	r0, #0
    8118:	f000 f808 	bl	812c <HAL_InitTick>

  /* Init the low level hardware */
  HAL_MspInit();
    811c:	f004 f8a4 	bl	c268 <HAL_MspInit>

  /* Return function status */
  return HAL_OK;
    8120:	2300      	movs	r3, #0
}
    8122:	4618      	mov	r0, r3
    8124:	bd80      	pop	{r7, pc}
    8126:	bf00      	nop
    8128:	40023c00 	.word	0x40023c00

0000812c <HAL_InitTick>:
  *       implementation  in user file.
  * @param TickPriority Tick interrupt priority.
  * @retval HAL status
  */
__weak HAL_StatusTypeDef HAL_InitTick(uint32_t TickPriority)
{
    812c:	b580      	push	{r7, lr}
    812e:	b082      	sub	sp, #8
    8130:	af00      	add	r7, sp, #0
    8132:	6078      	str	r0, [r7, #4]
  /* Configure the SysTick to have interrupt in 1ms time basis*/
  if (HAL_SYSTICK_Config(SystemCoreClock / (1000U / uwTickFreq)) > 0U)
    8134:	4b12      	ldr	r3, [pc, #72]	; (8180 <HAL_InitTick+0x54>)
    8136:	681a      	ldr	r2, [r3, #0]
    8138:	4b12      	ldr	r3, [pc, #72]	; (8184 <HAL_InitTick+0x58>)
    813a:	781b      	ldrb	r3, [r3, #0]
    813c:	4619      	mov	r1, r3
    813e:	f44f 737a 	mov.w	r3, #1000	; 0x3e8
    8142:	fbb3 f3f1 	udiv	r3, r3, r1
    8146:	fbb2 f3f3 	udiv	r3, r2, r3
    814a:	4618      	mov	r0, r3
    814c:	f000 f951 	bl	83f2 <HAL_SYSTICK_Config>
    8150:	4603      	mov	r3, r0
    8152:	2b00      	cmp	r3, #0
    8154:	d001      	beq.n	815a <HAL_InitTick+0x2e>
  {
    return HAL_ERROR;
    8156:	2301      	movs	r3, #1
    8158:	e00e      	b.n	8178 <HAL_InitTick+0x4c>
  }

  /* Configure the SysTick IRQ priority */
  if (TickPriority < (1UL << __NVIC_PRIO_BITS))
    815a:	687b      	ldr	r3, [r7, #4]
    815c:	2b0f      	cmp	r3, #15
    815e:	d80a      	bhi.n	8176 <HAL_InitTick+0x4a>
  {
    HAL_NVIC_SetPriority(SysTick_IRQn, TickPriority, 0U);
    8160:	2200      	movs	r2, #0
    8162:	6879      	ldr	r1, [r7, #4]
    8164:	f04f 30ff 	mov.w	r0, #4294967295	; 0xffffffff
    8168:	f000 f919 	bl	839e <HAL_NVIC_SetPriority>
    uwTickPrio = TickPriority;
    816c:	4a06      	ldr	r2, [pc, #24]	; (8188 <HAL_InitTick+0x5c>)
    816e:	687b      	ldr	r3, [r7, #4]
    8170:	6013      	str	r3, [r2, #0]
  {
    return HAL_ERROR;
  }

  /* Return function status */
  return HAL_OK;
    8172:	2300      	movs	r3, #0
    8174:	e000      	b.n	8178 <HAL_InitTick+0x4c>
    return HAL_ERROR;
    8176:	2301      	movs	r3, #1
}
    8178:	4618      	mov	r0, r3
    817a:	3708      	adds	r7, #8
    817c:	46bd      	mov	sp, r7
    817e:	bd80      	pop	{r7, pc}
    8180:	0001d2c4 	.word	0x0001d2c4
    8184:	0001d1b0 	.word	0x0001d1b0
    8188:	0001d1ac 	.word	0x0001d1ac

0000818c <HAL_GetTick>:
  * @note This function is declared as __weak to be overwritten in case of other 
  *       implementations in user file.
  * @retval tick value
  */
__weak uint32_t HAL_GetTick(void)
{
    818c:	b480      	push	{r7}
    818e:	af00      	add	r7, sp, #0
  return uwTick;
    8190:	4b03      	ldr	r3, [pc, #12]	; (81a0 <HAL_GetTick+0x14>)
    8192:	681b      	ldr	r3, [r3, #0]
}
    8194:	4618      	mov	r0, r3
    8196:	46bd      	mov	sp, r7
    8198:	f85d 7b04 	ldr.w	r7, [sp], #4
    819c:	4770      	bx	lr
    819e:	bf00      	nop
    81a0:	0001d3b4 	.word	0x0001d3b4

000081a4 <HAL_Delay>:
  *       implementations in user file.
  * @param Delay specifies the delay time length, in milliseconds.
  * @retval None
  */
__weak void HAL_Delay(uint32_t Delay)
{
    81a4:	b580      	push	{r7, lr}
    81a6:	b084      	sub	sp, #16
    81a8:	af00      	add	r7, sp, #0
    81aa:	6078      	str	r0, [r7, #4]
  uint32_t tickstart = HAL_GetTick();
    81ac:	f7ff ffee 	bl	818c <HAL_GetTick>
    81b0:	60b8      	str	r0, [r7, #8]
  uint32_t wait = Delay;
    81b2:	687b      	ldr	r3, [r7, #4]
    81b4:	60fb      	str	r3, [r7, #12]

  /* Add a freq to guarantee minimum wait */
  if (wait < HAL_MAX_DELAY)
    81b6:	68fb      	ldr	r3, [r7, #12]
    81b8:	f1b3 3fff 	cmp.w	r3, #4294967295	; 0xffffffff
    81bc:	d005      	beq.n	81ca <HAL_Delay+0x26>
  {
    wait += (uint32_t)(uwTickFreq);
    81be:	4b09      	ldr	r3, [pc, #36]	; (81e4 <HAL_Delay+0x40>)
    81c0:	781b      	ldrb	r3, [r3, #0]
    81c2:	461a      	mov	r2, r3
    81c4:	68fb      	ldr	r3, [r7, #12]
    81c6:	4413      	add	r3, r2
    81c8:	60fb      	str	r3, [r7, #12]
  }

  while((HAL_GetTick() - tickstart) < wait)
    81ca:	bf00      	nop
    81cc:	f7ff ffde 	bl	818c <HAL_GetTick>
    81d0:	4602      	mov	r2, r0
    81d2:	68bb      	ldr	r3, [r7, #8]
    81d4:	1ad3      	subs	r3, r2, r3
    81d6:	68fa      	ldr	r2, [r7, #12]
    81d8:	429a      	cmp	r2, r3
    81da:	d8f7      	bhi.n	81cc <HAL_Delay+0x28>
  {
  }
}
    81dc:	bf00      	nop
    81de:	3710      	adds	r7, #16
    81e0:	46bd      	mov	sp, r7
    81e2:	bd80      	pop	{r7, pc}
    81e4:	0001d1b0 	.word	0x0001d1b0

000081e8 <__NVIC_SetPriorityGrouping>:
           In case of a conflict between priority grouping and available
           priority bits (__NVIC_PRIO_BITS), the smallest possible priority group is set.
  \param [in]      PriorityGroup  Priority grouping field.
 */
__STATIC_INLINE void __NVIC_SetPriorityGrouping(uint32_t PriorityGroup)
{
    81e8:	b480      	push	{r7}
    81ea:	b085      	sub	sp, #20
    81ec:	af00      	add	r7, sp, #0
    81ee:	6078      	str	r0, [r7, #4]
  uint32_t reg_value;
  uint32_t PriorityGroupTmp = (PriorityGroup & (uint32_t)0x07UL);             /* only values 0..7 are used          */
    81f0:	687b      	ldr	r3, [r7, #4]
    81f2:	f003 0307 	and.w	r3, r3, #7
    81f6:	60fb      	str	r3, [r7, #12]

  reg_value  =  SCB->AIRCR;                                                   /* read old register configuration    */
    81f8:	4b0c      	ldr	r3, [pc, #48]	; (822c <__NVIC_SetPriorityGrouping+0x44>)
    81fa:	68db      	ldr	r3, [r3, #12]
    81fc:	60bb      	str	r3, [r7, #8]
  reg_value &= ~((uint32_t)(SCB_AIRCR_VECTKEY_Msk | SCB_AIRCR_PRIGROUP_Msk)); /* clear bits to change               */
    81fe:	68ba      	ldr	r2, [r7, #8]
    8200:	f64f 03ff 	movw	r3, #63743	; 0xf8ff
    8204:	4013      	ands	r3, r2
    8206:	60bb      	str	r3, [r7, #8]
  reg_value  =  (reg_value                                   |
                ((uint32_t)0x5FAUL << SCB_AIRCR_VECTKEY_Pos) |
                (PriorityGroupTmp << SCB_AIRCR_PRIGROUP_Pos)  );              /* Insert write key and priority group */
    8208:	68fb      	ldr	r3, [r7, #12]
    820a:	021a      	lsls	r2, r3, #8
                ((uint32_t)0x5FAUL << SCB_AIRCR_VECTKEY_Pos) |
    820c:	68bb      	ldr	r3, [r7, #8]
    820e:	4313      	orrs	r3, r2
  reg_value  =  (reg_value                                   |
    8210:	f043 63bf 	orr.w	r3, r3, #100139008	; 0x5f80000
    8214:	f443 3300 	orr.w	r3, r3, #131072	; 0x20000
    8218:	60bb      	str	r3, [r7, #8]
  SCB->AIRCR =  reg_value;
    821a:	4a04      	ldr	r2, [pc, #16]	; (822c <__NVIC_SetPriorityGrouping+0x44>)
    821c:	68bb      	ldr	r3, [r7, #8]
    821e:	60d3      	str	r3, [r2, #12]
}
    8220:	bf00      	nop
    8222:	3714      	adds	r7, #20
    8224:	46bd      	mov	sp, r7
    8226:	f85d 7b04 	ldr.w	r7, [sp], #4
    822a:	4770      	bx	lr
    822c:	e000ed00 	.word	0xe000ed00

00008230 <__NVIC_GetPriorityGrouping>:
  \brief   Get Priority Grouping
  \details Reads the priority grouping field from the NVIC Interrupt Controller.
  \return                Priority grouping field (SCB->AIRCR [10:8] PRIGROUP field).
 */
__STATIC_INLINE uint32_t __NVIC_GetPriorityGrouping(void)
{
    8230:	b480      	push	{r7}
    8232:	af00      	add	r7, sp, #0
  return ((uint32_t)((SCB->AIRCR & SCB_AIRCR_PRIGROUP_Msk) >> SCB_AIRCR_PRIGROUP_Pos));
    8234:	4b04      	ldr	r3, [pc, #16]	; (8248 <__NVIC_GetPriorityGrouping+0x18>)
    8236:	68db      	ldr	r3, [r3, #12]
    8238:	0a1b      	lsrs	r3, r3, #8
    823a:	f003 0307 	and.w	r3, r3, #7
}
    823e:	4618      	mov	r0, r3
    8240:	46bd      	mov	sp, r7
    8242:	f85d 7b04 	ldr.w	r7, [sp], #4
    8246:	4770      	bx	lr
    8248:	e000ed00 	.word	0xe000ed00

0000824c <__NVIC_EnableIRQ>:
  \details Enables a device specific interrupt in the NVIC interrupt controller.
  \param [in]      IRQn  Device specific interrupt number.
  \note    IRQn must not be negative.
 */
__STATIC_INLINE void __NVIC_EnableIRQ(IRQn_Type IRQn)
{
    824c:	b480      	push	{r7}
    824e:	b083      	sub	sp, #12
    8250:	af00      	add	r7, sp, #0
    8252:	4603      	mov	r3, r0
    8254:	71fb      	strb	r3, [r7, #7]
  if ((int32_t)(IRQn) >= 0)
    8256:	f997 3007 	ldrsb.w	r3, [r7, #7]
    825a:	2b00      	cmp	r3, #0
    825c:	db0b      	blt.n	8276 <__NVIC_EnableIRQ+0x2a>
  {
    NVIC->ISER[(((uint32_t)IRQn) >> 5UL)] = (uint32_t)(1UL << (((uint32_t)IRQn) & 0x1FUL));
    825e:	79fb      	ldrb	r3, [r7, #7]
    8260:	f003 021f 	and.w	r2, r3, #31
    8264:	4907      	ldr	r1, [pc, #28]	; (8284 <__NVIC_EnableIRQ+0x38>)
    8266:	f997 3007 	ldrsb.w	r3, [r7, #7]
    826a:	095b      	lsrs	r3, r3, #5
    826c:	2001      	movs	r0, #1
    826e:	fa00 f202 	lsl.w	r2, r0, r2
    8272:	f841 2023 	str.w	r2, [r1, r3, lsl #2]
  }
}
    8276:	bf00      	nop
    8278:	370c      	adds	r7, #12
    827a:	46bd      	mov	sp, r7
    827c:	f85d 7b04 	ldr.w	r7, [sp], #4
    8280:	4770      	bx	lr
    8282:	bf00      	nop
    8284:	e000e100 	.word	0xe000e100

00008288 <__NVIC_SetPriority>:
  \param [in]      IRQn  Interrupt number.
  \param [in]  priority  Priority to set.
  \note    The priority cannot be set for every processor exception.
 */
__STATIC_INLINE void __NVIC_SetPriority(IRQn_Type IRQn, uint32_t priority)
{
    8288:	b480      	push	{r7}
    828a:	b083      	sub	sp, #12
    828c:	af00      	add	r7, sp, #0
    828e:	4603      	mov	r3, r0
    8290:	6039      	str	r1, [r7, #0]
    8292:	71fb      	strb	r3, [r7, #7]
  if ((int32_t)(IRQn) >= 0)
    8294:	f997 3007 	ldrsb.w	r3, [r7, #7]
    8298:	2b00      	cmp	r3, #0
    829a:	db0a      	blt.n	82b2 <__NVIC_SetPriority+0x2a>
  {
    NVIC->IP[((uint32_t)IRQn)]               = (uint8_t)((priority << (8U - __NVIC_PRIO_BITS)) & (uint32_t)0xFFUL);
    829c:	683b      	ldr	r3, [r7, #0]
    829e:	b2da      	uxtb	r2, r3
    82a0:	490c      	ldr	r1, [pc, #48]	; (82d4 <__NVIC_SetPriority+0x4c>)
    82a2:	f997 3007 	ldrsb.w	r3, [r7, #7]
    82a6:	0112      	lsls	r2, r2, #4
    82a8:	b2d2      	uxtb	r2, r2
    82aa:	440b      	add	r3, r1
    82ac:	f883 2300 	strb.w	r2, [r3, #768]	; 0x300
  }
  else
  {
    SCB->SHP[(((uint32_t)IRQn) & 0xFUL)-4UL] = (uint8_t)((priority << (8U - __NVIC_PRIO_BITS)) & (uint32_t)0xFFUL);
  }
}
    82b0:	e00a      	b.n	82c8 <__NVIC_SetPriority+0x40>
    SCB->SHP[(((uint32_t)IRQn) & 0xFUL)-4UL] = (uint8_t)((priority << (8U - __NVIC_PRIO_BITS)) & (uint32_t)0xFFUL);
    82b2:	683b      	ldr	r3, [r7, #0]
    82b4:	b2da      	uxtb	r2, r3
    82b6:	4908      	ldr	r1, [pc, #32]	; (82d8 <__NVIC_SetPriority+0x50>)
    82b8:	79fb      	ldrb	r3, [r7, #7]
    82ba:	f003 030f 	and.w	r3, r3, #15
    82be:	3b04      	subs	r3, #4
    82c0:	0112      	lsls	r2, r2, #4
    82c2:	b2d2      	uxtb	r2, r2
    82c4:	440b      	add	r3, r1
    82c6:	761a      	strb	r2, [r3, #24]
}
    82c8:	bf00      	nop
    82ca:	370c      	adds	r7, #12
    82cc:	46bd      	mov	sp, r7
    82ce:	f85d 7b04 	ldr.w	r7, [sp], #4
    82d2:	4770      	bx	lr
    82d4:	e000e100 	.word	0xe000e100
    82d8:	e000ed00 	.word	0xe000ed00

000082dc <NVIC_EncodePriority>:
  \param [in]   PreemptPriority  Preemptive priority value (starting from 0).
  \param [in]       SubPriority  Subpriority value (starting from 0).
  \return                        Encoded priority. Value can be used in the function \ref NVIC_SetPriority().
 */
__STATIC_INLINE uint32_t NVIC_EncodePriority (uint32_t PriorityGroup, uint32_t PreemptPriority, uint32_t SubPriority)
{
    82dc:	b480      	push	{r7}
    82de:	b089      	sub	sp, #36	; 0x24
    82e0:	af00      	add	r7, sp, #0
    82e2:	60f8      	str	r0, [r7, #12]
    82e4:	60b9      	str	r1, [r7, #8]
    82e6:	607a      	str	r2, [r7, #4]
  uint32_t PriorityGroupTmp = (PriorityGroup & (uint32_t)0x07UL);   /* only values 0..7 are used          */
    82e8:	68fb      	ldr	r3, [r7, #12]
    82ea:	f003 0307 	and.w	r3, r3, #7
    82ee:	61fb      	str	r3, [r7, #28]
  uint32_t PreemptPriorityBits;
  uint32_t SubPriorityBits;

  PreemptPriorityBits = ((7UL - PriorityGroupTmp) > (uint32_t)(__NVIC_PRIO_BITS)) ? (uint32_t)(__NVIC_PRIO_BITS) : (uint32_t)(7UL - PriorityGroupTmp);
    82f0:	69fb      	ldr	r3, [r7, #28]
    82f2:	f1c3 0307 	rsb	r3, r3, #7
    82f6:	2b04      	cmp	r3, #4
    82f8:	bf28      	it	cs
    82fa:	2304      	movcs	r3, #4
    82fc:	61bb      	str	r3, [r7, #24]
  SubPriorityBits     = ((PriorityGroupTmp + (uint32_t)(__NVIC_PRIO_BITS)) < (uint32_t)7UL) ? (uint32_t)0UL : (uint32_t)((PriorityGroupTmp - 7UL) + (uint32_t)(__NVIC_PRIO_BITS));
    82fe:	69fb      	ldr	r3, [r7, #28]
    8300:	3304      	adds	r3, #4
    8302:	2b06      	cmp	r3, #6
    8304:	d902      	bls.n	830c <NVIC_EncodePriority+0x30>
    8306:	69fb      	ldr	r3, [r7, #28]
    8308:	3b03      	subs	r3, #3
    830a:	e000      	b.n	830e <NVIC_EncodePriority+0x32>
    830c:	2300      	movs	r3, #0
    830e:	617b      	str	r3, [r7, #20]

  return (
           ((PreemptPriority & (uint32_t)((1UL << (PreemptPriorityBits)) - 1UL)) << SubPriorityBits) |
    8310:	f04f 32ff 	mov.w	r2, #4294967295	; 0xffffffff
    8314:	69bb      	ldr	r3, [r7, #24]
    8316:	fa02 f303 	lsl.w	r3, r2, r3
    831a:	43da      	mvns	r2, r3
    831c:	68bb      	ldr	r3, [r7, #8]
    831e:	401a      	ands	r2, r3
    8320:	697b      	ldr	r3, [r7, #20]
    8322:	409a      	lsls	r2, r3
           ((SubPriority     & (uint32_t)((1UL << (SubPriorityBits    )) - 1UL)))
    8324:	f04f 31ff 	mov.w	r1, #4294967295	; 0xffffffff
    8328:	697b      	ldr	r3, [r7, #20]
    832a:	fa01 f303 	lsl.w	r3, r1, r3
    832e:	43d9      	mvns	r1, r3
    8330:	687b      	ldr	r3, [r7, #4]
    8332:	400b      	ands	r3, r1
           ((PreemptPriority & (uint32_t)((1UL << (PreemptPriorityBits)) - 1UL)) << SubPriorityBits) |
    8334:	4313      	orrs	r3, r2
         );
}
    8336:	4618      	mov	r0, r3
    8338:	3724      	adds	r7, #36	; 0x24
    833a:	46bd      	mov	sp, r7
    833c:	f85d 7b04 	ldr.w	r7, [sp], #4
    8340:	4770      	bx	lr
	...

00008344 <SysTick_Config>:
  \note    When the variable <b>__Vendor_SysTickConfig</b> is set to 1, then the
           function <b>SysTick_Config</b> is not included. In this case, the file <b><i>device</i>.h</b>
           must contain a vendor-specific implementation of this function.
 */
__STATIC_INLINE uint32_t SysTick_Config(uint32_t ticks)
{
    8344:	b580      	push	{r7, lr}
    8346:	b082      	sub	sp, #8
    8348:	af00      	add	r7, sp, #0
    834a:	6078      	str	r0, [r7, #4]
  if ((ticks - 1UL) > SysTick_LOAD_RELOAD_Msk)
    834c:	687b      	ldr	r3, [r7, #4]
    834e:	3b01      	subs	r3, #1
    8350:	f1b3 7f80 	cmp.w	r3, #16777216	; 0x1000000
    8354:	d301      	bcc.n	835a <SysTick_Config+0x16>
  {
    return (1UL);                                                   /* Reload value impossible */
    8356:	2301      	movs	r3, #1
    8358:	e00f      	b.n	837a <SysTick_Config+0x36>
  }

  SysTick->LOAD  = (uint32_t)(ticks - 1UL);                         /* set reload register */
    835a:	4a0a      	ldr	r2, [pc, #40]	; (8384 <SysTick_Config+0x40>)
    835c:	687b      	ldr	r3, [r7, #4]
    835e:	3b01      	subs	r3, #1
    8360:	6053      	str	r3, [r2, #4]
  NVIC_SetPriority (SysTick_IRQn, (1UL << __NVIC_PRIO_BITS) - 1UL); /* set Priority for Systick Interrupt */
    8362:	210f      	movs	r1, #15
    8364:	f04f 30ff 	mov.w	r0, #4294967295	; 0xffffffff
    8368:	f7ff ff8e 	bl	8288 <__NVIC_SetPriority>
  SysTick->VAL   = 0UL;                                             /* Load the SysTick Counter Value */
    836c:	4b05      	ldr	r3, [pc, #20]	; (8384 <SysTick_Config+0x40>)
    836e:	2200      	movs	r2, #0
    8370:	609a      	str	r2, [r3, #8]
  SysTick->CTRL  = SysTick_CTRL_CLKSOURCE_Msk |
    8372:	4b04      	ldr	r3, [pc, #16]	; (8384 <SysTick_Config+0x40>)
    8374:	2207      	movs	r2, #7
    8376:	601a      	str	r2, [r3, #0]
                   SysTick_CTRL_TICKINT_Msk   |
                   SysTick_CTRL_ENABLE_Msk;                         /* Enable SysTick IRQ and SysTick Timer */
  return (0UL);                                                     /* Function successful */
    8378:	2300      	movs	r3, #0
}
    837a:	4618      	mov	r0, r3
    837c:	3708      	adds	r7, #8
    837e:	46bd      	mov	sp, r7
    8380:	bd80      	pop	{r7, pc}
    8382:	bf00      	nop
    8384:	e000e010 	.word	0xe000e010

00008388 <HAL_NVIC_SetPriorityGrouping>:
  * @note   When the NVIC_PriorityGroup_0 is selected, IRQ preemption is no more possible. 
  *         The pending IRQ priority will be managed only by the subpriority. 
  * @retval None
  */
void HAL_NVIC_SetPriorityGrouping(uint32_t PriorityGroup)
{
    8388:	b580      	push	{r7, lr}
    838a:	b082      	sub	sp, #8
    838c:	af00      	add	r7, sp, #0
    838e:	6078      	str	r0, [r7, #4]
  /* Check the parameters */
  assert_param(IS_NVIC_PRIORITY_GROUP(PriorityGroup));
  
  /* Set the PRIGROUP[10:8] bits according to the PriorityGroup parameter value */
  NVIC_SetPriorityGrouping(PriorityGroup);
    8390:	6878      	ldr	r0, [r7, #4]
    8392:	f7ff ff29 	bl	81e8 <__NVIC_SetPriorityGrouping>
}
    8396:	bf00      	nop
    8398:	3708      	adds	r7, #8
    839a:	46bd      	mov	sp, r7
    839c:	bd80      	pop	{r7, pc}

0000839e <HAL_NVIC_SetPriority>:
  *         This parameter can be a value between 0 and 15
  *         A lower priority value indicates a higher priority.          
  * @retval None
  */
void HAL_NVIC_SetPriority(IRQn_Type IRQn, uint32_t PreemptPriority, uint32_t SubPriority)
{ 
    839e:	b580      	push	{r7, lr}
    83a0:	b086      	sub	sp, #24
    83a2:	af00      	add	r7, sp, #0
    83a4:	4603      	mov	r3, r0
    83a6:	60b9      	str	r1, [r7, #8]
    83a8:	607a      	str	r2, [r7, #4]
    83aa:	73fb      	strb	r3, [r7, #15]
  uint32_t prioritygroup = 0x00U;
    83ac:	2300      	movs	r3, #0
    83ae:	617b      	str	r3, [r7, #20]
  
  /* Check the parameters */
  assert_param(IS_NVIC_SUB_PRIORITY(SubPriority));
  assert_param(IS_NVIC_PREEMPTION_PRIORITY(PreemptPriority));
  
  prioritygroup = NVIC_GetPriorityGrouping();
    83b0:	f7ff ff3e 	bl	8230 <__NVIC_GetPriorityGrouping>
    83b4:	6178      	str	r0, [r7, #20]
  
  NVIC_SetPriority(IRQn, NVIC_EncodePriority(prioritygroup, PreemptPriority, SubPriority));
    83b6:	687a      	ldr	r2, [r7, #4]
    83b8:	68b9      	ldr	r1, [r7, #8]
    83ba:	6978      	ldr	r0, [r7, #20]
    83bc:	f7ff ff8e 	bl	82dc <NVIC_EncodePriority>
    83c0:	4602      	mov	r2, r0
    83c2:	f997 300f 	ldrsb.w	r3, [r7, #15]
    83c6:	4611      	mov	r1, r2
    83c8:	4618      	mov	r0, r3
    83ca:	f7ff ff5d 	bl	8288 <__NVIC_SetPriority>
}
    83ce:	bf00      	nop
    83d0:	3718      	adds	r7, #24
    83d2:	46bd      	mov	sp, r7
    83d4:	bd80      	pop	{r7, pc}

000083d6 <HAL_NVIC_EnableIRQ>:
  *         This parameter can be an enumerator of IRQn_Type enumeration
  *         (For the complete STM32 Devices IRQ Channels list, please refer to the appropriate CMSIS device file (stm32f4xxxx.h))
  * @retval None
  */
void HAL_NVIC_EnableIRQ(IRQn_Type IRQn)
{
    83d6:	b580      	push	{r7, lr}
    83d8:	b082      	sub	sp, #8
    83da:	af00      	add	r7, sp, #0
    83dc:	4603      	mov	r3, r0
    83de:	71fb      	strb	r3, [r7, #7]
  /* Check the parameters */
  assert_param(IS_NVIC_DEVICE_IRQ(IRQn));
  
  /* Enable interrupt */
  NVIC_EnableIRQ(IRQn);
    83e0:	f997 3007 	ldrsb.w	r3, [r7, #7]
    83e4:	4618      	mov	r0, r3
    83e6:	f7ff ff31 	bl	824c <__NVIC_EnableIRQ>
}
    83ea:	bf00      	nop
    83ec:	3708      	adds	r7, #8
    83ee:	46bd      	mov	sp, r7
    83f0:	bd80      	pop	{r7, pc}

000083f2 <HAL_SYSTICK_Config>:
  * @param  TicksNumb Specifies the ticks Number of ticks between two interrupts.
  * @retval status:  - 0  Function succeeded.
  *                  - 1  Function failed.
  */
uint32_t HAL_SYSTICK_Config(uint32_t TicksNumb)
{
    83f2:	b580      	push	{r7, lr}
    83f4:	b082      	sub	sp, #8
    83f6:	af00      	add	r7, sp, #0
    83f8:	6078      	str	r0, [r7, #4]
   return SysTick_Config(TicksNumb);
    83fa:	6878      	ldr	r0, [r7, #4]
    83fc:	f7ff ffa2 	bl	8344 <SysTick_Config>
    8400:	4603      	mov	r3, r0
}
    8402:	4618      	mov	r0, r3
    8404:	3708      	adds	r7, #8
    8406:	46bd      	mov	sp, r7
    8408:	bd80      	pop	{r7, pc}
	...

0000840c <HAL_GPIO_Init>:
  * @param  GPIO_Init pointer to a GPIO_InitTypeDef structure that contains
  *         the configuration information for the specified GPIO peripheral.
  * @retval None
  */
void HAL_GPIO_Init(GPIO_TypeDef  *GPIOx, GPIO_InitTypeDef *GPIO_Init)
{
    840c:	b480      	push	{r7}
    840e:	b089      	sub	sp, #36	; 0x24
    8410:	af00      	add	r7, sp, #0
    8412:	6078      	str	r0, [r7, #4]
    8414:	6039      	str	r1, [r7, #0]
  uint32_t position;
  uint32_t ioposition = 0x00U;
    8416:	2300      	movs	r3, #0
    8418:	617b      	str	r3, [r7, #20]
  uint32_t iocurrent = 0x00U;
    841a:	2300      	movs	r3, #0
    841c:	613b      	str	r3, [r7, #16]
  uint32_t temp = 0x00U;
    841e:	2300      	movs	r3, #0
    8420:	61bb      	str	r3, [r7, #24]
  assert_param(IS_GPIO_PIN(GPIO_Init->Pin));
  assert_param(IS_GPIO_MODE(GPIO_Init->Mode));
  assert_param(IS_GPIO_PULL(GPIO_Init->Pull));

  /* Configure the port pins */
  for(position = 0U; position < GPIO_NUMBER; position++)
    8422:	2300      	movs	r3, #0
    8424:	61fb      	str	r3, [r7, #28]
    8426:	e16b      	b.n	8700 <HAL_GPIO_Init+0x2f4>
  {
    /* Get the IO position */
    ioposition = 0x01U << position;
    8428:	2201      	movs	r2, #1
    842a:	69fb      	ldr	r3, [r7, #28]
    842c:	fa02 f303 	lsl.w	r3, r2, r3
    8430:	617b      	str	r3, [r7, #20]
    /* Get the current IO position */
    iocurrent = (uint32_t)(GPIO_Init->Pin) & ioposition;
    8432:	683b      	ldr	r3, [r7, #0]
    8434:	681b      	ldr	r3, [r3, #0]
    8436:	697a      	ldr	r2, [r7, #20]
    8438:	4013      	ands	r3, r2
    843a:	613b      	str	r3, [r7, #16]

    if(iocurrent == ioposition)
    843c:	693a      	ldr	r2, [r7, #16]
    843e:	697b      	ldr	r3, [r7, #20]
    8440:	429a      	cmp	r2, r3
    8442:	f040 815a 	bne.w	86fa <HAL_GPIO_Init+0x2ee>
    {
      /*--------------------- GPIO Mode Configuration ------------------------*/
      /* In case of Alternate function mode selection */
      if((GPIO_Init->Mode == GPIO_MODE_AF_PP) || (GPIO_Init->Mode == GPIO_MODE_AF_OD))
    8446:	683b      	ldr	r3, [r7, #0]
    8448:	685b      	ldr	r3, [r3, #4]
    844a:	2b02      	cmp	r3, #2
    844c:	d003      	beq.n	8456 <HAL_GPIO_Init+0x4a>
    844e:	683b      	ldr	r3, [r7, #0]
    8450:	685b      	ldr	r3, [r3, #4]
    8452:	2b12      	cmp	r3, #18
    8454:	d123      	bne.n	849e <HAL_GPIO_Init+0x92>
      {
        /* Check the Alternate function parameter */
        assert_param(IS_GPIO_AF(GPIO_Init->Alternate));
        /* Configure Alternate function mapped with the current IO */
        temp = GPIOx->AFR[position >> 3U];
    8456:	69fb      	ldr	r3, [r7, #28]
    8458:	08da      	lsrs	r2, r3, #3
    845a:	687b      	ldr	r3, [r7, #4]
    845c:	3208      	adds	r2, #8
    845e:	f853 3022 	ldr.w	r3, [r3, r2, lsl #2]
    8462:	61bb      	str	r3, [r7, #24]
        temp &= ~(0xFU << ((uint32_t)(position & 0x07U) * 4U)) ;
    8464:	69fb      	ldr	r3, [r7, #28]
    8466:	f003 0307 	and.w	r3, r3, #7
    846a:	009b      	lsls	r3, r3, #2
    846c:	220f      	movs	r2, #15
    846e:	fa02 f303 	lsl.w	r3, r2, r3
    8472:	43db      	mvns	r3, r3
    8474:	69ba      	ldr	r2, [r7, #24]
    8476:	4013      	ands	r3, r2
    8478:	61bb      	str	r3, [r7, #24]
        temp |= ((uint32_t)(GPIO_Init->Alternate) << (((uint32_t)position & 0x07U) * 4U));
    847a:	683b      	ldr	r3, [r7, #0]
    847c:	691a      	ldr	r2, [r3, #16]
    847e:	69fb      	ldr	r3, [r7, #28]
    8480:	f003 0307 	and.w	r3, r3, #7
    8484:	009b      	lsls	r3, r3, #2
    8486:	fa02 f303 	lsl.w	r3, r2, r3
    848a:	69ba      	ldr	r2, [r7, #24]
    848c:	4313      	orrs	r3, r2
    848e:	61bb      	str	r3, [r7, #24]
        GPIOx->AFR[position >> 3U] = temp;
    8490:	69fb      	ldr	r3, [r7, #28]
    8492:	08da      	lsrs	r2, r3, #3
    8494:	687b      	ldr	r3, [r7, #4]
    8496:	3208      	adds	r2, #8
    8498:	69b9      	ldr	r1, [r7, #24]
    849a:	f843 1022 	str.w	r1, [r3, r2, lsl #2]
      }

      /* Configure IO Direction mode (Input, Output, Alternate or Analog) */
      temp = GPIOx->MODER;
    849e:	687b      	ldr	r3, [r7, #4]
    84a0:	681b      	ldr	r3, [r3, #0]
    84a2:	61bb      	str	r3, [r7, #24]
      temp &= ~(GPIO_MODER_MODER0 << (position * 2U));
    84a4:	69fb      	ldr	r3, [r7, #28]
    84a6:	005b      	lsls	r3, r3, #1
    84a8:	2203      	movs	r2, #3
    84aa:	fa02 f303 	lsl.w	r3, r2, r3
    84ae:	43db      	mvns	r3, r3
    84b0:	69ba      	ldr	r2, [r7, #24]
    84b2:	4013      	ands	r3, r2
    84b4:	61bb      	str	r3, [r7, #24]
      temp |= ((GPIO_Init->Mode & GPIO_MODE) << (position * 2U));
    84b6:	683b      	ldr	r3, [r7, #0]
    84b8:	685b      	ldr	r3, [r3, #4]
    84ba:	f003 0203 	and.w	r2, r3, #3
    84be:	69fb      	ldr	r3, [r7, #28]
    84c0:	005b      	lsls	r3, r3, #1
    84c2:	fa02 f303 	lsl.w	r3, r2, r3
    84c6:	69ba      	ldr	r2, [r7, #24]
    84c8:	4313      	orrs	r3, r2
    84ca:	61bb      	str	r3, [r7, #24]
      GPIOx->MODER = temp;
    84cc:	687b      	ldr	r3, [r7, #4]
    84ce:	69ba      	ldr	r2, [r7, #24]
    84d0:	601a      	str	r2, [r3, #0]

      /* In case of Output or Alternate function mode selection */
      if((GPIO_Init->Mode == GPIO_MODE_OUTPUT_PP) || (GPIO_Init->Mode == GPIO_MODE_AF_PP) ||
    84d2:	683b      	ldr	r3, [r7, #0]
    84d4:	685b      	ldr	r3, [r3, #4]
    84d6:	2b01      	cmp	r3, #1
    84d8:	d00b      	beq.n	84f2 <HAL_GPIO_Init+0xe6>
    84da:	683b      	ldr	r3, [r7, #0]
    84dc:	685b      	ldr	r3, [r3, #4]
    84de:	2b02      	cmp	r3, #2
    84e0:	d007      	beq.n	84f2 <HAL_GPIO_Init+0xe6>
         (GPIO_Init->Mode == GPIO_MODE_OUTPUT_OD) || (GPIO_Init->Mode == GPIO_MODE_AF_OD))
    84e2:	683b      	ldr	r3, [r7, #0]
    84e4:	685b      	ldr	r3, [r3, #4]
      if((GPIO_Init->Mode == GPIO_MODE_OUTPUT_PP) || (GPIO_Init->Mode == GPIO_MODE_AF_PP) ||
    84e6:	2b11      	cmp	r3, #17
    84e8:	d003      	beq.n	84f2 <HAL_GPIO_Init+0xe6>
         (GPIO_Init->Mode == GPIO_MODE_OUTPUT_OD) || (GPIO_Init->Mode == GPIO_MODE_AF_OD))
    84ea:	683b      	ldr	r3, [r7, #0]
    84ec:	685b      	ldr	r3, [r3, #4]
    84ee:	2b12      	cmp	r3, #18
    84f0:	d130      	bne.n	8554 <HAL_GPIO_Init+0x148>
      {
        /* Check the Speed parameter */
        assert_param(IS_GPIO_SPEED(GPIO_Init->Speed));
        /* Configure the IO Speed */
        temp = GPIOx->OSPEEDR; 
    84f2:	687b      	ldr	r3, [r7, #4]
    84f4:	689b      	ldr	r3, [r3, #8]
    84f6:	61bb      	str	r3, [r7, #24]
        temp &= ~(GPIO_OSPEEDER_OSPEEDR0 << (position * 2U));
    84f8:	69fb      	ldr	r3, [r7, #28]
    84fa:	005b      	lsls	r3, r3, #1
    84fc:	2203      	movs	r2, #3
    84fe:	fa02 f303 	lsl.w	r3, r2, r3
    8502:	43db      	mvns	r3, r3
    8504:	69ba      	ldr	r2, [r7, #24]
    8506:	4013      	ands	r3, r2
    8508:	61bb      	str	r3, [r7, #24]
        temp |= (GPIO_Init->Speed << (position * 2U));
    850a:	683b      	ldr	r3, [r7, #0]
    850c:	68da      	ldr	r2, [r3, #12]
    850e:	69fb      	ldr	r3, [r7, #28]
    8510:	005b      	lsls	r3, r3, #1
    8512:	fa02 f303 	lsl.w	r3, r2, r3
    8516:	69ba      	ldr	r2, [r7, #24]
    8518:	4313      	orrs	r3, r2
    851a:	61bb      	str	r3, [r7, #24]
        GPIOx->OSPEEDR = temp;
    851c:	687b      	ldr	r3, [r7, #4]
    851e:	69ba      	ldr	r2, [r7, #24]
    8520:	609a      	str	r2, [r3, #8]

        /* Configure the IO Output Type */
        temp = GPIOx->OTYPER;
    8522:	687b      	ldr	r3, [r7, #4]
    8524:	685b      	ldr	r3, [r3, #4]
    8526:	61bb      	str	r3, [r7, #24]
        temp &= ~(GPIO_OTYPER_OT_0 << position) ;
    8528:	2201      	movs	r2, #1
    852a:	69fb      	ldr	r3, [r7, #28]
    852c:	fa02 f303 	lsl.w	r3, r2, r3
    8530:	43db      	mvns	r3, r3
    8532:	69ba      	ldr	r2, [r7, #24]
    8534:	4013      	ands	r3, r2
    8536:	61bb      	str	r3, [r7, #24]
        temp |= (((GPIO_Init->Mode & GPIO_OUTPUT_TYPE) >> 4U) << position);
    8538:	683b      	ldr	r3, [r7, #0]
    853a:	685b      	ldr	r3, [r3, #4]
    853c:	091b      	lsrs	r3, r3, #4
    853e:	f003 0201 	and.w	r2, r3, #1
    8542:	69fb      	ldr	r3, [r7, #28]
    8544:	fa02 f303 	lsl.w	r3, r2, r3
    8548:	69ba      	ldr	r2, [r7, #24]
    854a:	4313      	orrs	r3, r2
    854c:	61bb      	str	r3, [r7, #24]
        GPIOx->OTYPER = temp;
    854e:	687b      	ldr	r3, [r7, #4]
    8550:	69ba      	ldr	r2, [r7, #24]
    8552:	605a      	str	r2, [r3, #4]
      }

      /* Activate the Pull-up or Pull down resistor for the current IO */
      temp = GPIOx->PUPDR;
    8554:	687b      	ldr	r3, [r7, #4]
    8556:	68db      	ldr	r3, [r3, #12]
    8558:	61bb      	str	r3, [r7, #24]
      temp &= ~(GPIO_PUPDR_PUPDR0 << (position * 2U));
    855a:	69fb      	ldr	r3, [r7, #28]
    855c:	005b      	lsls	r3, r3, #1
    855e:	2203      	movs	r2, #3
    8560:	fa02 f303 	lsl.w	r3, r2, r3
    8564:	43db      	mvns	r3, r3
    8566:	69ba      	ldr	r2, [r7, #24]
    8568:	4013      	ands	r3, r2
    856a:	61bb      	str	r3, [r7, #24]
      temp |= ((GPIO_Init->Pull) << (position * 2U));
    856c:	683b      	ldr	r3, [r7, #0]
    856e:	689a      	ldr	r2, [r3, #8]
    8570:	69fb      	ldr	r3, [r7, #28]
    8572:	005b      	lsls	r3, r3, #1
    8574:	fa02 f303 	lsl.w	r3, r2, r3
    8578:	69ba      	ldr	r2, [r7, #24]
    857a:	4313      	orrs	r3, r2
    857c:	61bb      	str	r3, [r7, #24]
      GPIOx->PUPDR = temp;
    857e:	687b      	ldr	r3, [r7, #4]
    8580:	69ba      	ldr	r2, [r7, #24]
    8582:	60da      	str	r2, [r3, #12]

      /*--------------------- EXTI Mode Configuration ------------------------*/
      /* Configure the External Interrupt or event for the current IO */
      if((GPIO_Init->Mode & EXTI_MODE) == EXTI_MODE)
    8584:	683b      	ldr	r3, [r7, #0]
    8586:	685b      	ldr	r3, [r3, #4]
    8588:	f003 5380 	and.w	r3, r3, #268435456	; 0x10000000
    858c:	2b00      	cmp	r3, #0
    858e:	f000 80b4 	beq.w	86fa <HAL_GPIO_Init+0x2ee>
      {
        /* Enable SYSCFG Clock */
        __HAL_RCC_SYSCFG_CLK_ENABLE();
    8592:	2300      	movs	r3, #0
    8594:	60fb      	str	r3, [r7, #12]
    8596:	4b5f      	ldr	r3, [pc, #380]	; (8714 <HAL_GPIO_Init+0x308>)
    8598:	6c5b      	ldr	r3, [r3, #68]	; 0x44
    859a:	4a5e      	ldr	r2, [pc, #376]	; (8714 <HAL_GPIO_Init+0x308>)
    859c:	f443 4380 	orr.w	r3, r3, #16384	; 0x4000
    85a0:	6453      	str	r3, [r2, #68]	; 0x44
    85a2:	4b5c      	ldr	r3, [pc, #368]	; (8714 <HAL_GPIO_Init+0x308>)
    85a4:	6c5b      	ldr	r3, [r3, #68]	; 0x44
    85a6:	f403 4380 	and.w	r3, r3, #16384	; 0x4000
    85aa:	60fb      	str	r3, [r7, #12]
    85ac:	68fb      	ldr	r3, [r7, #12]

        temp = SYSCFG->EXTICR[position >> 2U];
    85ae:	4a5a      	ldr	r2, [pc, #360]	; (8718 <HAL_GPIO_Init+0x30c>)
    85b0:	69fb      	ldr	r3, [r7, #28]
    85b2:	089b      	lsrs	r3, r3, #2
    85b4:	3302      	adds	r3, #2
    85b6:	f852 3023 	ldr.w	r3, [r2, r3, lsl #2]
    85ba:	61bb      	str	r3, [r7, #24]
        temp &= ~(0x0FU << (4U * (position & 0x03U)));
    85bc:	69fb      	ldr	r3, [r7, #28]
    85be:	f003 0303 	and.w	r3, r3, #3
    85c2:	009b      	lsls	r3, r3, #2
    85c4:	220f      	movs	r2, #15
    85c6:	fa02 f303 	lsl.w	r3, r2, r3
    85ca:	43db      	mvns	r3, r3
    85cc:	69ba      	ldr	r2, [r7, #24]
    85ce:	4013      	ands	r3, r2
    85d0:	61bb      	str	r3, [r7, #24]
        temp |= ((uint32_t)(GPIO_GET_INDEX(GPIOx)) << (4U * (position & 0x03U)));
    85d2:	687b      	ldr	r3, [r7, #4]
    85d4:	4a51      	ldr	r2, [pc, #324]	; (871c <HAL_GPIO_Init+0x310>)
    85d6:	4293      	cmp	r3, r2
    85d8:	d02b      	beq.n	8632 <HAL_GPIO_Init+0x226>
    85da:	687b      	ldr	r3, [r7, #4]
    85dc:	4a50      	ldr	r2, [pc, #320]	; (8720 <HAL_GPIO_Init+0x314>)
    85de:	4293      	cmp	r3, r2
    85e0:	d025      	beq.n	862e <HAL_GPIO_Init+0x222>
    85e2:	687b      	ldr	r3, [r7, #4]
    85e4:	4a4f      	ldr	r2, [pc, #316]	; (8724 <HAL_GPIO_Init+0x318>)
    85e6:	4293      	cmp	r3, r2
    85e8:	d01f      	beq.n	862a <HAL_GPIO_Init+0x21e>
    85ea:	687b      	ldr	r3, [r7, #4]
    85ec:	4a4e      	ldr	r2, [pc, #312]	; (8728 <HAL_GPIO_Init+0x31c>)
    85ee:	4293      	cmp	r3, r2
    85f0:	d019      	beq.n	8626 <HAL_GPIO_Init+0x21a>
    85f2:	687b      	ldr	r3, [r7, #4]
    85f4:	4a4d      	ldr	r2, [pc, #308]	; (872c <HAL_GPIO_Init+0x320>)
    85f6:	4293      	cmp	r3, r2
    85f8:	d013      	beq.n	8622 <HAL_GPIO_Init+0x216>
    85fa:	687b      	ldr	r3, [r7, #4]
    85fc:	4a4c      	ldr	r2, [pc, #304]	; (8730 <HAL_GPIO_Init+0x324>)
    85fe:	4293      	cmp	r3, r2
    8600:	d00d      	beq.n	861e <HAL_GPIO_Init+0x212>
    8602:	687b      	ldr	r3, [r7, #4]
    8604:	4a4b      	ldr	r2, [pc, #300]	; (8734 <HAL_GPIO_Init+0x328>)
    8606:	4293      	cmp	r3, r2
    8608:	d007      	beq.n	861a <HAL_GPIO_Init+0x20e>
    860a:	687b      	ldr	r3, [r7, #4]
    860c:	4a4a      	ldr	r2, [pc, #296]	; (8738 <HAL_GPIO_Init+0x32c>)
    860e:	4293      	cmp	r3, r2
    8610:	d101      	bne.n	8616 <HAL_GPIO_Init+0x20a>
    8612:	2307      	movs	r3, #7
    8614:	e00e      	b.n	8634 <HAL_GPIO_Init+0x228>
    8616:	2308      	movs	r3, #8
    8618:	e00c      	b.n	8634 <HAL_GPIO_Init+0x228>
    861a:	2306      	movs	r3, #6
    861c:	e00a      	b.n	8634 <HAL_GPIO_Init+0x228>
    861e:	2305      	movs	r3, #5
    8620:	e008      	b.n	8634 <HAL_GPIO_Init+0x228>
    8622:	2304      	movs	r3, #4
    8624:	e006      	b.n	8634 <HAL_GPIO_Init+0x228>
    8626:	2303      	movs	r3, #3
    8628:	e004      	b.n	8634 <HAL_GPIO_Init+0x228>
    862a:	2302      	movs	r3, #2
    862c:	e002      	b.n	8634 <HAL_GPIO_Init+0x228>
    862e:	2301      	movs	r3, #1
    8630:	e000      	b.n	8634 <HAL_GPIO_Init+0x228>
    8632:	2300      	movs	r3, #0
    8634:	69fa      	ldr	r2, [r7, #28]
    8636:	f002 0203 	and.w	r2, r2, #3
    863a:	0092      	lsls	r2, r2, #2
    863c:	4093      	lsls	r3, r2
    863e:	69ba      	ldr	r2, [r7, #24]
    8640:	4313      	orrs	r3, r2
    8642:	61bb      	str	r3, [r7, #24]
        SYSCFG->EXTICR[position >> 2U] = temp;
    8644:	4934      	ldr	r1, [pc, #208]	; (8718 <HAL_GPIO_Init+0x30c>)
    8646:	69fb      	ldr	r3, [r7, #28]
    8648:	089b      	lsrs	r3, r3, #2
    864a:	3302      	adds	r3, #2
    864c:	69ba      	ldr	r2, [r7, #24]
    864e:	f841 2023 	str.w	r2, [r1, r3, lsl #2]

        /* Clear EXTI line configuration */
        temp = EXTI->IMR;
    8652:	4b3a      	ldr	r3, [pc, #232]	; (873c <HAL_GPIO_Init+0x330>)
    8654:	681b      	ldr	r3, [r3, #0]
    8656:	61bb      	str	r3, [r7, #24]
        temp &= ~((uint32_t)iocurrent);
    8658:	693b      	ldr	r3, [r7, #16]
    865a:	43db      	mvns	r3, r3
    865c:	69ba      	ldr	r2, [r7, #24]
    865e:	4013      	ands	r3, r2
    8660:	61bb      	str	r3, [r7, #24]
        if((GPIO_Init->Mode & GPIO_MODE_IT) == GPIO_MODE_IT)
    8662:	683b      	ldr	r3, [r7, #0]
    8664:	685b      	ldr	r3, [r3, #4]
    8666:	f403 3380 	and.w	r3, r3, #65536	; 0x10000
    866a:	2b00      	cmp	r3, #0
    866c:	d003      	beq.n	8676 <HAL_GPIO_Init+0x26a>
        {
          temp |= iocurrent;
    866e:	69ba      	ldr	r2, [r7, #24]
    8670:	693b      	ldr	r3, [r7, #16]
    8672:	4313      	orrs	r3, r2
    8674:	61bb      	str	r3, [r7, #24]
        }
        EXTI->IMR = temp;
    8676:	4a31      	ldr	r2, [pc, #196]	; (873c <HAL_GPIO_Init+0x330>)
    8678:	69bb      	ldr	r3, [r7, #24]
    867a:	6013      	str	r3, [r2, #0]

        temp = EXTI->EMR;
    867c:	4b2f      	ldr	r3, [pc, #188]	; (873c <HAL_GPIO_Init+0x330>)
    867e:	685b      	ldr	r3, [r3, #4]
    8680:	61bb      	str	r3, [r7, #24]
        temp &= ~((uint32_t)iocurrent);
    8682:	693b      	ldr	r3, [r7, #16]
    8684:	43db      	mvns	r3, r3
    8686:	69ba      	ldr	r2, [r7, #24]
    8688:	4013      	ands	r3, r2
    868a:	61bb      	str	r3, [r7, #24]
        if((GPIO_Init->Mode & GPIO_MODE_EVT) == GPIO_MODE_EVT)
    868c:	683b      	ldr	r3, [r7, #0]
    868e:	685b      	ldr	r3, [r3, #4]
    8690:	f403 3300 	and.w	r3, r3, #131072	; 0x20000
    8694:	2b00      	cmp	r3, #0
    8696:	d003      	beq.n	86a0 <HAL_GPIO_Init+0x294>
        {
          temp |= iocurrent;
    8698:	69ba      	ldr	r2, [r7, #24]
    869a:	693b      	ldr	r3, [r7, #16]
    869c:	4313      	orrs	r3, r2
    869e:	61bb      	str	r3, [r7, #24]
        }
        EXTI->EMR = temp;
    86a0:	4a26      	ldr	r2, [pc, #152]	; (873c <HAL_GPIO_Init+0x330>)
    86a2:	69bb      	ldr	r3, [r7, #24]
    86a4:	6053      	str	r3, [r2, #4]

        /* Clear Rising Falling edge configuration */
        temp = EXTI->RTSR;
    86a6:	4b25      	ldr	r3, [pc, #148]	; (873c <HAL_GPIO_Init+0x330>)
    86a8:	689b      	ldr	r3, [r3, #8]
    86aa:	61bb      	str	r3, [r7, #24]
        temp &= ~((uint32_t)iocurrent);
    86ac:	693b      	ldr	r3, [r7, #16]
    86ae:	43db      	mvns	r3, r3
    86b0:	69ba      	ldr	r2, [r7, #24]
    86b2:	4013      	ands	r3, r2
    86b4:	61bb      	str	r3, [r7, #24]
        if((GPIO_Init->Mode & RISING_EDGE) == RISING_EDGE)
    86b6:	683b      	ldr	r3, [r7, #0]
    86b8:	685b      	ldr	r3, [r3, #4]
    86ba:	f403 1380 	and.w	r3, r3, #1048576	; 0x100000
    86be:	2b00      	cmp	r3, #0
    86c0:	d003      	beq.n	86ca <HAL_GPIO_Init+0x2be>
        {
          temp |= iocurrent;
    86c2:	69ba      	ldr	r2, [r7, #24]
    86c4:	693b      	ldr	r3, [r7, #16]
    86c6:	4313      	orrs	r3, r2
    86c8:	61bb      	str	r3, [r7, #24]
        }
        EXTI->RTSR = temp;
    86ca:	4a1c      	ldr	r2, [pc, #112]	; (873c <HAL_GPIO_Init+0x330>)
    86cc:	69bb      	ldr	r3, [r7, #24]
    86ce:	6093      	str	r3, [r2, #8]

        temp = EXTI->FTSR;
    86d0:	4b1a      	ldr	r3, [pc, #104]	; (873c <HAL_GPIO_Init+0x330>)
    86d2:	68db      	ldr	r3, [r3, #12]
    86d4:	61bb      	str	r3, [r7, #24]
        temp &= ~((uint32_t)iocurrent);
    86d6:	693b      	ldr	r3, [r7, #16]
    86d8:	43db      	mvns	r3, r3
    86da:	69ba      	ldr	r2, [r7, #24]
    86dc:	4013      	ands	r3, r2
    86de:	61bb      	str	r3, [r7, #24]
        if((GPIO_Init->Mode & FALLING_EDGE) == FALLING_EDGE)
    86e0:	683b      	ldr	r3, [r7, #0]
    86e2:	685b      	ldr	r3, [r3, #4]
    86e4:	f403 1300 	and.w	r3, r3, #2097152	; 0x200000
    86e8:	2b00      	cmp	r3, #0
    86ea:	d003      	beq.n	86f4 <HAL_GPIO_Init+0x2e8>
        {
          temp |= iocurrent;
    86ec:	69ba      	ldr	r2, [r7, #24]
    86ee:	693b      	ldr	r3, [r7, #16]
    86f0:	4313      	orrs	r3, r2
    86f2:	61bb      	str	r3, [r7, #24]
        }
        EXTI->FTSR = temp;
    86f4:	4a11      	ldr	r2, [pc, #68]	; (873c <HAL_GPIO_Init+0x330>)
    86f6:	69bb      	ldr	r3, [r7, #24]
    86f8:	60d3      	str	r3, [r2, #12]
  for(position = 0U; position < GPIO_NUMBER; position++)
    86fa:	69fb      	ldr	r3, [r7, #28]
    86fc:	3301      	adds	r3, #1
    86fe:	61fb      	str	r3, [r7, #28]
    8700:	69fb      	ldr	r3, [r7, #28]
    8702:	2b0f      	cmp	r3, #15
    8704:	f67f ae90 	bls.w	8428 <HAL_GPIO_Init+0x1c>
      }
    }
  }
}
    8708:	bf00      	nop
    870a:	3724      	adds	r7, #36	; 0x24
    870c:	46bd      	mov	sp, r7
    870e:	f85d 7b04 	ldr.w	r7, [sp], #4
    8712:	4770      	bx	lr
    8714:	40023800 	.word	0x40023800
    8718:	40013800 	.word	0x40013800
    871c:	40020000 	.word	0x40020000
    8720:	40020400 	.word	0x40020400
    8724:	40020800 	.word	0x40020800
    8728:	40020c00 	.word	0x40020c00
    872c:	40021000 	.word	0x40021000
    8730:	40021400 	.word	0x40021400
    8734:	40021800 	.word	0x40021800
    8738:	40021c00 	.word	0x40021c00
    873c:	40013c00 	.word	0x40013c00

00008740 <HAL_GPIO_WritePin>:
  *            @arg GPIO_PIN_RESET: to clear the port pin
  *            @arg GPIO_PIN_SET: to set the port pin
  * @retval None
  */
void HAL_GPIO_WritePin(GPIO_TypeDef* GPIOx, uint16_t GPIO_Pin, GPIO_PinState PinState)
{
    8740:	b480      	push	{r7}
    8742:	b083      	sub	sp, #12
    8744:	af00      	add	r7, sp, #0
    8746:	6078      	str	r0, [r7, #4]
    8748:	460b      	mov	r3, r1
    874a:	807b      	strh	r3, [r7, #2]
    874c:	4613      	mov	r3, r2
    874e:	707b      	strb	r3, [r7, #1]
  /* Check the parameters */
  assert_param(IS_GPIO_PIN(GPIO_Pin));
  assert_param(IS_GPIO_PIN_ACTION(PinState));

  if(PinState != GPIO_PIN_RESET)
    8750:	787b      	ldrb	r3, [r7, #1]
    8752:	2b00      	cmp	r3, #0
    8754:	d003      	beq.n	875e <HAL_GPIO_WritePin+0x1e>
  {
    GPIOx->BSRR = GPIO_Pin;
    8756:	887a      	ldrh	r2, [r7, #2]
    8758:	687b      	ldr	r3, [r7, #4]
    875a:	619a      	str	r2, [r3, #24]
  }
  else
  {
    GPIOx->BSRR = (uint32_t)GPIO_Pin << 16U;
  }
}
    875c:	e003      	b.n	8766 <HAL_GPIO_WritePin+0x26>
    GPIOx->BSRR = (uint32_t)GPIO_Pin << 16U;
    875e:	887b      	ldrh	r3, [r7, #2]
    8760:	041a      	lsls	r2, r3, #16
    8762:	687b      	ldr	r3, [r7, #4]
    8764:	619a      	str	r2, [r3, #24]
}
    8766:	bf00      	nop
    8768:	370c      	adds	r7, #12
    876a:	46bd      	mov	sp, r7
    876c:	f85d 7b04 	ldr.w	r7, [sp], #4
    8770:	4770      	bx	lr
	...

00008774 <HAL_I2C_Init>:
  * @param  hi2c Pointer to a I2C_HandleTypeDef structure that contains
  *                the configuration information for the specified I2C.
  * @retval HAL status
  */
HAL_StatusTypeDef HAL_I2C_Init(I2C_HandleTypeDef *hi2c)
{
    8774:	b580      	push	{r7, lr}
    8776:	b084      	sub	sp, #16
    8778:	af00      	add	r7, sp, #0
    877a:	6078      	str	r0, [r7, #4]
  uint32_t freqrange;
  uint32_t pclk1;

  /* Check the I2C handle allocation */
  if (hi2c == NULL)
    877c:	687b      	ldr	r3, [r7, #4]
    877e:	2b00      	cmp	r3, #0
    8780:	d101      	bne.n	8786 <HAL_I2C_Init+0x12>
  {
    return HAL_ERROR;
    8782:	2301      	movs	r3, #1
    8784:	e10f      	b.n	89a6 <HAL_I2C_Init+0x232>
  assert_param(IS_I2C_DUAL_ADDRESS(hi2c->Init.DualAddressMode));
  assert_param(IS_I2C_OWN_ADDRESS2(hi2c->Init.OwnAddress2));
  assert_param(IS_I2C_GENERAL_CALL(hi2c->Init.GeneralCallMode));
  assert_param(IS_I2C_NO_STRETCH(hi2c->Init.NoStretchMode));

  if (hi2c->State == HAL_I2C_STATE_RESET)
    8786:	687b      	ldr	r3, [r7, #4]
    8788:	f893 303d 	ldrb.w	r3, [r3, #61]	; 0x3d
    878c:	b2db      	uxtb	r3, r3
    878e:	2b00      	cmp	r3, #0
    8790:	d106      	bne.n	87a0 <HAL_I2C_Init+0x2c>
  {
    /* Allocate lock resource and initialize it */
    hi2c->Lock = HAL_UNLOCKED;
    8792:	687b      	ldr	r3, [r7, #4]
    8794:	2200      	movs	r2, #0
    8796:	f883 203c 	strb.w	r2, [r3, #60]	; 0x3c

    /* Init the low level hardware : GPIO, CLOCK, NVIC */
    hi2c->MspInitCallback(hi2c);
#else
    /* Init the low level hardware : GPIO, CLOCK, NVIC */
    HAL_I2C_MspInit(hi2c);
    879a:	6878      	ldr	r0, [r7, #4]
    879c:	f003 fd8c 	bl	c2b8 <HAL_I2C_MspInit>
#endif /* USE_HAL_I2C_REGISTER_CALLBACKS */
  }

  hi2c->State = HAL_I2C_STATE_BUSY;
    87a0:	687b      	ldr	r3, [r7, #4]
    87a2:	2224      	movs	r2, #36	; 0x24
    87a4:	f883 203d 	strb.w	r2, [r3, #61]	; 0x3d

  /* Disable the selected I2C peripheral */
  __HAL_I2C_DISABLE(hi2c);
    87a8:	687b      	ldr	r3, [r7, #4]
    87aa:	681b      	ldr	r3, [r3, #0]
    87ac:	681a      	ldr	r2, [r3, #0]
    87ae:	687b      	ldr	r3, [r7, #4]
    87b0:	681b      	ldr	r3, [r3, #0]
    87b2:	f022 0201 	bic.w	r2, r2, #1
    87b6:	601a      	str	r2, [r3, #0]

  /* Get PCLK1 frequency */
  pclk1 = HAL_RCC_GetPCLK1Freq();
    87b8:	f001 fd18 	bl	a1ec <HAL_RCC_GetPCLK1Freq>
    87bc:	60f8      	str	r0, [r7, #12]

  /* Check the minimum allowed PCLK1 frequency */
  if (I2C_MIN_PCLK_FREQ(pclk1, hi2c->Init.ClockSpeed) == 1U)
    87be:	687b      	ldr	r3, [r7, #4]
    87c0:	685b      	ldr	r3, [r3, #4]
    87c2:	4a7b      	ldr	r2, [pc, #492]	; (89b0 <HAL_I2C_Init+0x23c>)
    87c4:	4293      	cmp	r3, r2
    87c6:	d807      	bhi.n	87d8 <HAL_I2C_Init+0x64>
    87c8:	68fb      	ldr	r3, [r7, #12]
    87ca:	4a7a      	ldr	r2, [pc, #488]	; (89b4 <HAL_I2C_Init+0x240>)
    87cc:	4293      	cmp	r3, r2
    87ce:	bf94      	ite	ls
    87d0:	2301      	movls	r3, #1
    87d2:	2300      	movhi	r3, #0
    87d4:	b2db      	uxtb	r3, r3
    87d6:	e006      	b.n	87e6 <HAL_I2C_Init+0x72>
    87d8:	68fb      	ldr	r3, [r7, #12]
    87da:	4a77      	ldr	r2, [pc, #476]	; (89b8 <HAL_I2C_Init+0x244>)
    87dc:	4293      	cmp	r3, r2
    87de:	bf94      	ite	ls
    87e0:	2301      	movls	r3, #1
    87e2:	2300      	movhi	r3, #0
    87e4:	b2db      	uxtb	r3, r3
    87e6:	2b00      	cmp	r3, #0
    87e8:	d001      	beq.n	87ee <HAL_I2C_Init+0x7a>
  {
    return HAL_ERROR;
    87ea:	2301      	movs	r3, #1
    87ec:	e0db      	b.n	89a6 <HAL_I2C_Init+0x232>
  }

  /* Calculate frequency range */
  freqrange = I2C_FREQRANGE(pclk1);
    87ee:	68fb      	ldr	r3, [r7, #12]
    87f0:	4a72      	ldr	r2, [pc, #456]	; (89bc <HAL_I2C_Init+0x248>)
    87f2:	fba2 2303 	umull	r2, r3, r2, r3
    87f6:	0c9b      	lsrs	r3, r3, #18
    87f8:	60bb      	str	r3, [r7, #8]

  /*---------------------------- I2Cx CR2 Configuration ----------------------*/
  /* Configure I2Cx: Frequency range */
  MODIFY_REG(hi2c->Instance->CR2, I2C_CR2_FREQ, freqrange);
    87fa:	687b      	ldr	r3, [r7, #4]
    87fc:	681b      	ldr	r3, [r3, #0]
    87fe:	685b      	ldr	r3, [r3, #4]
    8800:	f023 013f 	bic.w	r1, r3, #63	; 0x3f
    8804:	687b      	ldr	r3, [r7, #4]
    8806:	681b      	ldr	r3, [r3, #0]
    8808:	68ba      	ldr	r2, [r7, #8]
    880a:	430a      	orrs	r2, r1
    880c:	605a      	str	r2, [r3, #4]

  /*---------------------------- I2Cx TRISE Configuration --------------------*/
  /* Configure I2Cx: Rise Time */
  MODIFY_REG(hi2c->Instance->TRISE, I2C_TRISE_TRISE, I2C_RISE_TIME(freqrange, hi2c->Init.ClockSpeed));
    880e:	687b      	ldr	r3, [r7, #4]
    8810:	681b      	ldr	r3, [r3, #0]
    8812:	6a1b      	ldr	r3, [r3, #32]
    8814:	f023 013f 	bic.w	r1, r3, #63	; 0x3f
    8818:	687b      	ldr	r3, [r7, #4]
    881a:	685b      	ldr	r3, [r3, #4]
    881c:	4a64      	ldr	r2, [pc, #400]	; (89b0 <HAL_I2C_Init+0x23c>)
    881e:	4293      	cmp	r3, r2
    8820:	d802      	bhi.n	8828 <HAL_I2C_Init+0xb4>
    8822:	68bb      	ldr	r3, [r7, #8]
    8824:	3301      	adds	r3, #1
    8826:	e009      	b.n	883c <HAL_I2C_Init+0xc8>
    8828:	68bb      	ldr	r3, [r7, #8]
    882a:	f44f 7296 	mov.w	r2, #300	; 0x12c
    882e:	fb02 f303 	mul.w	r3, r2, r3
    8832:	4a63      	ldr	r2, [pc, #396]	; (89c0 <HAL_I2C_Init+0x24c>)
    8834:	fba2 2303 	umull	r2, r3, r2, r3
    8838:	099b      	lsrs	r3, r3, #6
    883a:	3301      	adds	r3, #1
    883c:	687a      	ldr	r2, [r7, #4]
    883e:	6812      	ldr	r2, [r2, #0]
    8840:	430b      	orrs	r3, r1
    8842:	6213      	str	r3, [r2, #32]

  /*---------------------------- I2Cx CCR Configuration ----------------------*/
  /* Configure I2Cx: Speed */
  MODIFY_REG(hi2c->Instance->CCR, (I2C_CCR_FS | I2C_CCR_DUTY | I2C_CCR_CCR), I2C_SPEED(pclk1, hi2c->Init.ClockSpeed, hi2c->Init.DutyCycle));
    8844:	687b      	ldr	r3, [r7, #4]
    8846:	681b      	ldr	r3, [r3, #0]
    8848:	69db      	ldr	r3, [r3, #28]
    884a:	f423 424f 	bic.w	r2, r3, #52992	; 0xcf00
    884e:	f022 02ff 	bic.w	r2, r2, #255	; 0xff
    8852:	687b      	ldr	r3, [r7, #4]
    8854:	685b      	ldr	r3, [r3, #4]
    8856:	4956      	ldr	r1, [pc, #344]	; (89b0 <HAL_I2C_Init+0x23c>)
    8858:	428b      	cmp	r3, r1
    885a:	d80d      	bhi.n	8878 <HAL_I2C_Init+0x104>
    885c:	68fb      	ldr	r3, [r7, #12]
    885e:	1e59      	subs	r1, r3, #1
    8860:	687b      	ldr	r3, [r7, #4]
    8862:	685b      	ldr	r3, [r3, #4]
    8864:	005b      	lsls	r3, r3, #1
    8866:	fbb1 f3f3 	udiv	r3, r1, r3
    886a:	3301      	adds	r3, #1
    886c:	f3c3 030b 	ubfx	r3, r3, #0, #12
    8870:	2b04      	cmp	r3, #4
    8872:	bf38      	it	cc
    8874:	2304      	movcc	r3, #4
    8876:	e04f      	b.n	8918 <HAL_I2C_Init+0x1a4>
    8878:	687b      	ldr	r3, [r7, #4]
    887a:	689b      	ldr	r3, [r3, #8]
    887c:	2b00      	cmp	r3, #0
    887e:	d111      	bne.n	88a4 <HAL_I2C_Init+0x130>
    8880:	68fb      	ldr	r3, [r7, #12]
    8882:	1e58      	subs	r0, r3, #1
    8884:	687b      	ldr	r3, [r7, #4]
    8886:	6859      	ldr	r1, [r3, #4]
    8888:	460b      	mov	r3, r1
    888a:	005b      	lsls	r3, r3, #1
    888c:	440b      	add	r3, r1
    888e:	fbb0 f3f3 	udiv	r3, r0, r3
    8892:	3301      	adds	r3, #1
    8894:	f3c3 030b 	ubfx	r3, r3, #0, #12
    8898:	2b00      	cmp	r3, #0
    889a:	bf0c      	ite	eq
    889c:	2301      	moveq	r3, #1
    889e:	2300      	movne	r3, #0
    88a0:	b2db      	uxtb	r3, r3
    88a2:	e012      	b.n	88ca <HAL_I2C_Init+0x156>
    88a4:	68fb      	ldr	r3, [r7, #12]
    88a6:	1e58      	subs	r0, r3, #1
    88a8:	687b      	ldr	r3, [r7, #4]
    88aa:	6859      	ldr	r1, [r3, #4]
    88ac:	460b      	mov	r3, r1
    88ae:	009b      	lsls	r3, r3, #2
    88b0:	440b      	add	r3, r1
    88b2:	0099      	lsls	r1, r3, #2
    88b4:	440b      	add	r3, r1
    88b6:	fbb0 f3f3 	udiv	r3, r0, r3
    88ba:	3301      	adds	r3, #1
    88bc:	f3c3 030b 	ubfx	r3, r3, #0, #12
    88c0:	2b00      	cmp	r3, #0
    88c2:	bf0c      	ite	eq
    88c4:	2301      	moveq	r3, #1
    88c6:	2300      	movne	r3, #0
    88c8:	b2db      	uxtb	r3, r3
    88ca:	2b00      	cmp	r3, #0
    88cc:	d001      	beq.n	88d2 <HAL_I2C_Init+0x15e>
    88ce:	2301      	movs	r3, #1
    88d0:	e022      	b.n	8918 <HAL_I2C_Init+0x1a4>
    88d2:	687b      	ldr	r3, [r7, #4]
    88d4:	689b      	ldr	r3, [r3, #8]
    88d6:	2b00      	cmp	r3, #0
    88d8:	d10e      	bne.n	88f8 <HAL_I2C_Init+0x184>
    88da:	68fb      	ldr	r3, [r7, #12]
    88dc:	1e58      	subs	r0, r3, #1
    88de:	687b      	ldr	r3, [r7, #4]
    88e0:	6859      	ldr	r1, [r3, #4]
    88e2:	460b      	mov	r3, r1
    88e4:	005b      	lsls	r3, r3, #1
    88e6:	440b      	add	r3, r1
    88e8:	fbb0 f3f3 	udiv	r3, r0, r3
    88ec:	3301      	adds	r3, #1
    88ee:	f3c3 030b 	ubfx	r3, r3, #0, #12
    88f2:	f443 4300 	orr.w	r3, r3, #32768	; 0x8000
    88f6:	e00f      	b.n	8918 <HAL_I2C_Init+0x1a4>
    88f8:	68fb      	ldr	r3, [r7, #12]
    88fa:	1e58      	subs	r0, r3, #1
    88fc:	687b      	ldr	r3, [r7, #4]
    88fe:	6859      	ldr	r1, [r3, #4]
    8900:	460b      	mov	r3, r1
    8902:	009b      	lsls	r3, r3, #2
    8904:	440b      	add	r3, r1
    8906:	0099      	lsls	r1, r3, #2
    8908:	440b      	add	r3, r1
    890a:	fbb0 f3f3 	udiv	r3, r0, r3
    890e:	3301      	adds	r3, #1
    8910:	f3c3 030b 	ubfx	r3, r3, #0, #12
    8914:	f443 4340 	orr.w	r3, r3, #49152	; 0xc000
    8918:	6879      	ldr	r1, [r7, #4]
    891a:	6809      	ldr	r1, [r1, #0]
    891c:	4313      	orrs	r3, r2
    891e:	61cb      	str	r3, [r1, #28]

  /*---------------------------- I2Cx CR1 Configuration ----------------------*/
  /* Configure I2Cx: Generalcall and NoStretch mode */
  MODIFY_REG(hi2c->Instance->CR1, (I2C_CR1_ENGC | I2C_CR1_NOSTRETCH), (hi2c->Init.GeneralCallMode | hi2c->Init.NoStretchMode));
    8920:	687b      	ldr	r3, [r7, #4]
    8922:	681b      	ldr	r3, [r3, #0]
    8924:	681b      	ldr	r3, [r3, #0]
    8926:	f023 01c0 	bic.w	r1, r3, #192	; 0xc0
    892a:	687b      	ldr	r3, [r7, #4]
    892c:	69da      	ldr	r2, [r3, #28]
    892e:	687b      	ldr	r3, [r7, #4]
    8930:	6a1b      	ldr	r3, [r3, #32]
    8932:	431a      	orrs	r2, r3
    8934:	687b      	ldr	r3, [r7, #4]
    8936:	681b      	ldr	r3, [r3, #0]
    8938:	430a      	orrs	r2, r1
    893a:	601a      	str	r2, [r3, #0]

  /*---------------------------- I2Cx OAR1 Configuration ---------------------*/
  /* Configure I2Cx: Own Address1 and addressing mode */
  MODIFY_REG(hi2c->Instance->OAR1, (I2C_OAR1_ADDMODE | I2C_OAR1_ADD8_9 | I2C_OAR1_ADD1_7 | I2C_OAR1_ADD0), (hi2c->Init.AddressingMode | hi2c->Init.OwnAddress1));
    893c:	687b      	ldr	r3, [r7, #4]
    893e:	681b      	ldr	r3, [r3, #0]
    8940:	689b      	ldr	r3, [r3, #8]
    8942:	f423 4303 	bic.w	r3, r3, #33536	; 0x8300
    8946:	f023 03ff 	bic.w	r3, r3, #255	; 0xff
    894a:	687a      	ldr	r2, [r7, #4]
    894c:	6911      	ldr	r1, [r2, #16]
    894e:	687a      	ldr	r2, [r7, #4]
    8950:	68d2      	ldr	r2, [r2, #12]
    8952:	4311      	orrs	r1, r2
    8954:	687a      	ldr	r2, [r7, #4]
    8956:	6812      	ldr	r2, [r2, #0]
    8958:	430b      	orrs	r3, r1
    895a:	6093      	str	r3, [r2, #8]

  /*---------------------------- I2Cx OAR2 Configuration ---------------------*/
  /* Configure I2Cx: Dual mode and Own Address2 */
  MODIFY_REG(hi2c->Instance->OAR2, (I2C_OAR2_ENDUAL | I2C_OAR2_ADD2), (hi2c->Init.DualAddressMode | hi2c->Init.OwnAddress2));
    895c:	687b      	ldr	r3, [r7, #4]
    895e:	681b      	ldr	r3, [r3, #0]
    8960:	68db      	ldr	r3, [r3, #12]
    8962:	f023 01ff 	bic.w	r1, r3, #255	; 0xff
    8966:	687b      	ldr	r3, [r7, #4]
    8968:	695a      	ldr	r2, [r3, #20]
    896a:	687b      	ldr	r3, [r7, #4]
    896c:	699b      	ldr	r3, [r3, #24]
    896e:	431a      	orrs	r2, r3
    8970:	687b      	ldr	r3, [r7, #4]
    8972:	681b      	ldr	r3, [r3, #0]
    8974:	430a      	orrs	r2, r1
    8976:	60da      	str	r2, [r3, #12]

  /* Enable the selected I2C peripheral */
  __HAL_I2C_ENABLE(hi2c);
    8978:	687b      	ldr	r3, [r7, #4]
    897a:	681b      	ldr	r3, [r3, #0]
    897c:	681a      	ldr	r2, [r3, #0]
    897e:	687b      	ldr	r3, [r7, #4]
    8980:	681b      	ldr	r3, [r3, #0]
    8982:	f042 0201 	orr.w	r2, r2, #1
    8986:	601a      	str	r2, [r3, #0]

  hi2c->ErrorCode = HAL_I2C_ERROR_NONE;
    8988:	687b      	ldr	r3, [r7, #4]
    898a:	2200      	movs	r2, #0
    898c:	641a      	str	r2, [r3, #64]	; 0x40
  hi2c->State = HAL_I2C_STATE_READY;
    898e:	687b      	ldr	r3, [r7, #4]
    8990:	2220      	movs	r2, #32
    8992:	f883 203d 	strb.w	r2, [r3, #61]	; 0x3d
  hi2c->PreviousState = I2C_STATE_NONE;
    8996:	687b      	ldr	r3, [r7, #4]
    8998:	2200      	movs	r2, #0
    899a:	631a      	str	r2, [r3, #48]	; 0x30
  hi2c->Mode = HAL_I2C_MODE_NONE;
    899c:	687b      	ldr	r3, [r7, #4]
    899e:	2200      	movs	r2, #0
    89a0:	f883 203e 	strb.w	r2, [r3, #62]	; 0x3e

  return HAL_OK;
    89a4:	2300      	movs	r3, #0
}
    89a6:	4618      	mov	r0, r3
    89a8:	3710      	adds	r7, #16
    89aa:	46bd      	mov	sp, r7
    89ac:	bd80      	pop	{r7, pc}
    89ae:	bf00      	nop
    89b0:	000186a0 	.word	0x000186a0
    89b4:	001e847f 	.word	0x001e847f
    89b8:	003d08ff 	.word	0x003d08ff
    89bc:	431bde83 	.word	0x431bde83
    89c0:	10624dd3 	.word	0x10624dd3

000089c4 <HAL_I2S_Init>:
  * @param  hi2s pointer to a I2S_HandleTypeDef structure that contains
  *         the configuration information for I2S module
  * @retval HAL status
  */
HAL_StatusTypeDef HAL_I2S_Init(I2S_HandleTypeDef *hi2s)
{
    89c4:	b580      	push	{r7, lr}
    89c6:	b088      	sub	sp, #32
    89c8:	af00      	add	r7, sp, #0
    89ca:	6078      	str	r0, [r7, #4]
#if defined (SPI_I2S_FULLDUPLEX_SUPPORT)
  uint16_t tmpreg;
#endif

  /* Check the I2S handle allocation */
  if (hi2s == NULL)
    89cc:	687b      	ldr	r3, [r7, #4]
    89ce:	2b00      	cmp	r3, #0
    89d0:	d101      	bne.n	89d6 <HAL_I2S_Init+0x12>
  {
    return HAL_ERROR;
    89d2:	2301      	movs	r3, #1
    89d4:	e128      	b.n	8c28 <HAL_I2S_Init+0x264>
  assert_param(IS_I2S_MCLK_OUTPUT(hi2s->Init.MCLKOutput));
  assert_param(IS_I2S_AUDIO_FREQ(hi2s->Init.AudioFreq));
  assert_param(IS_I2S_CPOL(hi2s->Init.CPOL));
  assert_param(IS_I2S_CLOCKSOURCE(hi2s->Init.ClockSource));

  if (hi2s->State == HAL_I2S_STATE_RESET)
    89d6:	687b      	ldr	r3, [r7, #4]
    89d8:	f893 3041 	ldrb.w	r3, [r3, #65]	; 0x41
    89dc:	b2db      	uxtb	r3, r3
    89de:	2b00      	cmp	r3, #0
    89e0:	d109      	bne.n	89f6 <HAL_I2S_Init+0x32>
  {
    /* Allocate lock resource and initialize it */
    hi2s->Lock = HAL_UNLOCKED;
    89e2:	687b      	ldr	r3, [r7, #4]
    89e4:	2200      	movs	r2, #0
    89e6:	f883 2040 	strb.w	r2, [r3, #64]	; 0x40

    /* Initialize Default I2S IrqHandler ISR */
    hi2s->IrqHandlerISR = I2S_IRQHandler;
    89ea:	687b      	ldr	r3, [r7, #4]
    89ec:	4a90      	ldr	r2, [pc, #576]	; (8c30 <HAL_I2S_Init+0x26c>)
    89ee:	635a      	str	r2, [r3, #52]	; 0x34

    /* Init the low level hardware : GPIO, CLOCK, NVIC... */
    hi2s->MspInitCallback(hi2s);
#else
    /* Init the low level hardware : GPIO, CLOCK, CORTEX...etc */
    HAL_I2S_MspInit(hi2s);
    89f0:	6878      	ldr	r0, [r7, #4]
    89f2:	f003 fca9 	bl	c348 <HAL_I2S_MspInit>
#endif /* USE_HAL_I2S_REGISTER_CALLBACKS */
  }

  hi2s->State = HAL_I2S_STATE_BUSY;
    89f6:	687b      	ldr	r3, [r7, #4]
    89f8:	2202      	movs	r2, #2
    89fa:	f883 2041 	strb.w	r2, [r3, #65]	; 0x41

  /*----------------------- SPIx I2SCFGR & I2SPR Configuration ----------------*/
  /* Clear I2SMOD, I2SE, I2SCFG, PCMSYNC, I2SSTD, CKPOL, DATLEN and CHLEN bits */
  CLEAR_BIT(hi2s->Instance->I2SCFGR, (SPI_I2SCFGR_CHLEN | SPI_I2SCFGR_DATLEN | SPI_I2SCFGR_CKPOL | \
    89fe:	687b      	ldr	r3, [r7, #4]
    8a00:	681b      	ldr	r3, [r3, #0]
    8a02:	69db      	ldr	r3, [r3, #28]
    8a04:	687a      	ldr	r2, [r7, #4]
    8a06:	6812      	ldr	r2, [r2, #0]
    8a08:	f423 637b 	bic.w	r3, r3, #4016	; 0xfb0
    8a0c:	f023 030f 	bic.w	r3, r3, #15
    8a10:	61d3      	str	r3, [r2, #28]
                                      SPI_I2SCFGR_I2SSTD | SPI_I2SCFGR_PCMSYNC | SPI_I2SCFGR_I2SCFG | \
                                      SPI_I2SCFGR_I2SE | SPI_I2SCFGR_I2SMOD));
  hi2s->Instance->I2SPR = 0x0002U;
    8a12:	687b      	ldr	r3, [r7, #4]
    8a14:	681b      	ldr	r3, [r3, #0]
    8a16:	2202      	movs	r2, #2
    8a18:	621a      	str	r2, [r3, #32]

  /*----------------------- I2SPR: I2SDIV and ODD Calculation -----------------*/
  /* If the requested audio frequency is not the default, compute the prescaler */
  if (hi2s->Init.AudioFreq != I2S_AUDIOFREQ_DEFAULT)
    8a1a:	687b      	ldr	r3, [r7, #4]
    8a1c:	695b      	ldr	r3, [r3, #20]
    8a1e:	2b02      	cmp	r3, #2
    8a20:	d060      	beq.n	8ae4 <HAL_I2S_Init+0x120>
  {
    /* Check the frame length (For the Prescaler computing) ********************/
    if (hi2s->Init.DataFormat == I2S_DATAFORMAT_16B)
    8a22:	687b      	ldr	r3, [r7, #4]
    8a24:	68db      	ldr	r3, [r3, #12]
    8a26:	2b00      	cmp	r3, #0
    8a28:	d102      	bne.n	8a30 <HAL_I2S_Init+0x6c>
    {
      /* Packet length is 16 bits */
      packetlength = 16U;
    8a2a:	2310      	movs	r3, #16
    8a2c:	617b      	str	r3, [r7, #20]
    8a2e:	e001      	b.n	8a34 <HAL_I2S_Init+0x70>
    }
    else
    {
      /* Packet length is 32 bits */
      packetlength = 32U;
    8a30:	2320      	movs	r3, #32
    8a32:	617b      	str	r3, [r7, #20]
    }

    /* I2S standard */
    if (hi2s->Init.Standard <= I2S_STANDARD_LSB)
    8a34:	687b      	ldr	r3, [r7, #4]
    8a36:	689b      	ldr	r3, [r3, #8]
    8a38:	2b20      	cmp	r3, #32
    8a3a:	d802      	bhi.n	8a42 <HAL_I2S_Init+0x7e>
    {
      /* In I2S standard packet lenght is multiplied by 2 */
      packetlength = packetlength * 2U;
    8a3c:	697b      	ldr	r3, [r7, #20]
    8a3e:	005b      	lsls	r3, r3, #1
    8a40:	617b      	str	r3, [r7, #20]
    else
    {
      i2sclk = HAL_RCCEx_GetPeriphCLKFreq(RCC_PERIPHCLK_I2S_APB2);
    }
#else
    i2sclk = HAL_RCCEx_GetPeriphCLKFreq(RCC_PERIPHCLK_I2S);
    8a42:	2001      	movs	r0, #1
    8a44:	f001 fcc8 	bl	a3d8 <HAL_RCCEx_GetPeriphCLKFreq>
    8a48:	60f8      	str	r0, [r7, #12]
#endif

    /* Compute the Real divider depending on the MCLK output state, with a floating point */
    if (hi2s->Init.MCLKOutput == I2S_MCLKOUTPUT_ENABLE)
    8a4a:	687b      	ldr	r3, [r7, #4]
    8a4c:	691b      	ldr	r3, [r3, #16]
    8a4e:	f5b3 7f00 	cmp.w	r3, #512	; 0x200
    8a52:	d125      	bne.n	8aa0 <HAL_I2S_Init+0xdc>
    {
      /* MCLK output is enabled */
      if (hi2s->Init.DataFormat != I2S_DATAFORMAT_16B)
    8a54:	687b      	ldr	r3, [r7, #4]
    8a56:	68db      	ldr	r3, [r3, #12]
    8a58:	2b00      	cmp	r3, #0
    8a5a:	d010      	beq.n	8a7e <HAL_I2S_Init+0xba>
      {
        tmp = (uint32_t)(((((i2sclk / (packetlength * 4U)) * 10U) / hi2s->Init.AudioFreq)) + 5U);
    8a5c:	697b      	ldr	r3, [r7, #20]
    8a5e:	009b      	lsls	r3, r3, #2
    8a60:	68fa      	ldr	r2, [r7, #12]
    8a62:	fbb2 f2f3 	udiv	r2, r2, r3
    8a66:	4613      	mov	r3, r2
    8a68:	009b      	lsls	r3, r3, #2
    8a6a:	4413      	add	r3, r2
    8a6c:	005b      	lsls	r3, r3, #1
    8a6e:	461a      	mov	r2, r3
    8a70:	687b      	ldr	r3, [r7, #4]
    8a72:	695b      	ldr	r3, [r3, #20]
    8a74:	fbb2 f3f3 	udiv	r3, r2, r3
    8a78:	3305      	adds	r3, #5
    8a7a:	613b      	str	r3, [r7, #16]
    8a7c:	e01f      	b.n	8abe <HAL_I2S_Init+0xfa>
      }
      else
      {
        tmp = (uint32_t)(((((i2sclk / (packetlength * 8U)) * 10U) / hi2s->Init.AudioFreq)) + 5U);
    8a7e:	697b      	ldr	r3, [r7, #20]
    8a80:	00db      	lsls	r3, r3, #3
    8a82:	68fa      	ldr	r2, [r7, #12]
    8a84:	fbb2 f2f3 	udiv	r2, r2, r3
    8a88:	4613      	mov	r3, r2
    8a8a:	009b      	lsls	r3, r3, #2
    8a8c:	4413      	add	r3, r2
    8a8e:	005b      	lsls	r3, r3, #1
    8a90:	461a      	mov	r2, r3
    8a92:	687b      	ldr	r3, [r7, #4]
    8a94:	695b      	ldr	r3, [r3, #20]
    8a96:	fbb2 f3f3 	udiv	r3, r2, r3
    8a9a:	3305      	adds	r3, #5
    8a9c:	613b      	str	r3, [r7, #16]
    8a9e:	e00e      	b.n	8abe <HAL_I2S_Init+0xfa>
      }
    }
    else
    {
      /* MCLK output is disabled */
      tmp = (uint32_t)(((((i2sclk / packetlength) * 10U) / hi2s->Init.AudioFreq)) + 5U);
    8aa0:	68fa      	ldr	r2, [r7, #12]
    8aa2:	697b      	ldr	r3, [r7, #20]
    8aa4:	fbb2 f2f3 	udiv	r2, r2, r3
    8aa8:	4613      	mov	r3, r2
    8aaa:	009b      	lsls	r3, r3, #2
    8aac:	4413      	add	r3, r2
    8aae:	005b      	lsls	r3, r3, #1
    8ab0:	461a      	mov	r2, r3
    8ab2:	687b      	ldr	r3, [r7, #4]
    8ab4:	695b      	ldr	r3, [r3, #20]
    8ab6:	fbb2 f3f3 	udiv	r3, r2, r3
    8aba:	3305      	adds	r3, #5
    8abc:	613b      	str	r3, [r7, #16]
    }

    /* Remove the flatting point */
    tmp = tmp / 10U;
    8abe:	693b      	ldr	r3, [r7, #16]
    8ac0:	4a5c      	ldr	r2, [pc, #368]	; (8c34 <HAL_I2S_Init+0x270>)
    8ac2:	fba2 2303 	umull	r2, r3, r2, r3
    8ac6:	08db      	lsrs	r3, r3, #3
    8ac8:	613b      	str	r3, [r7, #16]

    /* Check the parity of the divider */
    i2sodd = (uint32_t)(tmp & (uint32_t)1U);
    8aca:	693b      	ldr	r3, [r7, #16]
    8acc:	f003 0301 	and.w	r3, r3, #1
    8ad0:	61bb      	str	r3, [r7, #24]

    /* Compute the i2sdiv prescaler */
    i2sdiv = (uint32_t)((tmp - i2sodd) / 2U);
    8ad2:	693a      	ldr	r2, [r7, #16]
    8ad4:	69bb      	ldr	r3, [r7, #24]
    8ad6:	1ad3      	subs	r3, r2, r3
    8ad8:	085b      	lsrs	r3, r3, #1
    8ada:	61fb      	str	r3, [r7, #28]

    /* Get the Mask for the Odd bit (SPI_I2SPR[8]) register */
    i2sodd = (uint32_t)(i2sodd << 8U);
    8adc:	69bb      	ldr	r3, [r7, #24]
    8ade:	021b      	lsls	r3, r3, #8
    8ae0:	61bb      	str	r3, [r7, #24]
    8ae2:	e003      	b.n	8aec <HAL_I2S_Init+0x128>
  }
  else
  {
    /* Set the default values */
    i2sdiv = 2U;
    8ae4:	2302      	movs	r3, #2
    8ae6:	61fb      	str	r3, [r7, #28]
    i2sodd = 0U;
    8ae8:	2300      	movs	r3, #0
    8aea:	61bb      	str	r3, [r7, #24]
  }

  /* Test if the divider is 1 or 0 or greater than 0xFF */
  if ((i2sdiv < 2U) || (i2sdiv > 0xFFU))
    8aec:	69fb      	ldr	r3, [r7, #28]
    8aee:	2b01      	cmp	r3, #1
    8af0:	d902      	bls.n	8af8 <HAL_I2S_Init+0x134>
    8af2:	69fb      	ldr	r3, [r7, #28]
    8af4:	2bff      	cmp	r3, #255	; 0xff
    8af6:	d907      	bls.n	8b08 <HAL_I2S_Init+0x144>
  {
    /* Set the error code and execute error callback*/
    SET_BIT(hi2s->ErrorCode, HAL_I2S_ERROR_PRESCALER);
    8af8:	687b      	ldr	r3, [r7, #4]
    8afa:	6c5b      	ldr	r3, [r3, #68]	; 0x44
    8afc:	f043 0210 	orr.w	r2, r3, #16
    8b00:	687b      	ldr	r3, [r7, #4]
    8b02:	645a      	str	r2, [r3, #68]	; 0x44
    return  HAL_ERROR;
    8b04:	2301      	movs	r3, #1
    8b06:	e08f      	b.n	8c28 <HAL_I2S_Init+0x264>
  }

  /*----------------------- SPIx I2SCFGR & I2SPR Configuration ----------------*/

  /* Write to SPIx I2SPR register the computed value */
  hi2s->Instance->I2SPR = (uint32_t)((uint32_t)i2sdiv | (uint32_t)(i2sodd | (uint32_t)hi2s->Init.MCLKOutput));
    8b08:	687b      	ldr	r3, [r7, #4]
    8b0a:	691a      	ldr	r2, [r3, #16]
    8b0c:	69bb      	ldr	r3, [r7, #24]
    8b0e:	ea42 0103 	orr.w	r1, r2, r3
    8b12:	687b      	ldr	r3, [r7, #4]
    8b14:	681b      	ldr	r3, [r3, #0]
    8b16:	69fa      	ldr	r2, [r7, #28]
    8b18:	430a      	orrs	r2, r1
    8b1a:	621a      	str	r2, [r3, #32]

  /* Clear I2SMOD, I2SE, I2SCFG, PCMSYNC, I2SSTD, CKPOL, DATLEN and CHLEN bits */
  /* And configure the I2S with the I2S_InitStruct values                      */
  MODIFY_REG(hi2s->Instance->I2SCFGR, (SPI_I2SCFGR_CHLEN | SPI_I2SCFGR_DATLEN | \
    8b1c:	687b      	ldr	r3, [r7, #4]
    8b1e:	681b      	ldr	r3, [r3, #0]
    8b20:	69db      	ldr	r3, [r3, #28]
    8b22:	f423 637b 	bic.w	r3, r3, #4016	; 0xfb0
    8b26:	f023 030f 	bic.w	r3, r3, #15
    8b2a:	687a      	ldr	r2, [r7, #4]
    8b2c:	6851      	ldr	r1, [r2, #4]
    8b2e:	687a      	ldr	r2, [r7, #4]
    8b30:	6892      	ldr	r2, [r2, #8]
    8b32:	4311      	orrs	r1, r2
    8b34:	687a      	ldr	r2, [r7, #4]
    8b36:	68d2      	ldr	r2, [r2, #12]
    8b38:	4311      	orrs	r1, r2
    8b3a:	687a      	ldr	r2, [r7, #4]
    8b3c:	6992      	ldr	r2, [r2, #24]
    8b3e:	430a      	orrs	r2, r1
    8b40:	431a      	orrs	r2, r3
    8b42:	687b      	ldr	r3, [r7, #4]
    8b44:	681b      	ldr	r3, [r3, #0]
    8b46:	f442 6200 	orr.w	r2, r2, #2048	; 0x800
    8b4a:	61da      	str	r2, [r3, #28]
#if defined (SPI_I2S_FULLDUPLEX_SUPPORT)

  /* Configure the I2S extended if the full duplex mode is enabled */
  assert_param(IS_I2S_FULLDUPLEX_MODE(hi2s->Init.FullDuplexMode));

  if (hi2s->Init.FullDuplexMode == I2S_FULLDUPLEXMODE_ENABLE)
    8b4c:	687b      	ldr	r3, [r7, #4]
    8b4e:	6a1b      	ldr	r3, [r3, #32]
    8b50:	2b01      	cmp	r3, #1
    8b52:	d161      	bne.n	8c18 <HAL_I2S_Init+0x254>
  {
    /* Set FullDuplex I2S IrqHandler ISR if FULLDUPLEXMODE is enabled */
    hi2s->IrqHandlerISR = HAL_I2SEx_FullDuplex_IRQHandler;
    8b54:	687b      	ldr	r3, [r7, #4]
    8b56:	4a38      	ldr	r2, [pc, #224]	; (8c38 <HAL_I2S_Init+0x274>)
    8b58:	635a      	str	r2, [r3, #52]	; 0x34

    /* Clear I2SMOD, I2SE, I2SCFG, PCMSYNC, I2SSTD, CKPOL, DATLEN and CHLEN bits */
    CLEAR_BIT(I2SxEXT(hi2s->Instance)->I2SCFGR, (SPI_I2SCFGR_CHLEN | SPI_I2SCFGR_DATLEN | SPI_I2SCFGR_CKPOL | \
    8b5a:	687b      	ldr	r3, [r7, #4]
    8b5c:	681b      	ldr	r3, [r3, #0]
    8b5e:	4a37      	ldr	r2, [pc, #220]	; (8c3c <HAL_I2S_Init+0x278>)
    8b60:	4293      	cmp	r3, r2
    8b62:	d101      	bne.n	8b68 <HAL_I2S_Init+0x1a4>
    8b64:	4b36      	ldr	r3, [pc, #216]	; (8c40 <HAL_I2S_Init+0x27c>)
    8b66:	e001      	b.n	8b6c <HAL_I2S_Init+0x1a8>
    8b68:	f04f 2340 	mov.w	r3, #1073758208	; 0x40004000
    8b6c:	69db      	ldr	r3, [r3, #28]
    8b6e:	687a      	ldr	r2, [r7, #4]
    8b70:	6812      	ldr	r2, [r2, #0]
    8b72:	4932      	ldr	r1, [pc, #200]	; (8c3c <HAL_I2S_Init+0x278>)
    8b74:	428a      	cmp	r2, r1
    8b76:	d101      	bne.n	8b7c <HAL_I2S_Init+0x1b8>
    8b78:	4a31      	ldr	r2, [pc, #196]	; (8c40 <HAL_I2S_Init+0x27c>)
    8b7a:	e001      	b.n	8b80 <HAL_I2S_Init+0x1bc>
    8b7c:	f04f 2240 	mov.w	r2, #1073758208	; 0x40004000
    8b80:	f423 637b 	bic.w	r3, r3, #4016	; 0xfb0
    8b84:	f023 030f 	bic.w	r3, r3, #15
    8b88:	61d3      	str	r3, [r2, #28]
                                                 SPI_I2SCFGR_I2SSTD | SPI_I2SCFGR_PCMSYNC | SPI_I2SCFGR_I2SCFG | \
                                                 SPI_I2SCFGR_I2SE | SPI_I2SCFGR_I2SMOD));
    I2SxEXT(hi2s->Instance)->I2SPR = 2U;
    8b8a:	687b      	ldr	r3, [r7, #4]
    8b8c:	681b      	ldr	r3, [r3, #0]
    8b8e:	4a2b      	ldr	r2, [pc, #172]	; (8c3c <HAL_I2S_Init+0x278>)
    8b90:	4293      	cmp	r3, r2
    8b92:	d101      	bne.n	8b98 <HAL_I2S_Init+0x1d4>
    8b94:	4b2a      	ldr	r3, [pc, #168]	; (8c40 <HAL_I2S_Init+0x27c>)
    8b96:	e001      	b.n	8b9c <HAL_I2S_Init+0x1d8>
    8b98:	f04f 2340 	mov.w	r3, #1073758208	; 0x40004000
    8b9c:	2202      	movs	r2, #2
    8b9e:	621a      	str	r2, [r3, #32]

    /* Get the I2SCFGR register value */
    tmpreg = I2SxEXT(hi2s->Instance)->I2SCFGR;
    8ba0:	687b      	ldr	r3, [r7, #4]
    8ba2:	681b      	ldr	r3, [r3, #0]
    8ba4:	4a25      	ldr	r2, [pc, #148]	; (8c3c <HAL_I2S_Init+0x278>)
    8ba6:	4293      	cmp	r3, r2
    8ba8:	d101      	bne.n	8bae <HAL_I2S_Init+0x1ea>
    8baa:	4b25      	ldr	r3, [pc, #148]	; (8c40 <HAL_I2S_Init+0x27c>)
    8bac:	e001      	b.n	8bb2 <HAL_I2S_Init+0x1ee>
    8bae:	f04f 2340 	mov.w	r3, #1073758208	; 0x40004000
    8bb2:	69db      	ldr	r3, [r3, #28]
    8bb4:	817b      	strh	r3, [r7, #10]

    /* Get the mode to be configured for the extended I2S */
    if ((hi2s->Init.Mode == I2S_MODE_MASTER_TX) || (hi2s->Init.Mode == I2S_MODE_SLAVE_TX))
    8bb6:	687b      	ldr	r3, [r7, #4]
    8bb8:	685b      	ldr	r3, [r3, #4]
    8bba:	f5b3 7f00 	cmp.w	r3, #512	; 0x200
    8bbe:	d003      	beq.n	8bc8 <HAL_I2S_Init+0x204>
    8bc0:	687b      	ldr	r3, [r7, #4]
    8bc2:	685b      	ldr	r3, [r3, #4]
    8bc4:	2b00      	cmp	r3, #0
    8bc6:	d103      	bne.n	8bd0 <HAL_I2S_Init+0x20c>
    {
      tmp = I2S_MODE_SLAVE_RX;
    8bc8:	f44f 7380 	mov.w	r3, #256	; 0x100
    8bcc:	613b      	str	r3, [r7, #16]
    8bce:	e001      	b.n	8bd4 <HAL_I2S_Init+0x210>
    }
    else /* I2S_MODE_MASTER_RX ||  I2S_MODE_SLAVE_RX */
    {
      tmp = I2S_MODE_SLAVE_TX;
    8bd0:	2300      	movs	r3, #0
    8bd2:	613b      	str	r3, [r7, #16]
    }

    /* Configure the I2S Slave with the I2S Master parameter values */
    tmpreg |= (uint16_t)((uint16_t)SPI_I2SCFGR_I2SMOD | (uint16_t)(tmp | \
    8bd4:	693b      	ldr	r3, [r7, #16]
    8bd6:	b29a      	uxth	r2, r3
                         (uint16_t)(hi2s->Init.Standard | (uint16_t)(hi2s->Init.DataFormat | \
    8bd8:	687b      	ldr	r3, [r7, #4]
    8bda:	689b      	ldr	r3, [r3, #8]
    8bdc:	b299      	uxth	r1, r3
    8bde:	687b      	ldr	r3, [r7, #4]
    8be0:	68db      	ldr	r3, [r3, #12]
    8be2:	b298      	uxth	r0, r3
                                    (uint16_t)hi2s->Init.CPOL))));
    8be4:	687b      	ldr	r3, [r7, #4]
    8be6:	699b      	ldr	r3, [r3, #24]
    8be8:	b29b      	uxth	r3, r3
                         (uint16_t)(hi2s->Init.Standard | (uint16_t)(hi2s->Init.DataFormat | \
    8bea:	4303      	orrs	r3, r0
    8bec:	b29b      	uxth	r3, r3
    8bee:	430b      	orrs	r3, r1
    8bf0:	b29b      	uxth	r3, r3
    tmpreg |= (uint16_t)((uint16_t)SPI_I2SCFGR_I2SMOD | (uint16_t)(tmp | \
    8bf2:	4313      	orrs	r3, r2
    8bf4:	b29a      	uxth	r2, r3
    8bf6:	897b      	ldrh	r3, [r7, #10]
    8bf8:	4313      	orrs	r3, r2
    8bfa:	b29b      	uxth	r3, r3
    8bfc:	f443 6300 	orr.w	r3, r3, #2048	; 0x800
    8c00:	817b      	strh	r3, [r7, #10]

    /* Write to SPIx I2SCFGR */
    WRITE_REG(I2SxEXT(hi2s->Instance)->I2SCFGR, tmpreg);
    8c02:	687b      	ldr	r3, [r7, #4]
    8c04:	681b      	ldr	r3, [r3, #0]
    8c06:	4a0d      	ldr	r2, [pc, #52]	; (8c3c <HAL_I2S_Init+0x278>)
    8c08:	4293      	cmp	r3, r2
    8c0a:	d101      	bne.n	8c10 <HAL_I2S_Init+0x24c>
    8c0c:	4b0c      	ldr	r3, [pc, #48]	; (8c40 <HAL_I2S_Init+0x27c>)
    8c0e:	e001      	b.n	8c14 <HAL_I2S_Init+0x250>
    8c10:	f04f 2340 	mov.w	r3, #1073758208	; 0x40004000
    8c14:	897a      	ldrh	r2, [r7, #10]
    8c16:	61da      	str	r2, [r3, #28]
  }
#endif /* SPI_I2S_FULLDUPLEX_SUPPORT */

  hi2s->ErrorCode = HAL_I2S_ERROR_NONE;
    8c18:	687b      	ldr	r3, [r7, #4]
    8c1a:	2200      	movs	r2, #0
    8c1c:	645a      	str	r2, [r3, #68]	; 0x44
  hi2s->State     = HAL_I2S_STATE_READY;
    8c1e:	687b      	ldr	r3, [r7, #4]
    8c20:	2201      	movs	r2, #1
    8c22:	f883 2041 	strb.w	r2, [r3, #65]	; 0x41

  return HAL_OK;
    8c26:	2300      	movs	r3, #0
}
    8c28:	4618      	mov	r0, r3
    8c2a:	3720      	adds	r7, #32
    8c2c:	46bd      	mov	sp, r7
    8c2e:	bd80      	pop	{r7, pc}
    8c30:	00008d3b 	.word	0x00008d3b
    8c34:	cccccccd 	.word	0xcccccccd
    8c38:	00008e51 	.word	0x00008e51
    8c3c:	40003800 	.word	0x40003800
    8c40:	40003400 	.word	0x40003400

00008c44 <HAL_I2S_TxCpltCallback>:
  * @param  hi2s pointer to a I2S_HandleTypeDef structure that contains
  *         the configuration information for I2S module
  * @retval None
  */
__weak void HAL_I2S_TxCpltCallback(I2S_HandleTypeDef *hi2s)
{
    8c44:	b480      	push	{r7}
    8c46:	b083      	sub	sp, #12
    8c48:	af00      	add	r7, sp, #0
    8c4a:	6078      	str	r0, [r7, #4]
  UNUSED(hi2s);

  /* NOTE : This function Should not be modified, when the callback is needed,
            the HAL_I2S_TxCpltCallback could be implemented in the user file
   */
}
    8c4c:	bf00      	nop
    8c4e:	370c      	adds	r7, #12
    8c50:	46bd      	mov	sp, r7
    8c52:	f85d 7b04 	ldr.w	r7, [sp], #4
    8c56:	4770      	bx	lr

00008c58 <HAL_I2S_RxCpltCallback>:
  * @param  hi2s pointer to a I2S_HandleTypeDef structure that contains
  *         the configuration information for I2S module
  * @retval None
  */
__weak void HAL_I2S_RxCpltCallback(I2S_HandleTypeDef *hi2s)
{
    8c58:	b480      	push	{r7}
    8c5a:	b083      	sub	sp, #12
    8c5c:	af00      	add	r7, sp, #0
    8c5e:	6078      	str	r0, [r7, #4]
  UNUSED(hi2s);

  /* NOTE : This function Should not be modified, when the callback is needed,
            the HAL_I2S_RxCpltCallback could be implemented in the user file
   */
}
    8c60:	bf00      	nop
    8c62:	370c      	adds	r7, #12
    8c64:	46bd      	mov	sp, r7
    8c66:	f85d 7b04 	ldr.w	r7, [sp], #4
    8c6a:	4770      	bx	lr

00008c6c <HAL_I2S_ErrorCallback>:
  * @param  hi2s pointer to a I2S_HandleTypeDef structure that contains
  *         the configuration information for I2S module
  * @retval None
  */
__weak void HAL_I2S_ErrorCallback(I2S_HandleTypeDef *hi2s)
{
    8c6c:	b480      	push	{r7}
    8c6e:	b083      	sub	sp, #12
    8c70:	af00      	add	r7, sp, #0
    8c72:	6078      	str	r0, [r7, #4]
  UNUSED(hi2s);

  /* NOTE : This function Should not be modified, when the callback is needed,
            the HAL_I2S_ErrorCallback could be implemented in the user file
   */
}
    8c74:	bf00      	nop
    8c76:	370c      	adds	r7, #12
    8c78:	46bd      	mov	sp, r7
    8c7a:	f85d 7b04 	ldr.w	r7, [sp], #4
    8c7e:	4770      	bx	lr

00008c80 <I2S_Transmit_IT>:
  * @param  hi2s pointer to a I2S_HandleTypeDef structure that contains
  *         the configuration information for I2S module
  * @retval None
  */
static void I2S_Transmit_IT(I2S_HandleTypeDef *hi2s)
{
    8c80:	b580      	push	{r7, lr}
    8c82:	b082      	sub	sp, #8
    8c84:	af00      	add	r7, sp, #0
    8c86:	6078      	str	r0, [r7, #4]
  /* Transmit data */
  hi2s->Instance->DR = (*hi2s->pTxBuffPtr);
    8c88:	687b      	ldr	r3, [r7, #4]
    8c8a:	6a5b      	ldr	r3, [r3, #36]	; 0x24
    8c8c:	881a      	ldrh	r2, [r3, #0]
    8c8e:	687b      	ldr	r3, [r7, #4]
    8c90:	681b      	ldr	r3, [r3, #0]
    8c92:	60da      	str	r2, [r3, #12]
  hi2s->pTxBuffPtr++;
    8c94:	687b      	ldr	r3, [r7, #4]
    8c96:	6a5b      	ldr	r3, [r3, #36]	; 0x24
    8c98:	1c9a      	adds	r2, r3, #2
    8c9a:	687b      	ldr	r3, [r7, #4]
    8c9c:	625a      	str	r2, [r3, #36]	; 0x24
  hi2s->TxXferCount--;
    8c9e:	687b      	ldr	r3, [r7, #4]
    8ca0:	8d5b      	ldrh	r3, [r3, #42]	; 0x2a
    8ca2:	b29b      	uxth	r3, r3
    8ca4:	3b01      	subs	r3, #1
    8ca6:	b29a      	uxth	r2, r3
    8ca8:	687b      	ldr	r3, [r7, #4]
    8caa:	855a      	strh	r2, [r3, #42]	; 0x2a

  if (hi2s->TxXferCount == 0U)
    8cac:	687b      	ldr	r3, [r7, #4]
    8cae:	8d5b      	ldrh	r3, [r3, #42]	; 0x2a
    8cb0:	b29b      	uxth	r3, r3
    8cb2:	2b00      	cmp	r3, #0
    8cb4:	d10e      	bne.n	8cd4 <I2S_Transmit_IT+0x54>
  {
    /* Disable TXE and ERR interrupt */
    __HAL_I2S_DISABLE_IT(hi2s, (I2S_IT_TXE | I2S_IT_ERR));
    8cb6:	687b      	ldr	r3, [r7, #4]
    8cb8:	681b      	ldr	r3, [r3, #0]
    8cba:	685a      	ldr	r2, [r3, #4]
    8cbc:	687b      	ldr	r3, [r7, #4]
    8cbe:	681b      	ldr	r3, [r3, #0]
    8cc0:	f022 02a0 	bic.w	r2, r2, #160	; 0xa0
    8cc4:	605a      	str	r2, [r3, #4]

    hi2s->State = HAL_I2S_STATE_READY;
    8cc6:	687b      	ldr	r3, [r7, #4]
    8cc8:	2201      	movs	r2, #1
    8cca:	f883 2041 	strb.w	r2, [r3, #65]	; 0x41
    /* Call user Tx complete callback */
#if (USE_HAL_I2S_REGISTER_CALLBACKS == 1U)
    hi2s->TxCpltCallback(hi2s);
#else
    HAL_I2S_TxCpltCallback(hi2s);
    8cce:	6878      	ldr	r0, [r7, #4]
    8cd0:	f7ff ffb8 	bl	8c44 <HAL_I2S_TxCpltCallback>
#endif /* USE_HAL_I2S_REGISTER_CALLBACKS */
  }
}
    8cd4:	bf00      	nop
    8cd6:	3708      	adds	r7, #8
    8cd8:	46bd      	mov	sp, r7
    8cda:	bd80      	pop	{r7, pc}

00008cdc <I2S_Receive_IT>:
  * @param  hi2s pointer to a I2S_HandleTypeDef structure that contains
  *         the configuration information for I2S module
  * @retval None
  */
static void I2S_Receive_IT(I2S_HandleTypeDef *hi2s)
{
    8cdc:	b580      	push	{r7, lr}
    8cde:	b082      	sub	sp, #8
    8ce0:	af00      	add	r7, sp, #0
    8ce2:	6078      	str	r0, [r7, #4]
  /* Receive data */
  (*hi2s->pRxBuffPtr) = (uint16_t)hi2s->Instance->DR;
    8ce4:	687b      	ldr	r3, [r7, #4]
    8ce6:	681b      	ldr	r3, [r3, #0]
    8ce8:	68da      	ldr	r2, [r3, #12]
    8cea:	687b      	ldr	r3, [r7, #4]
    8cec:	6adb      	ldr	r3, [r3, #44]	; 0x2c
    8cee:	b292      	uxth	r2, r2
    8cf0:	801a      	strh	r2, [r3, #0]
  hi2s->pRxBuffPtr++;
    8cf2:	687b      	ldr	r3, [r7, #4]
    8cf4:	6adb      	ldr	r3, [r3, #44]	; 0x2c
    8cf6:	1c9a      	adds	r2, r3, #2
    8cf8:	687b      	ldr	r3, [r7, #4]
    8cfa:	62da      	str	r2, [r3, #44]	; 0x2c
  hi2s->RxXferCount--;
    8cfc:	687b      	ldr	r3, [r7, #4]
    8cfe:	8e5b      	ldrh	r3, [r3, #50]	; 0x32
    8d00:	b29b      	uxth	r3, r3
    8d02:	3b01      	subs	r3, #1
    8d04:	b29a      	uxth	r2, r3
    8d06:	687b      	ldr	r3, [r7, #4]
    8d08:	865a      	strh	r2, [r3, #50]	; 0x32

  if (hi2s->RxXferCount == 0U)
    8d0a:	687b      	ldr	r3, [r7, #4]
    8d0c:	8e5b      	ldrh	r3, [r3, #50]	; 0x32
    8d0e:	b29b      	uxth	r3, r3
    8d10:	2b00      	cmp	r3, #0
    8d12:	d10e      	bne.n	8d32 <I2S_Receive_IT+0x56>
  {
    /* Disable RXNE and ERR interrupt */
    __HAL_I2S_DISABLE_IT(hi2s, (I2S_IT_RXNE | I2S_IT_ERR));
    8d14:	687b      	ldr	r3, [r7, #4]
    8d16:	681b      	ldr	r3, [r3, #0]
    8d18:	685a      	ldr	r2, [r3, #4]
    8d1a:	687b      	ldr	r3, [r7, #4]
    8d1c:	681b      	ldr	r3, [r3, #0]
    8d1e:	f022 0260 	bic.w	r2, r2, #96	; 0x60
    8d22:	605a      	str	r2, [r3, #4]

    hi2s->State = HAL_I2S_STATE_READY;
    8d24:	687b      	ldr	r3, [r7, #4]
    8d26:	2201      	movs	r2, #1
    8d28:	f883 2041 	strb.w	r2, [r3, #65]	; 0x41
    /* Call user Rx complete callback */
#if (USE_HAL_I2S_REGISTER_CALLBACKS == 1U)
    hi2s->RxCpltCallback(hi2s);
#else
    HAL_I2S_RxCpltCallback(hi2s);
    8d2c:	6878      	ldr	r0, [r7, #4]
    8d2e:	f7ff ff93 	bl	8c58 <HAL_I2S_RxCpltCallback>
#endif /* USE_HAL_I2S_REGISTER_CALLBACKS */
  }
}
    8d32:	bf00      	nop
    8d34:	3708      	adds	r7, #8
    8d36:	46bd      	mov	sp, r7
    8d38:	bd80      	pop	{r7, pc}

00008d3a <I2S_IRQHandler>:
  * @param  hi2s: pointer to a I2S_HandleTypeDef structure that contains
  *         the configuration information for I2S module
  * @retval None
  */
static void I2S_IRQHandler(I2S_HandleTypeDef *hi2s)
{
    8d3a:	b580      	push	{r7, lr}
    8d3c:	b086      	sub	sp, #24
    8d3e:	af00      	add	r7, sp, #0
    8d40:	6078      	str	r0, [r7, #4]
  __IO uint32_t i2ssr = hi2s->Instance->SR;
    8d42:	687b      	ldr	r3, [r7, #4]
    8d44:	681b      	ldr	r3, [r3, #0]
    8d46:	689b      	ldr	r3, [r3, #8]
    8d48:	617b      	str	r3, [r7, #20]

  if (hi2s->State == HAL_I2S_STATE_BUSY_RX)
    8d4a:	687b      	ldr	r3, [r7, #4]
    8d4c:	f893 3041 	ldrb.w	r3, [r3, #65]	; 0x41
    8d50:	b2db      	uxtb	r3, r3
    8d52:	2b04      	cmp	r3, #4
    8d54:	d13a      	bne.n	8dcc <I2S_IRQHandler+0x92>
  {
    /* I2S in mode Receiver ------------------------------------------------*/
    if (((i2ssr & I2S_FLAG_RXNE) == I2S_FLAG_RXNE) && (__HAL_I2S_GET_IT_SOURCE(hi2s, I2S_IT_RXNE) != RESET))
    8d56:	697b      	ldr	r3, [r7, #20]
    8d58:	f003 0301 	and.w	r3, r3, #1
    8d5c:	2b01      	cmp	r3, #1
    8d5e:	d109      	bne.n	8d74 <I2S_IRQHandler+0x3a>
    8d60:	687b      	ldr	r3, [r7, #4]
    8d62:	681b      	ldr	r3, [r3, #0]
    8d64:	685b      	ldr	r3, [r3, #4]
    8d66:	f003 0340 	and.w	r3, r3, #64	; 0x40
    8d6a:	2b40      	cmp	r3, #64	; 0x40
    8d6c:	d102      	bne.n	8d74 <I2S_IRQHandler+0x3a>
    {
      I2S_Receive_IT(hi2s);
    8d6e:	6878      	ldr	r0, [r7, #4]
    8d70:	f7ff ffb4 	bl	8cdc <I2S_Receive_IT>
    }

    /* I2S Overrun error interrupt occurred -------------------------------------*/
    if (((i2ssr & I2S_FLAG_OVR) == I2S_FLAG_OVR) && (__HAL_I2S_GET_IT_SOURCE(hi2s, I2S_IT_ERR) != RESET))
    8d74:	697b      	ldr	r3, [r7, #20]
    8d76:	f003 0340 	and.w	r3, r3, #64	; 0x40
    8d7a:	2b40      	cmp	r3, #64	; 0x40
    8d7c:	d126      	bne.n	8dcc <I2S_IRQHandler+0x92>
    8d7e:	687b      	ldr	r3, [r7, #4]
    8d80:	681b      	ldr	r3, [r3, #0]
    8d82:	685b      	ldr	r3, [r3, #4]
    8d84:	f003 0320 	and.w	r3, r3, #32
    8d88:	2b20      	cmp	r3, #32
    8d8a:	d11f      	bne.n	8dcc <I2S_IRQHandler+0x92>
    {
      /* Disable RXNE and ERR interrupt */
      __HAL_I2S_DISABLE_IT(hi2s, (I2S_IT_RXNE | I2S_IT_ERR));
    8d8c:	687b      	ldr	r3, [r7, #4]
    8d8e:	681b      	ldr	r3, [r3, #0]
    8d90:	685a      	ldr	r2, [r3, #4]
    8d92:	687b      	ldr	r3, [r7, #4]
    8d94:	681b      	ldr	r3, [r3, #0]
    8d96:	f022 0260 	bic.w	r2, r2, #96	; 0x60
    8d9a:	605a      	str	r2, [r3, #4]

      /* Clear Overrun flag */
      __HAL_I2S_CLEAR_OVRFLAG(hi2s);
    8d9c:	2300      	movs	r3, #0
    8d9e:	613b      	str	r3, [r7, #16]
    8da0:	687b      	ldr	r3, [r7, #4]
    8da2:	681b      	ldr	r3, [r3, #0]
    8da4:	68db      	ldr	r3, [r3, #12]
    8da6:	613b      	str	r3, [r7, #16]
    8da8:	687b      	ldr	r3, [r7, #4]
    8daa:	681b      	ldr	r3, [r3, #0]
    8dac:	689b      	ldr	r3, [r3, #8]
    8dae:	613b      	str	r3, [r7, #16]
    8db0:	693b      	ldr	r3, [r7, #16]

      /* Set the I2S State ready */
      hi2s->State = HAL_I2S_STATE_READY;
    8db2:	687b      	ldr	r3, [r7, #4]
    8db4:	2201      	movs	r2, #1
    8db6:	f883 2041 	strb.w	r2, [r3, #65]	; 0x41


      /* Set the error code and execute error callback*/
      SET_BIT(hi2s->ErrorCode, HAL_I2S_ERROR_OVR);
    8dba:	687b      	ldr	r3, [r7, #4]
    8dbc:	6c5b      	ldr	r3, [r3, #68]	; 0x44
    8dbe:	f043 0202 	orr.w	r2, r3, #2
    8dc2:	687b      	ldr	r3, [r7, #4]
    8dc4:	645a      	str	r2, [r3, #68]	; 0x44
      /* Call user error callback */
#if (USE_HAL_I2S_REGISTER_CALLBACKS == 1U)
      hi2s->ErrorCallback(hi2s);
#else
      HAL_I2S_ErrorCallback(hi2s);
    8dc6:	6878      	ldr	r0, [r7, #4]
    8dc8:	f7ff ff50 	bl	8c6c <HAL_I2S_ErrorCallback>
#endif /* USE_HAL_I2S_REGISTER_CALLBACKS */
    }
  }

  if (hi2s->State == HAL_I2S_STATE_BUSY_TX)
    8dcc:	687b      	ldr	r3, [r7, #4]
    8dce:	f893 3041 	ldrb.w	r3, [r3, #65]	; 0x41
    8dd2:	b2db      	uxtb	r3, r3
    8dd4:	2b03      	cmp	r3, #3
    8dd6:	d136      	bne.n	8e46 <I2S_IRQHandler+0x10c>
  {
    /* I2S in mode Transmitter -----------------------------------------------*/
    if (((i2ssr & I2S_FLAG_TXE) == I2S_FLAG_TXE) && (__HAL_I2S_GET_IT_SOURCE(hi2s, I2S_IT_TXE) != RESET))
    8dd8:	697b      	ldr	r3, [r7, #20]
    8dda:	f003 0302 	and.w	r3, r3, #2
    8dde:	2b02      	cmp	r3, #2
    8de0:	d109      	bne.n	8df6 <I2S_IRQHandler+0xbc>
    8de2:	687b      	ldr	r3, [r7, #4]
    8de4:	681b      	ldr	r3, [r3, #0]
    8de6:	685b      	ldr	r3, [r3, #4]
    8de8:	f003 0380 	and.w	r3, r3, #128	; 0x80
    8dec:	2b80      	cmp	r3, #128	; 0x80
    8dee:	d102      	bne.n	8df6 <I2S_IRQHandler+0xbc>
    {
      I2S_Transmit_IT(hi2s);
    8df0:	6878      	ldr	r0, [r7, #4]
    8df2:	f7ff ff45 	bl	8c80 <I2S_Transmit_IT>
    }

    /* I2S Underrun error interrupt occurred --------------------------------*/
    if (((i2ssr & I2S_FLAG_UDR) == I2S_FLAG_UDR) && (__HAL_I2S_GET_IT_SOURCE(hi2s, I2S_IT_ERR) != RESET))
    8df6:	697b      	ldr	r3, [r7, #20]
    8df8:	f003 0308 	and.w	r3, r3, #8
    8dfc:	2b08      	cmp	r3, #8
    8dfe:	d122      	bne.n	8e46 <I2S_IRQHandler+0x10c>
    8e00:	687b      	ldr	r3, [r7, #4]
    8e02:	681b      	ldr	r3, [r3, #0]
    8e04:	685b      	ldr	r3, [r3, #4]
    8e06:	f003 0320 	and.w	r3, r3, #32
    8e0a:	2b20      	cmp	r3, #32
    8e0c:	d11b      	bne.n	8e46 <I2S_IRQHandler+0x10c>
    {
      /* Disable TXE and ERR interrupt */
      __HAL_I2S_DISABLE_IT(hi2s, (I2S_IT_TXE | I2S_IT_ERR));
    8e0e:	687b      	ldr	r3, [r7, #4]
    8e10:	681b      	ldr	r3, [r3, #0]
    8e12:	685a      	ldr	r2, [r3, #4]
    8e14:	687b      	ldr	r3, [r7, #4]
    8e16:	681b      	ldr	r3, [r3, #0]
    8e18:	f022 02a0 	bic.w	r2, r2, #160	; 0xa0
    8e1c:	605a      	str	r2, [r3, #4]

      /* Clear Underrun flag */
      __HAL_I2S_CLEAR_UDRFLAG(hi2s);
    8e1e:	2300      	movs	r3, #0
    8e20:	60fb      	str	r3, [r7, #12]
    8e22:	687b      	ldr	r3, [r7, #4]
    8e24:	681b      	ldr	r3, [r3, #0]
    8e26:	689b      	ldr	r3, [r3, #8]
    8e28:	60fb      	str	r3, [r7, #12]
    8e2a:	68fb      	ldr	r3, [r7, #12]

      /* Set the I2S State ready */
      hi2s->State = HAL_I2S_STATE_READY;
    8e2c:	687b      	ldr	r3, [r7, #4]
    8e2e:	2201      	movs	r2, #1
    8e30:	f883 2041 	strb.w	r2, [r3, #65]	; 0x41

      /* Set the error code and execute error callback*/
      SET_BIT(hi2s->ErrorCode, HAL_I2S_ERROR_UDR);
    8e34:	687b      	ldr	r3, [r7, #4]
    8e36:	6c5b      	ldr	r3, [r3, #68]	; 0x44
    8e38:	f043 0204 	orr.w	r2, r3, #4
    8e3c:	687b      	ldr	r3, [r7, #4]
    8e3e:	645a      	str	r2, [r3, #68]	; 0x44
      /* Call user error callback */
#if (USE_HAL_I2S_REGISTER_CALLBACKS == 1U)
      hi2s->ErrorCallback(hi2s);
#else
      HAL_I2S_ErrorCallback(hi2s);
    8e40:	6878      	ldr	r0, [r7, #4]
    8e42:	f7ff ff13 	bl	8c6c <HAL_I2S_ErrorCallback>
#endif /* USE_HAL_I2S_REGISTER_CALLBACKS */
    }
  }
}
    8e46:	bf00      	nop
    8e48:	3718      	adds	r7, #24
    8e4a:	46bd      	mov	sp, r7
    8e4c:	bd80      	pop	{r7, pc}
	...

00008e50 <HAL_I2SEx_FullDuplex_IRQHandler>:
  * @brief  This function handles I2S/I2Sext interrupt requests in full-duplex mode.
  * @param  hi2s I2S handle
  * @retval HAL status
  */
void HAL_I2SEx_FullDuplex_IRQHandler(I2S_HandleTypeDef *hi2s)
{
    8e50:	b580      	push	{r7, lr}
    8e52:	b088      	sub	sp, #32
    8e54:	af00      	add	r7, sp, #0
    8e56:	6078      	str	r0, [r7, #4]
  __IO uint32_t i2ssr     = hi2s->Instance->SR;
    8e58:	687b      	ldr	r3, [r7, #4]
    8e5a:	681b      	ldr	r3, [r3, #0]
    8e5c:	689b      	ldr	r3, [r3, #8]
    8e5e:	61fb      	str	r3, [r7, #28]
  __IO uint32_t i2sextsr  = I2SxEXT(hi2s->Instance)->SR;
    8e60:	687b      	ldr	r3, [r7, #4]
    8e62:	681b      	ldr	r3, [r3, #0]
    8e64:	4aa2      	ldr	r2, [pc, #648]	; (90f0 <HAL_I2SEx_FullDuplex_IRQHandler+0x2a0>)
    8e66:	4293      	cmp	r3, r2
    8e68:	d101      	bne.n	8e6e <HAL_I2SEx_FullDuplex_IRQHandler+0x1e>
    8e6a:	4ba2      	ldr	r3, [pc, #648]	; (90f4 <HAL_I2SEx_FullDuplex_IRQHandler+0x2a4>)
    8e6c:	e001      	b.n	8e72 <HAL_I2SEx_FullDuplex_IRQHandler+0x22>
    8e6e:	f04f 2340 	mov.w	r3, #1073758208	; 0x40004000
    8e72:	689b      	ldr	r3, [r3, #8]
    8e74:	61bb      	str	r3, [r7, #24]
  __IO uint32_t i2scr2    = hi2s->Instance->CR2;
    8e76:	687b      	ldr	r3, [r7, #4]
    8e78:	681b      	ldr	r3, [r3, #0]
    8e7a:	685b      	ldr	r3, [r3, #4]
    8e7c:	617b      	str	r3, [r7, #20]
  __IO uint32_t i2sextcr2 = I2SxEXT(hi2s->Instance)->CR2;
    8e7e:	687b      	ldr	r3, [r7, #4]
    8e80:	681b      	ldr	r3, [r3, #0]
    8e82:	4a9b      	ldr	r2, [pc, #620]	; (90f0 <HAL_I2SEx_FullDuplex_IRQHandler+0x2a0>)
    8e84:	4293      	cmp	r3, r2
    8e86:	d101      	bne.n	8e8c <HAL_I2SEx_FullDuplex_IRQHandler+0x3c>
    8e88:	4b9a      	ldr	r3, [pc, #616]	; (90f4 <HAL_I2SEx_FullDuplex_IRQHandler+0x2a4>)
    8e8a:	e001      	b.n	8e90 <HAL_I2SEx_FullDuplex_IRQHandler+0x40>
    8e8c:	f04f 2340 	mov.w	r3, #1073758208	; 0x40004000
    8e90:	685b      	ldr	r3, [r3, #4]
    8e92:	613b      	str	r3, [r7, #16]

  /* Check if the I2S_MODE_MASTER_TX or I2S_MODE_SLAVE_TX Mode is selected */
  if ((hi2s->Init.Mode == I2S_MODE_MASTER_TX) || (hi2s->Init.Mode == I2S_MODE_SLAVE_TX))
    8e94:	687b      	ldr	r3, [r7, #4]
    8e96:	685b      	ldr	r3, [r3, #4]
    8e98:	f5b3 7f00 	cmp.w	r3, #512	; 0x200
    8e9c:	d004      	beq.n	8ea8 <HAL_I2SEx_FullDuplex_IRQHandler+0x58>
    8e9e:	687b      	ldr	r3, [r7, #4]
    8ea0:	685b      	ldr	r3, [r3, #4]
    8ea2:	2b00      	cmp	r3, #0
    8ea4:	f040 8099 	bne.w	8fda <HAL_I2SEx_FullDuplex_IRQHandler+0x18a>
  {
    /* I2S in mode Transmitter -------------------------------------------------*/
    if (((i2ssr & I2S_FLAG_TXE) == I2S_FLAG_TXE) && ((i2scr2 & I2S_IT_TXE) != RESET))
    8ea8:	69fb      	ldr	r3, [r7, #28]
    8eaa:	f003 0302 	and.w	r3, r3, #2
    8eae:	2b02      	cmp	r3, #2
    8eb0:	d107      	bne.n	8ec2 <HAL_I2SEx_FullDuplex_IRQHandler+0x72>
    8eb2:	697b      	ldr	r3, [r7, #20]
    8eb4:	f003 0380 	and.w	r3, r3, #128	; 0x80
    8eb8:	2b00      	cmp	r3, #0
    8eba:	d002      	beq.n	8ec2 <HAL_I2SEx_FullDuplex_IRQHandler+0x72>
    {
      /* When the I2S mode is configured as I2S_MODE_MASTER_TX or I2S_MODE_SLAVE_TX,
      the I2S TXE interrupt will be generated to manage the full-duplex transmit phase. */
      I2SEx_TxISR_I2S(hi2s);
    8ebc:	6878      	ldr	r0, [r7, #4]
    8ebe:	f000 f925 	bl	910c <I2SEx_TxISR_I2S>
    }

    /* I2Sext in mode Receiver -----------------------------------------------*/
    if (((i2sextsr & I2S_FLAG_RXNE) == I2S_FLAG_RXNE) && ((i2sextcr2 & I2S_IT_RXNE) != RESET))
    8ec2:	69bb      	ldr	r3, [r7, #24]
    8ec4:	f003 0301 	and.w	r3, r3, #1
    8ec8:	2b01      	cmp	r3, #1
    8eca:	d107      	bne.n	8edc <HAL_I2SEx_FullDuplex_IRQHandler+0x8c>
    8ecc:	693b      	ldr	r3, [r7, #16]
    8ece:	f003 0340 	and.w	r3, r3, #64	; 0x40
    8ed2:	2b00      	cmp	r3, #0
    8ed4:	d002      	beq.n	8edc <HAL_I2SEx_FullDuplex_IRQHandler+0x8c>
    {
      /* When the I2S mode is configured as I2S_MODE_MASTER_TX or I2S_MODE_SLAVE_TX,
      the I2Sext RXNE interrupt will be generated to manage the full-duplex receive phase. */
      I2SEx_RxISR_I2SExt(hi2s);
    8ed6:	6878      	ldr	r0, [r7, #4]
    8ed8:	f000 f9c8 	bl	926c <I2SEx_RxISR_I2SExt>
    }

    /* I2Sext Overrun error interrupt occurred --------------------------------*/
    if (((i2sextsr & I2S_FLAG_OVR) == I2S_FLAG_OVR) && ((i2sextcr2 & I2S_IT_ERR) != RESET))
    8edc:	69bb      	ldr	r3, [r7, #24]
    8ede:	f003 0340 	and.w	r3, r3, #64	; 0x40
    8ee2:	2b40      	cmp	r3, #64	; 0x40
    8ee4:	d13a      	bne.n	8f5c <HAL_I2SEx_FullDuplex_IRQHandler+0x10c>
    8ee6:	693b      	ldr	r3, [r7, #16]
    8ee8:	f003 0320 	and.w	r3, r3, #32
    8eec:	2b00      	cmp	r3, #0
    8eee:	d035      	beq.n	8f5c <HAL_I2SEx_FullDuplex_IRQHandler+0x10c>
    {
      /* Disable RXNE and ERR interrupt */
      __HAL_I2SEXT_DISABLE_IT(hi2s, (I2S_IT_RXNE | I2S_IT_ERR));
    8ef0:	687b      	ldr	r3, [r7, #4]
    8ef2:	681b      	ldr	r3, [r3, #0]
    8ef4:	4a7e      	ldr	r2, [pc, #504]	; (90f0 <HAL_I2SEx_FullDuplex_IRQHandler+0x2a0>)
    8ef6:	4293      	cmp	r3, r2
    8ef8:	d101      	bne.n	8efe <HAL_I2SEx_FullDuplex_IRQHandler+0xae>
    8efa:	4b7e      	ldr	r3, [pc, #504]	; (90f4 <HAL_I2SEx_FullDuplex_IRQHandler+0x2a4>)
    8efc:	e001      	b.n	8f02 <HAL_I2SEx_FullDuplex_IRQHandler+0xb2>
    8efe:	f04f 2340 	mov.w	r3, #1073758208	; 0x40004000
    8f02:	685a      	ldr	r2, [r3, #4]
    8f04:	687b      	ldr	r3, [r7, #4]
    8f06:	681b      	ldr	r3, [r3, #0]
    8f08:	4979      	ldr	r1, [pc, #484]	; (90f0 <HAL_I2SEx_FullDuplex_IRQHandler+0x2a0>)
    8f0a:	428b      	cmp	r3, r1
    8f0c:	d101      	bne.n	8f12 <HAL_I2SEx_FullDuplex_IRQHandler+0xc2>
    8f0e:	4b79      	ldr	r3, [pc, #484]	; (90f4 <HAL_I2SEx_FullDuplex_IRQHandler+0x2a4>)
    8f10:	e001      	b.n	8f16 <HAL_I2SEx_FullDuplex_IRQHandler+0xc6>
    8f12:	f04f 2340 	mov.w	r3, #1073758208	; 0x40004000
    8f16:	f022 0260 	bic.w	r2, r2, #96	; 0x60
    8f1a:	605a      	str	r2, [r3, #4]

      /* Disable TXE and ERR interrupt */
      __HAL_I2S_DISABLE_IT(hi2s, (I2S_IT_TXE | I2S_IT_ERR));
    8f1c:	687b      	ldr	r3, [r7, #4]
    8f1e:	681b      	ldr	r3, [r3, #0]
    8f20:	685a      	ldr	r2, [r3, #4]
    8f22:	687b      	ldr	r3, [r7, #4]
    8f24:	681b      	ldr	r3, [r3, #0]
    8f26:	f022 02a0 	bic.w	r2, r2, #160	; 0xa0
    8f2a:	605a      	str	r2, [r3, #4]

      /* Clear Overrun flag */
      __HAL_I2S_CLEAR_OVRFLAG(hi2s);
    8f2c:	2300      	movs	r3, #0
    8f2e:	60fb      	str	r3, [r7, #12]
    8f30:	687b      	ldr	r3, [r7, #4]
    8f32:	681b      	ldr	r3, [r3, #0]
    8f34:	68db      	ldr	r3, [r3, #12]
    8f36:	60fb      	str	r3, [r7, #12]
    8f38:	687b      	ldr	r3, [r7, #4]
    8f3a:	681b      	ldr	r3, [r3, #0]
    8f3c:	689b      	ldr	r3, [r3, #8]
    8f3e:	60fb      	str	r3, [r7, #12]
    8f40:	68fb      	ldr	r3, [r7, #12]

      /* Set the I2S State ready */
      hi2s->State = HAL_I2S_STATE_READY;
    8f42:	687b      	ldr	r3, [r7, #4]
    8f44:	2201      	movs	r2, #1
    8f46:	f883 2041 	strb.w	r2, [r3, #65]	; 0x41

      /* Set the error code and execute error callback*/
      SET_BIT(hi2s->ErrorCode, HAL_I2S_ERROR_OVR);
    8f4a:	687b      	ldr	r3, [r7, #4]
    8f4c:	6c5b      	ldr	r3, [r3, #68]	; 0x44
    8f4e:	f043 0202 	orr.w	r2, r3, #2
    8f52:	687b      	ldr	r3, [r7, #4]
    8f54:	645a      	str	r2, [r3, #68]	; 0x44
      /* Call user error callback */
#if (USE_HAL_I2S_REGISTER_CALLBACKS == 1U)
      hi2s->ErrorCallback(hi2s);
#else
      HAL_I2S_ErrorCallback(hi2s);
    8f56:	6878      	ldr	r0, [r7, #4]
    8f58:	f7ff fe88 	bl	8c6c <HAL_I2S_ErrorCallback>
#endif /* USE_HAL_I2S_REGISTER_CALLBACKS */
    }

    /* I2S Underrun error interrupt occurred ----------------------------------*/
    if (((i2ssr & I2S_FLAG_UDR) == I2S_FLAG_UDR) && ((i2scr2 & I2S_IT_ERR) != RESET))
    8f5c:	69fb      	ldr	r3, [r7, #28]
    8f5e:	f003 0308 	and.w	r3, r3, #8
    8f62:	2b08      	cmp	r3, #8
    8f64:	f040 80be 	bne.w	90e4 <HAL_I2SEx_FullDuplex_IRQHandler+0x294>
    8f68:	697b      	ldr	r3, [r7, #20]
    8f6a:	f003 0320 	and.w	r3, r3, #32
    8f6e:	2b00      	cmp	r3, #0
    8f70:	f000 80b8 	beq.w	90e4 <HAL_I2SEx_FullDuplex_IRQHandler+0x294>
    {
      /* Disable TXE and ERR interrupt */
      __HAL_I2S_DISABLE_IT(hi2s, (I2S_IT_TXE | I2S_IT_ERR));
    8f74:	687b      	ldr	r3, [r7, #4]
    8f76:	681b      	ldr	r3, [r3, #0]
    8f78:	685a      	ldr	r2, [r3, #4]
    8f7a:	687b      	ldr	r3, [r7, #4]
    8f7c:	681b      	ldr	r3, [r3, #0]
    8f7e:	f022 02a0 	bic.w	r2, r2, #160	; 0xa0
    8f82:	605a      	str	r2, [r3, #4]

      /* Disable RXNE and ERR interrupt */
      __HAL_I2SEXT_DISABLE_IT(hi2s, (I2S_IT_RXNE | I2S_IT_ERR));
    8f84:	687b      	ldr	r3, [r7, #4]
    8f86:	681b      	ldr	r3, [r3, #0]
    8f88:	4a59      	ldr	r2, [pc, #356]	; (90f0 <HAL_I2SEx_FullDuplex_IRQHandler+0x2a0>)
    8f8a:	4293      	cmp	r3, r2
    8f8c:	d101      	bne.n	8f92 <HAL_I2SEx_FullDuplex_IRQHandler+0x142>
    8f8e:	4b59      	ldr	r3, [pc, #356]	; (90f4 <HAL_I2SEx_FullDuplex_IRQHandler+0x2a4>)
    8f90:	e001      	b.n	8f96 <HAL_I2SEx_FullDuplex_IRQHandler+0x146>
    8f92:	f04f 2340 	mov.w	r3, #1073758208	; 0x40004000
    8f96:	685a      	ldr	r2, [r3, #4]
    8f98:	687b      	ldr	r3, [r7, #4]
    8f9a:	681b      	ldr	r3, [r3, #0]
    8f9c:	4954      	ldr	r1, [pc, #336]	; (90f0 <HAL_I2SEx_FullDuplex_IRQHandler+0x2a0>)
    8f9e:	428b      	cmp	r3, r1
    8fa0:	d101      	bne.n	8fa6 <HAL_I2SEx_FullDuplex_IRQHandler+0x156>
    8fa2:	4b54      	ldr	r3, [pc, #336]	; (90f4 <HAL_I2SEx_FullDuplex_IRQHandler+0x2a4>)
    8fa4:	e001      	b.n	8faa <HAL_I2SEx_FullDuplex_IRQHandler+0x15a>
    8fa6:	f04f 2340 	mov.w	r3, #1073758208	; 0x40004000
    8faa:	f022 0260 	bic.w	r2, r2, #96	; 0x60
    8fae:	605a      	str	r2, [r3, #4]

      /* Clear underrun flag */
      __HAL_I2S_CLEAR_UDRFLAG(hi2s);
    8fb0:	2300      	movs	r3, #0
    8fb2:	60bb      	str	r3, [r7, #8]
    8fb4:	687b      	ldr	r3, [r7, #4]
    8fb6:	681b      	ldr	r3, [r3, #0]
    8fb8:	689b      	ldr	r3, [r3, #8]
    8fba:	60bb      	str	r3, [r7, #8]
    8fbc:	68bb      	ldr	r3, [r7, #8]

      /* Set the I2S State ready */
      hi2s->State = HAL_I2S_STATE_READY;
    8fbe:	687b      	ldr	r3, [r7, #4]
    8fc0:	2201      	movs	r2, #1
    8fc2:	f883 2041 	strb.w	r2, [r3, #65]	; 0x41

      /* Set the error code and execute error callback*/
      SET_BIT(hi2s->ErrorCode, HAL_I2S_ERROR_UDR);
    8fc6:	687b      	ldr	r3, [r7, #4]
    8fc8:	6c5b      	ldr	r3, [r3, #68]	; 0x44
    8fca:	f043 0204 	orr.w	r2, r3, #4
    8fce:	687b      	ldr	r3, [r7, #4]
    8fd0:	645a      	str	r2, [r3, #68]	; 0x44
      /* Call user error callback */
#if (USE_HAL_I2S_REGISTER_CALLBACKS == 1U)
      hi2s->ErrorCallback(hi2s);
#else
      HAL_I2S_ErrorCallback(hi2s);
    8fd2:	6878      	ldr	r0, [r7, #4]
    8fd4:	f7ff fe4a 	bl	8c6c <HAL_I2S_ErrorCallback>
    if (((i2ssr & I2S_FLAG_UDR) == I2S_FLAG_UDR) && ((i2scr2 & I2S_IT_ERR) != RESET))
    8fd8:	e084      	b.n	90e4 <HAL_I2SEx_FullDuplex_IRQHandler+0x294>
  }
  /* The I2S_MODE_MASTER_RX or I2S_MODE_SLAVE_RX Mode is selected */
  else
  {
    /* I2Sext in mode Transmitter ----------------------------------------------*/
    if (((i2sextsr & I2S_FLAG_TXE) == I2S_FLAG_TXE) && ((i2sextcr2 & I2S_IT_TXE) != RESET))
    8fda:	69bb      	ldr	r3, [r7, #24]
    8fdc:	f003 0302 	and.w	r3, r3, #2
    8fe0:	2b02      	cmp	r3, #2
    8fe2:	d107      	bne.n	8ff4 <HAL_I2SEx_FullDuplex_IRQHandler+0x1a4>
    8fe4:	693b      	ldr	r3, [r7, #16]
    8fe6:	f003 0380 	and.w	r3, r3, #128	; 0x80
    8fea:	2b00      	cmp	r3, #0
    8fec:	d002      	beq.n	8ff4 <HAL_I2SEx_FullDuplex_IRQHandler+0x1a4>
    {
      /* When the I2S mode is configured as I2S_MODE_MASTER_RX or I2S_MODE_SLAVE_RX,
      the I2Sext TXE interrupt will be generated to manage the full-duplex transmit phase. */
      I2SEx_TxISR_I2SExt(hi2s);
    8fee:	6878      	ldr	r0, [r7, #4]
    8ff0:	f000 f8be 	bl	9170 <I2SEx_TxISR_I2SExt>
    }

    /* I2S in mode Receiver --------------------------------------------------*/
    if (((i2ssr & I2S_FLAG_RXNE) == I2S_FLAG_RXNE) && ((i2scr2 & I2S_IT_RXNE) != RESET))
    8ff4:	69fb      	ldr	r3, [r7, #28]
    8ff6:	f003 0301 	and.w	r3, r3, #1
    8ffa:	2b01      	cmp	r3, #1
    8ffc:	d107      	bne.n	900e <HAL_I2SEx_FullDuplex_IRQHandler+0x1be>
    8ffe:	697b      	ldr	r3, [r7, #20]
    9000:	f003 0340 	and.w	r3, r3, #64	; 0x40
    9004:	2b00      	cmp	r3, #0
    9006:	d002      	beq.n	900e <HAL_I2SEx_FullDuplex_IRQHandler+0x1be>
    {
      /* When the I2S mode is configured as I2S_MODE_MASTER_RX or I2S_MODE_SLAVE_RX,
      the I2S RXNE interrupt will be generated to manage the full-duplex receive phase. */
      I2SEx_RxISR_I2S(hi2s);
    9008:	6878      	ldr	r0, [r7, #4]
    900a:	f000 f8fd 	bl	9208 <I2SEx_RxISR_I2S>
    }

    /* I2S Overrun error interrupt occurred -------------------------------------*/
    if (((i2ssr & I2S_FLAG_OVR) == I2S_FLAG_OVR) && ((i2scr2 & I2S_IT_ERR) != RESET))
    900e:	69fb      	ldr	r3, [r7, #28]
    9010:	f003 0340 	and.w	r3, r3, #64	; 0x40
    9014:	2b40      	cmp	r3, #64	; 0x40
    9016:	d12f      	bne.n	9078 <HAL_I2SEx_FullDuplex_IRQHandler+0x228>
    9018:	697b      	ldr	r3, [r7, #20]
    901a:	f003 0320 	and.w	r3, r3, #32
    901e:	2b00      	cmp	r3, #0
    9020:	d02a      	beq.n	9078 <HAL_I2SEx_FullDuplex_IRQHandler+0x228>
    {
      /* Disable RXNE and ERR interrupt */
      __HAL_I2S_DISABLE_IT(hi2s, (I2S_IT_RXNE | I2S_IT_ERR));
    9022:	687b      	ldr	r3, [r7, #4]
    9024:	681b      	ldr	r3, [r3, #0]
    9026:	685a      	ldr	r2, [r3, #4]
    9028:	687b      	ldr	r3, [r7, #4]
    902a:	681b      	ldr	r3, [r3, #0]
    902c:	f022 0260 	bic.w	r2, r2, #96	; 0x60
    9030:	605a      	str	r2, [r3, #4]

      /* Disable TXE and ERR interrupt */
      __HAL_I2SEXT_DISABLE_IT(hi2s, (I2S_IT_TXE | I2S_IT_ERR));
    9032:	687b      	ldr	r3, [r7, #4]
    9034:	681b      	ldr	r3, [r3, #0]
    9036:	4a2e      	ldr	r2, [pc, #184]	; (90f0 <HAL_I2SEx_FullDuplex_IRQHandler+0x2a0>)
    9038:	4293      	cmp	r3, r2
    903a:	d101      	bne.n	9040 <HAL_I2SEx_FullDuplex_IRQHandler+0x1f0>
    903c:	4b2d      	ldr	r3, [pc, #180]	; (90f4 <HAL_I2SEx_FullDuplex_IRQHandler+0x2a4>)
    903e:	e001      	b.n	9044 <HAL_I2SEx_FullDuplex_IRQHandler+0x1f4>
    9040:	f04f 2340 	mov.w	r3, #1073758208	; 0x40004000
    9044:	685a      	ldr	r2, [r3, #4]
    9046:	687b      	ldr	r3, [r7, #4]
    9048:	681b      	ldr	r3, [r3, #0]
    904a:	4929      	ldr	r1, [pc, #164]	; (90f0 <HAL_I2SEx_FullDuplex_IRQHandler+0x2a0>)
    904c:	428b      	cmp	r3, r1
    904e:	d101      	bne.n	9054 <HAL_I2SEx_FullDuplex_IRQHandler+0x204>
    9050:	4b28      	ldr	r3, [pc, #160]	; (90f4 <HAL_I2SEx_FullDuplex_IRQHandler+0x2a4>)
    9052:	e001      	b.n	9058 <HAL_I2SEx_FullDuplex_IRQHandler+0x208>
    9054:	f04f 2340 	mov.w	r3, #1073758208	; 0x40004000
    9058:	f022 02a0 	bic.w	r2, r2, #160	; 0xa0
    905c:	605a      	str	r2, [r3, #4]

      /* Set the I2S State ready */
      hi2s->State = HAL_I2S_STATE_READY;
    905e:	687b      	ldr	r3, [r7, #4]
    9060:	2201      	movs	r2, #1
    9062:	f883 2041 	strb.w	r2, [r3, #65]	; 0x41

      /* Set the error code and execute error callback*/
      SET_BIT(hi2s->ErrorCode, HAL_I2S_ERROR_OVR);
    9066:	687b      	ldr	r3, [r7, #4]
    9068:	6c5b      	ldr	r3, [r3, #68]	; 0x44
    906a:	f043 0202 	orr.w	r2, r3, #2
    906e:	687b      	ldr	r3, [r7, #4]
    9070:	645a      	str	r2, [r3, #68]	; 0x44
      /* Call user error callback */
#if (USE_HAL_I2S_REGISTER_CALLBACKS == 1U)
      hi2s->ErrorCallback(hi2s);
#else
      HAL_I2S_ErrorCallback(hi2s);
    9072:	6878      	ldr	r0, [r7, #4]
    9074:	f7ff fdfa 	bl	8c6c <HAL_I2S_ErrorCallback>
#endif /* USE_HAL_I2S_REGISTER_CALLBACKS */
    }

    /* I2Sext Underrun error interrupt occurred -------------------------------*/
    if (((i2sextsr & I2S_FLAG_UDR) == I2S_FLAG_UDR) && ((i2sextcr2 & I2S_IT_ERR) != RESET))
    9078:	69bb      	ldr	r3, [r7, #24]
    907a:	f003 0308 	and.w	r3, r3, #8
    907e:	2b08      	cmp	r3, #8
    9080:	d131      	bne.n	90e6 <HAL_I2SEx_FullDuplex_IRQHandler+0x296>
    9082:	693b      	ldr	r3, [r7, #16]
    9084:	f003 0320 	and.w	r3, r3, #32
    9088:	2b00      	cmp	r3, #0
    908a:	d02c      	beq.n	90e6 <HAL_I2SEx_FullDuplex_IRQHandler+0x296>
    {
      /* Disable TXE and ERR interrupt */
      __HAL_I2SEXT_DISABLE_IT(hi2s, (I2S_IT_TXE | I2S_IT_ERR));
    908c:	687b      	ldr	r3, [r7, #4]
    908e:	681b      	ldr	r3, [r3, #0]
    9090:	4a17      	ldr	r2, [pc, #92]	; (90f0 <HAL_I2SEx_FullDuplex_IRQHandler+0x2a0>)
    9092:	4293      	cmp	r3, r2
    9094:	d101      	bne.n	909a <HAL_I2SEx_FullDuplex_IRQHandler+0x24a>
    9096:	4b17      	ldr	r3, [pc, #92]	; (90f4 <HAL_I2SEx_FullDuplex_IRQHandler+0x2a4>)
    9098:	e001      	b.n	909e <HAL_I2SEx_FullDuplex_IRQHandler+0x24e>
    909a:	f04f 2340 	mov.w	r3, #1073758208	; 0x40004000
    909e:	685a      	ldr	r2, [r3, #4]
    90a0:	687b      	ldr	r3, [r7, #4]
    90a2:	681b      	ldr	r3, [r3, #0]
    90a4:	4912      	ldr	r1, [pc, #72]	; (90f0 <HAL_I2SEx_FullDuplex_IRQHandler+0x2a0>)
    90a6:	428b      	cmp	r3, r1
    90a8:	d101      	bne.n	90ae <HAL_I2SEx_FullDuplex_IRQHandler+0x25e>
    90aa:	4b12      	ldr	r3, [pc, #72]	; (90f4 <HAL_I2SEx_FullDuplex_IRQHandler+0x2a4>)
    90ac:	e001      	b.n	90b2 <HAL_I2SEx_FullDuplex_IRQHandler+0x262>
    90ae:	f04f 2340 	mov.w	r3, #1073758208	; 0x40004000
    90b2:	f022 02a0 	bic.w	r2, r2, #160	; 0xa0
    90b6:	605a      	str	r2, [r3, #4]

      /* Disable RXNE and ERR interrupt */
      __HAL_I2S_DISABLE_IT(hi2s, (I2S_IT_RXNE | I2S_IT_ERR));
    90b8:	687b      	ldr	r3, [r7, #4]
    90ba:	681b      	ldr	r3, [r3, #0]
    90bc:	685a      	ldr	r2, [r3, #4]
    90be:	687b      	ldr	r3, [r7, #4]
    90c0:	681b      	ldr	r3, [r3, #0]
    90c2:	f022 0260 	bic.w	r2, r2, #96	; 0x60
    90c6:	605a      	str	r2, [r3, #4]

      /* Set the I2S State ready */
      hi2s->State = HAL_I2S_STATE_READY;
    90c8:	687b      	ldr	r3, [r7, #4]
    90ca:	2201      	movs	r2, #1
    90cc:	f883 2041 	strb.w	r2, [r3, #65]	; 0x41

      /* Set the error code and execute error callback*/
      SET_BIT(hi2s->ErrorCode, HAL_I2S_ERROR_UDR);
    90d0:	687b      	ldr	r3, [r7, #4]
    90d2:	6c5b      	ldr	r3, [r3, #68]	; 0x44
    90d4:	f043 0204 	orr.w	r2, r3, #4
    90d8:	687b      	ldr	r3, [r7, #4]
    90da:	645a      	str	r2, [r3, #68]	; 0x44
      /* Call user error callback */
#if (USE_HAL_I2S_REGISTER_CALLBACKS == 1U)
      hi2s->ErrorCallback(hi2s);
#else
      HAL_I2S_ErrorCallback(hi2s);
    90dc:	6878      	ldr	r0, [r7, #4]
    90de:	f7ff fdc5 	bl	8c6c <HAL_I2S_ErrorCallback>
#endif /* USE_HAL_I2S_REGISTER_CALLBACKS */
    }
  }
}
    90e2:	e000      	b.n	90e6 <HAL_I2SEx_FullDuplex_IRQHandler+0x296>
    if (((i2ssr & I2S_FLAG_UDR) == I2S_FLAG_UDR) && ((i2scr2 & I2S_IT_ERR) != RESET))
    90e4:	bf00      	nop
}
    90e6:	bf00      	nop
    90e8:	3720      	adds	r7, #32
    90ea:	46bd      	mov	sp, r7
    90ec:	bd80      	pop	{r7, pc}
    90ee:	bf00      	nop
    90f0:	40003800 	.word	0x40003800
    90f4:	40003400 	.word	0x40003400

000090f8 <HAL_I2SEx_TxRxCpltCallback>:
  * @brief  Tx and Rx Transfer completed callback
  * @param  hi2s I2S handle
  * @retval None
  */
__weak void HAL_I2SEx_TxRxCpltCallback(I2S_HandleTypeDef *hi2s)
{
    90f8:	b480      	push	{r7}
    90fa:	b083      	sub	sp, #12
    90fc:	af00      	add	r7, sp, #0
    90fe:	6078      	str	r0, [r7, #4]
  UNUSED(hi2s);

  /* NOTE : This function should not be modified, when the callback is needed,
            the HAL_I2SEx_TxRxCpltCallback could be implemented in the user file
   */
}
    9100:	bf00      	nop
    9102:	370c      	adds	r7, #12
    9104:	46bd      	mov	sp, r7
    9106:	f85d 7b04 	ldr.w	r7, [sp], #4
    910a:	4770      	bx	lr

0000910c <I2SEx_TxISR_I2S>:
  * @brief  I2S Full-Duplex IT handler transmit function
  * @param  hi2s I2S handle
  * @retval None
  */
static void I2SEx_TxISR_I2S(I2S_HandleTypeDef *hi2s)
{
    910c:	b580      	push	{r7, lr}
    910e:	b082      	sub	sp, #8
    9110:	af00      	add	r7, sp, #0
    9112:	6078      	str	r0, [r7, #4]
  /* Write Data on DR register */
  hi2s->Instance->DR = (*hi2s->pTxBuffPtr++);
    9114:	687b      	ldr	r3, [r7, #4]
    9116:	6a5b      	ldr	r3, [r3, #36]	; 0x24
    9118:	1c99      	adds	r1, r3, #2
    911a:	687a      	ldr	r2, [r7, #4]
    911c:	6251      	str	r1, [r2, #36]	; 0x24
    911e:	881a      	ldrh	r2, [r3, #0]
    9120:	687b      	ldr	r3, [r7, #4]
    9122:	681b      	ldr	r3, [r3, #0]
    9124:	60da      	str	r2, [r3, #12]
  hi2s->TxXferCount--;
    9126:	687b      	ldr	r3, [r7, #4]
    9128:	8d5b      	ldrh	r3, [r3, #42]	; 0x2a
    912a:	b29b      	uxth	r3, r3
    912c:	3b01      	subs	r3, #1
    912e:	b29a      	uxth	r2, r3
    9130:	687b      	ldr	r3, [r7, #4]
    9132:	855a      	strh	r2, [r3, #42]	; 0x2a

  if (hi2s->TxXferCount == 0U)
    9134:	687b      	ldr	r3, [r7, #4]
    9136:	8d5b      	ldrh	r3, [r3, #42]	; 0x2a
    9138:	b29b      	uxth	r3, r3
    913a:	2b00      	cmp	r3, #0
    913c:	d113      	bne.n	9166 <I2SEx_TxISR_I2S+0x5a>
  {
    /* Disable TXE and ERR interrupt */
    __HAL_I2S_DISABLE_IT(hi2s, (I2S_IT_TXE | I2S_IT_ERR));
    913e:	687b      	ldr	r3, [r7, #4]
    9140:	681b      	ldr	r3, [r3, #0]
    9142:	685a      	ldr	r2, [r3, #4]
    9144:	687b      	ldr	r3, [r7, #4]
    9146:	681b      	ldr	r3, [r3, #0]
    9148:	f022 02a0 	bic.w	r2, r2, #160	; 0xa0
    914c:	605a      	str	r2, [r3, #4]

    if (hi2s->RxXferCount == 0U)
    914e:	687b      	ldr	r3, [r7, #4]
    9150:	8e5b      	ldrh	r3, [r3, #50]	; 0x32
    9152:	b29b      	uxth	r3, r3
    9154:	2b00      	cmp	r3, #0
    9156:	d106      	bne.n	9166 <I2SEx_TxISR_I2S+0x5a>
    {
      hi2s->State = HAL_I2S_STATE_READY;
    9158:	687b      	ldr	r3, [r7, #4]
    915a:	2201      	movs	r2, #1
    915c:	f883 2041 	strb.w	r2, [r3, #65]	; 0x41
      /* Call user TxRx complete callback */
#if (USE_HAL_I2S_REGISTER_CALLBACKS == 1U)
      hi2s->TxRxCpltCallback(hi2s);
#else
      HAL_I2SEx_TxRxCpltCallback(hi2s);
    9160:	6878      	ldr	r0, [r7, #4]
    9162:	f7ff ffc9 	bl	90f8 <HAL_I2SEx_TxRxCpltCallback>
#endif /* USE_HAL_I2S_REGISTER_CALLBACKS */
    }
  }
}
    9166:	bf00      	nop
    9168:	3708      	adds	r7, #8
    916a:	46bd      	mov	sp, r7
    916c:	bd80      	pop	{r7, pc}
	...

00009170 <I2SEx_TxISR_I2SExt>:
  * @brief  I2SExt Full-Duplex IT handler transmit function
  * @param  hi2s I2S handle
  * @retval None
  */
static void I2SEx_TxISR_I2SExt(I2S_HandleTypeDef *hi2s)
{
    9170:	b580      	push	{r7, lr}
    9172:	b082      	sub	sp, #8
    9174:	af00      	add	r7, sp, #0
    9176:	6078      	str	r0, [r7, #4]
  /* Write Data on DR register */
  I2SxEXT(hi2s->Instance)->DR = (*hi2s->pTxBuffPtr++);
    9178:	687b      	ldr	r3, [r7, #4]
    917a:	6a5b      	ldr	r3, [r3, #36]	; 0x24
    917c:	1c99      	adds	r1, r3, #2
    917e:	687a      	ldr	r2, [r7, #4]
    9180:	6251      	str	r1, [r2, #36]	; 0x24
    9182:	8819      	ldrh	r1, [r3, #0]
    9184:	687b      	ldr	r3, [r7, #4]
    9186:	681b      	ldr	r3, [r3, #0]
    9188:	4a1d      	ldr	r2, [pc, #116]	; (9200 <I2SEx_TxISR_I2SExt+0x90>)
    918a:	4293      	cmp	r3, r2
    918c:	d101      	bne.n	9192 <I2SEx_TxISR_I2SExt+0x22>
    918e:	4b1d      	ldr	r3, [pc, #116]	; (9204 <I2SEx_TxISR_I2SExt+0x94>)
    9190:	e001      	b.n	9196 <I2SEx_TxISR_I2SExt+0x26>
    9192:	f04f 2340 	mov.w	r3, #1073758208	; 0x40004000
    9196:	460a      	mov	r2, r1
    9198:	60da      	str	r2, [r3, #12]
  hi2s->TxXferCount--;
    919a:	687b      	ldr	r3, [r7, #4]
    919c:	8d5b      	ldrh	r3, [r3, #42]	; 0x2a
    919e:	b29b      	uxth	r3, r3
    91a0:	3b01      	subs	r3, #1
    91a2:	b29a      	uxth	r2, r3
    91a4:	687b      	ldr	r3, [r7, #4]
    91a6:	855a      	strh	r2, [r3, #42]	; 0x2a

  if (hi2s->TxXferCount == 0U)
    91a8:	687b      	ldr	r3, [r7, #4]
    91aa:	8d5b      	ldrh	r3, [r3, #42]	; 0x2a
    91ac:	b29b      	uxth	r3, r3
    91ae:	2b00      	cmp	r3, #0
    91b0:	d121      	bne.n	91f6 <I2SEx_TxISR_I2SExt+0x86>
  {
    /* Disable I2Sext TXE and ERR interrupt */
    __HAL_I2SEXT_DISABLE_IT(hi2s, (I2S_IT_TXE | I2S_IT_ERR));
    91b2:	687b      	ldr	r3, [r7, #4]
    91b4:	681b      	ldr	r3, [r3, #0]
    91b6:	4a12      	ldr	r2, [pc, #72]	; (9200 <I2SEx_TxISR_I2SExt+0x90>)
    91b8:	4293      	cmp	r3, r2
    91ba:	d101      	bne.n	91c0 <I2SEx_TxISR_I2SExt+0x50>
    91bc:	4b11      	ldr	r3, [pc, #68]	; (9204 <I2SEx_TxISR_I2SExt+0x94>)
    91be:	e001      	b.n	91c4 <I2SEx_TxISR_I2SExt+0x54>
    91c0:	f04f 2340 	mov.w	r3, #1073758208	; 0x40004000
    91c4:	685a      	ldr	r2, [r3, #4]
    91c6:	687b      	ldr	r3, [r7, #4]
    91c8:	681b      	ldr	r3, [r3, #0]
    91ca:	490d      	ldr	r1, [pc, #52]	; (9200 <I2SEx_TxISR_I2SExt+0x90>)
    91cc:	428b      	cmp	r3, r1
    91ce:	d101      	bne.n	91d4 <I2SEx_TxISR_I2SExt+0x64>
    91d0:	4b0c      	ldr	r3, [pc, #48]	; (9204 <I2SEx_TxISR_I2SExt+0x94>)
    91d2:	e001      	b.n	91d8 <I2SEx_TxISR_I2SExt+0x68>
    91d4:	f04f 2340 	mov.w	r3, #1073758208	; 0x40004000
    91d8:	f022 02a0 	bic.w	r2, r2, #160	; 0xa0
    91dc:	605a      	str	r2, [r3, #4]

    if (hi2s->RxXferCount == 0U)
    91de:	687b      	ldr	r3, [r7, #4]
    91e0:	8e5b      	ldrh	r3, [r3, #50]	; 0x32
    91e2:	b29b      	uxth	r3, r3
    91e4:	2b00      	cmp	r3, #0
    91e6:	d106      	bne.n	91f6 <I2SEx_TxISR_I2SExt+0x86>
    {
      hi2s->State = HAL_I2S_STATE_READY;
    91e8:	687b      	ldr	r3, [r7, #4]
    91ea:	2201      	movs	r2, #1
    91ec:	f883 2041 	strb.w	r2, [r3, #65]	; 0x41
      /* Call user TxRx complete callback */
#if (USE_HAL_I2S_REGISTER_CALLBACKS == 1U)
      hi2s->TxRxCpltCallback(hi2s);
#else
      HAL_I2SEx_TxRxCpltCallback(hi2s);
    91f0:	6878      	ldr	r0, [r7, #4]
    91f2:	f7ff ff81 	bl	90f8 <HAL_I2SEx_TxRxCpltCallback>
#endif /* USE_HAL_I2S_REGISTER_CALLBACKS */
    }
  }
}
    91f6:	bf00      	nop
    91f8:	3708      	adds	r7, #8
    91fa:	46bd      	mov	sp, r7
    91fc:	bd80      	pop	{r7, pc}
    91fe:	bf00      	nop
    9200:	40003800 	.word	0x40003800
    9204:	40003400 	.word	0x40003400

00009208 <I2SEx_RxISR_I2S>:
  * @brief  I2S Full-Duplex IT handler receive function
  * @param  hi2s I2S handle
  * @retval None
  */
static void I2SEx_RxISR_I2S(I2S_HandleTypeDef *hi2s)
{
    9208:	b580      	push	{r7, lr}
    920a:	b082      	sub	sp, #8
    920c:	af00      	add	r7, sp, #0
    920e:	6078      	str	r0, [r7, #4]
  /* Read Data from DR register */
  (*hi2s->pRxBuffPtr++) = hi2s->Instance->DR;
    9210:	687b      	ldr	r3, [r7, #4]
    9212:	681b      	ldr	r3, [r3, #0]
    9214:	68d8      	ldr	r0, [r3, #12]
    9216:	687b      	ldr	r3, [r7, #4]
    9218:	6adb      	ldr	r3, [r3, #44]	; 0x2c
    921a:	1c99      	adds	r1, r3, #2
    921c:	687a      	ldr	r2, [r7, #4]
    921e:	62d1      	str	r1, [r2, #44]	; 0x2c
    9220:	b282      	uxth	r2, r0
    9222:	801a      	strh	r2, [r3, #0]
  hi2s->RxXferCount--;
    9224:	687b      	ldr	r3, [r7, #4]
    9226:	8e5b      	ldrh	r3, [r3, #50]	; 0x32
    9228:	b29b      	uxth	r3, r3
    922a:	3b01      	subs	r3, #1
    922c:	b29a      	uxth	r2, r3
    922e:	687b      	ldr	r3, [r7, #4]
    9230:	865a      	strh	r2, [r3, #50]	; 0x32

  if (hi2s->RxXferCount == 0U)
    9232:	687b      	ldr	r3, [r7, #4]
    9234:	8e5b      	ldrh	r3, [r3, #50]	; 0x32
    9236:	b29b      	uxth	r3, r3
    9238:	2b00      	cmp	r3, #0
    923a:	d113      	bne.n	9264 <I2SEx_RxISR_I2S+0x5c>
  {
    /* Disable RXNE and ERR interrupt */
    __HAL_I2S_DISABLE_IT(hi2s, (I2S_IT_RXNE | I2S_IT_ERR));
    923c:	687b      	ldr	r3, [r7, #4]
    923e:	681b      	ldr	r3, [r3, #0]
    9240:	685a      	ldr	r2, [r3, #4]
    9242:	687b      	ldr	r3, [r7, #4]
    9244:	681b      	ldr	r3, [r3, #0]
    9246:	f022 0260 	bic.w	r2, r2, #96	; 0x60
    924a:	605a      	str	r2, [r3, #4]

    if (hi2s->TxXferCount == 0U)
    924c:	687b      	ldr	r3, [r7, #4]
    924e:	8d5b      	ldrh	r3, [r3, #42]	; 0x2a
    9250:	b29b      	uxth	r3, r3
    9252:	2b00      	cmp	r3, #0
    9254:	d106      	bne.n	9264 <I2SEx_RxISR_I2S+0x5c>
    {
      hi2s->State = HAL_I2S_STATE_READY;
    9256:	687b      	ldr	r3, [r7, #4]
    9258:	2201      	movs	r2, #1
    925a:	f883 2041 	strb.w	r2, [r3, #65]	; 0x41
      /* Call user TxRx complete callback */
#if (USE_HAL_I2S_REGISTER_CALLBACKS == 1U)
      hi2s->TxRxCpltCallback(hi2s);
#else
      HAL_I2SEx_TxRxCpltCallback(hi2s);
    925e:	6878      	ldr	r0, [r7, #4]
    9260:	f7ff ff4a 	bl	90f8 <HAL_I2SEx_TxRxCpltCallback>
#endif /* USE_HAL_I2S_REGISTER_CALLBACKS */
    }
  }
}
    9264:	bf00      	nop
    9266:	3708      	adds	r7, #8
    9268:	46bd      	mov	sp, r7
    926a:	bd80      	pop	{r7, pc}

0000926c <I2SEx_RxISR_I2SExt>:
  * @brief  I2SExt Full-Duplex IT handler receive function
  * @param  hi2s I2S handle
  * @retval None
  */
static void I2SEx_RxISR_I2SExt(I2S_HandleTypeDef *hi2s)
{
    926c:	b580      	push	{r7, lr}
    926e:	b082      	sub	sp, #8
    9270:	af00      	add	r7, sp, #0
    9272:	6078      	str	r0, [r7, #4]
  /* Read Data from DR register */
  (*hi2s->pRxBuffPtr++) = I2SxEXT(hi2s->Instance)->DR;
    9274:	687b      	ldr	r3, [r7, #4]
    9276:	681b      	ldr	r3, [r3, #0]
    9278:	4a20      	ldr	r2, [pc, #128]	; (92fc <I2SEx_RxISR_I2SExt+0x90>)
    927a:	4293      	cmp	r3, r2
    927c:	d101      	bne.n	9282 <I2SEx_RxISR_I2SExt+0x16>
    927e:	4b20      	ldr	r3, [pc, #128]	; (9300 <I2SEx_RxISR_I2SExt+0x94>)
    9280:	e001      	b.n	9286 <I2SEx_RxISR_I2SExt+0x1a>
    9282:	f04f 2340 	mov.w	r3, #1073758208	; 0x40004000
    9286:	68d8      	ldr	r0, [r3, #12]
    9288:	687b      	ldr	r3, [r7, #4]
    928a:	6adb      	ldr	r3, [r3, #44]	; 0x2c
    928c:	1c99      	adds	r1, r3, #2
    928e:	687a      	ldr	r2, [r7, #4]
    9290:	62d1      	str	r1, [r2, #44]	; 0x2c
    9292:	b282      	uxth	r2, r0
    9294:	801a      	strh	r2, [r3, #0]
  hi2s->RxXferCount--;
    9296:	687b      	ldr	r3, [r7, #4]
    9298:	8e5b      	ldrh	r3, [r3, #50]	; 0x32
    929a:	b29b      	uxth	r3, r3
    929c:	3b01      	subs	r3, #1
    929e:	b29a      	uxth	r2, r3
    92a0:	687b      	ldr	r3, [r7, #4]
    92a2:	865a      	strh	r2, [r3, #50]	; 0x32

  if (hi2s->RxXferCount == 0U)
    92a4:	687b      	ldr	r3, [r7, #4]
    92a6:	8e5b      	ldrh	r3, [r3, #50]	; 0x32
    92a8:	b29b      	uxth	r3, r3
    92aa:	2b00      	cmp	r3, #0
    92ac:	d121      	bne.n	92f2 <I2SEx_RxISR_I2SExt+0x86>
  {
    /* Disable I2Sext RXNE and ERR interrupt */
    __HAL_I2SEXT_DISABLE_IT(hi2s, (I2S_IT_RXNE | I2S_IT_ERR));
    92ae:	687b      	ldr	r3, [r7, #4]
    92b0:	681b      	ldr	r3, [r3, #0]
    92b2:	4a12      	ldr	r2, [pc, #72]	; (92fc <I2SEx_RxISR_I2SExt+0x90>)
    92b4:	4293      	cmp	r3, r2
    92b6:	d101      	bne.n	92bc <I2SEx_RxISR_I2SExt+0x50>
    92b8:	4b11      	ldr	r3, [pc, #68]	; (9300 <I2SEx_RxISR_I2SExt+0x94>)
    92ba:	e001      	b.n	92c0 <I2SEx_RxISR_I2SExt+0x54>
    92bc:	f04f 2340 	mov.w	r3, #1073758208	; 0x40004000
    92c0:	685a      	ldr	r2, [r3, #4]
    92c2:	687b      	ldr	r3, [r7, #4]
    92c4:	681b      	ldr	r3, [r3, #0]
    92c6:	490d      	ldr	r1, [pc, #52]	; (92fc <I2SEx_RxISR_I2SExt+0x90>)
    92c8:	428b      	cmp	r3, r1
    92ca:	d101      	bne.n	92d0 <I2SEx_RxISR_I2SExt+0x64>
    92cc:	4b0c      	ldr	r3, [pc, #48]	; (9300 <I2SEx_RxISR_I2SExt+0x94>)
    92ce:	e001      	b.n	92d4 <I2SEx_RxISR_I2SExt+0x68>
    92d0:	f04f 2340 	mov.w	r3, #1073758208	; 0x40004000
    92d4:	f022 0260 	bic.w	r2, r2, #96	; 0x60
    92d8:	605a      	str	r2, [r3, #4]

    if (hi2s->TxXferCount == 0U)
    92da:	687b      	ldr	r3, [r7, #4]
    92dc:	8d5b      	ldrh	r3, [r3, #42]	; 0x2a
    92de:	b29b      	uxth	r3, r3
    92e0:	2b00      	cmp	r3, #0
    92e2:	d106      	bne.n	92f2 <I2SEx_RxISR_I2SExt+0x86>
    {
      hi2s->State = HAL_I2S_STATE_READY;
    92e4:	687b      	ldr	r3, [r7, #4]
    92e6:	2201      	movs	r2, #1
    92e8:	f883 2041 	strb.w	r2, [r3, #65]	; 0x41
      /* Call user TxRx complete callback */
#if (USE_HAL_I2S_REGISTER_CALLBACKS == 1U)
      hi2s->TxRxCpltCallback(hi2s);
#else
      HAL_I2SEx_TxRxCpltCallback(hi2s);
    92ec:	6878      	ldr	r0, [r7, #4]
    92ee:	f7ff ff03 	bl	90f8 <HAL_I2SEx_TxRxCpltCallback>
#endif /* USE_HAL_I2S_REGISTER_CALLBACKS */
    }
  }
}
    92f2:	bf00      	nop
    92f4:	3708      	adds	r7, #8
    92f6:	46bd      	mov	sp, r7
    92f8:	bd80      	pop	{r7, pc}
    92fa:	bf00      	nop
    92fc:	40003800 	.word	0x40003800
    9300:	40003400 	.word	0x40003400

00009304 <HAL_PCD_Init>:
  *         parameters in the PCD_InitTypeDef and initialize the associated handle.
  * @param  hpcd PCD handle
  * @retval HAL status
  */
HAL_StatusTypeDef HAL_PCD_Init(PCD_HandleTypeDef *hpcd)
{
    9304:	b5f0      	push	{r4, r5, r6, r7, lr}
    9306:	b08f      	sub	sp, #60	; 0x3c
    9308:	af0a      	add	r7, sp, #40	; 0x28
    930a:	6078      	str	r0, [r7, #4]
  USB_OTG_GlobalTypeDef *USBx;
  uint8_t i;

  /* Check the PCD handle allocation */
  if (hpcd == NULL)
    930c:	687b      	ldr	r3, [r7, #4]
    930e:	2b00      	cmp	r3, #0
    9310:	d101      	bne.n	9316 <HAL_PCD_Init+0x12>
  {
    return HAL_ERROR;
    9312:	2301      	movs	r3, #1
    9314:	e10f      	b.n	9536 <HAL_PCD_Init+0x232>
  }

  /* Check the parameters */
  assert_param(IS_PCD_ALL_INSTANCE(hpcd->Instance));

  USBx = hpcd->Instance;
    9316:	687b      	ldr	r3, [r7, #4]
    9318:	681b      	ldr	r3, [r3, #0]
    931a:	60bb      	str	r3, [r7, #8]

  if (hpcd->State == HAL_PCD_STATE_RESET)
    931c:	687b      	ldr	r3, [r7, #4]
    931e:	f893 33bd 	ldrb.w	r3, [r3, #957]	; 0x3bd
    9322:	b2db      	uxtb	r3, r3
    9324:	2b00      	cmp	r3, #0
    9326:	d106      	bne.n	9336 <HAL_PCD_Init+0x32>
  {
    /* Allocate lock resource and initialize it */
    hpcd->Lock = HAL_UNLOCKED;
    9328:	687b      	ldr	r3, [r7, #4]
    932a:	2200      	movs	r2, #0
    932c:	f883 23bc 	strb.w	r2, [r3, #956]	; 0x3bc

    /* Init the low level hardware */
    hpcd->MspInitCallback(hpcd);
#else
    /* Init the low level hardware : GPIO, CLOCK, NVIC... */
    HAL_PCD_MspInit(hpcd);
    9330:	6878      	ldr	r0, [r7, #4]
    9332:	f003 f99d 	bl	c670 <HAL_PCD_MspInit>
#endif /* (USE_HAL_PCD_REGISTER_CALLBACKS) */
  }

  hpcd->State = HAL_PCD_STATE_BUSY;
    9336:	687b      	ldr	r3, [r7, #4]
    9338:	2203      	movs	r2, #3
    933a:	f883 23bd 	strb.w	r2, [r3, #957]	; 0x3bd

  /* Disable DMA mode for FS instance */
  if ((USBx->CID & (0x1U << 8)) == 0U)
    933e:	68bb      	ldr	r3, [r7, #8]
    9340:	6bdb      	ldr	r3, [r3, #60]	; 0x3c
    9342:	f403 7380 	and.w	r3, r3, #256	; 0x100
    9346:	2b00      	cmp	r3, #0
    9348:	d102      	bne.n	9350 <HAL_PCD_Init+0x4c>
  {
    hpcd->Init.dma_enable = 0U;
    934a:	687b      	ldr	r3, [r7, #4]
    934c:	2200      	movs	r2, #0
    934e:	611a      	str	r2, [r3, #16]
  }

  /* Disable the Interrupts */
  __HAL_PCD_DISABLE(hpcd);
    9350:	687b      	ldr	r3, [r7, #4]
    9352:	681b      	ldr	r3, [r3, #0]
    9354:	4618      	mov	r0, r3
    9356:	f001 f971 	bl	a63c <USB_DisableGlobalInt>

  /*Init the Core (common init.) */
  if (USB_CoreInit(hpcd->Instance, hpcd->Init) != HAL_OK)
    935a:	687b      	ldr	r3, [r7, #4]
    935c:	681b      	ldr	r3, [r3, #0]
    935e:	603b      	str	r3, [r7, #0]
    9360:	687e      	ldr	r6, [r7, #4]
    9362:	466d      	mov	r5, sp
    9364:	f106 0410 	add.w	r4, r6, #16
    9368:	cc0f      	ldmia	r4!, {r0, r1, r2, r3}
    936a:	c50f      	stmia	r5!, {r0, r1, r2, r3}
    936c:	cc0f      	ldmia	r4!, {r0, r1, r2, r3}
    936e:	c50f      	stmia	r5!, {r0, r1, r2, r3}
    9370:	e894 0003 	ldmia.w	r4, {r0, r1}
    9374:	e885 0003 	stmia.w	r5, {r0, r1}
    9378:	1d33      	adds	r3, r6, #4
    937a:	cb0e      	ldmia	r3, {r1, r2, r3}
    937c:	6838      	ldr	r0, [r7, #0]
    937e:	f001 f8eb 	bl	a558 <USB_CoreInit>
    9382:	4603      	mov	r3, r0
    9384:	2b00      	cmp	r3, #0
    9386:	d005      	beq.n	9394 <HAL_PCD_Init+0x90>
  {
    hpcd->State = HAL_PCD_STATE_ERROR;
    9388:	687b      	ldr	r3, [r7, #4]
    938a:	2202      	movs	r2, #2
    938c:	f883 23bd 	strb.w	r2, [r3, #957]	; 0x3bd
    return HAL_ERROR;
    9390:	2301      	movs	r3, #1
    9392:	e0d0      	b.n	9536 <HAL_PCD_Init+0x232>
  }

  /* Force Device Mode*/
  (void)USB_SetCurrentMode(hpcd->Instance, USB_DEVICE_MODE);
    9394:	687b      	ldr	r3, [r7, #4]
    9396:	681b      	ldr	r3, [r3, #0]
    9398:	2100      	movs	r1, #0
    939a:	4618      	mov	r0, r3
    939c:	f001 f95f 	bl	a65e <USB_SetCurrentMode>

  /* Init endpoints structures */
  for (i = 0U; i < hpcd->Init.dev_endpoints; i++)
    93a0:	2300      	movs	r3, #0
    93a2:	73fb      	strb	r3, [r7, #15]
    93a4:	e04a      	b.n	943c <HAL_PCD_Init+0x138>
  {
    /* Init ep structure */
    hpcd->IN_ep[i].is_in = 1U;
    93a6:	7bfa      	ldrb	r2, [r7, #15]
    93a8:	6879      	ldr	r1, [r7, #4]
    93aa:	4613      	mov	r3, r2
    93ac:	00db      	lsls	r3, r3, #3
    93ae:	1a9b      	subs	r3, r3, r2
    93b0:	009b      	lsls	r3, r3, #2
    93b2:	440b      	add	r3, r1
    93b4:	333d      	adds	r3, #61	; 0x3d
    93b6:	2201      	movs	r2, #1
    93b8:	701a      	strb	r2, [r3, #0]
    hpcd->IN_ep[i].num = i;
    93ba:	7bfa      	ldrb	r2, [r7, #15]
    93bc:	6879      	ldr	r1, [r7, #4]
    93be:	4613      	mov	r3, r2
    93c0:	00db      	lsls	r3, r3, #3
    93c2:	1a9b      	subs	r3, r3, r2
    93c4:	009b      	lsls	r3, r3, #2
    93c6:	440b      	add	r3, r1
    93c8:	333c      	adds	r3, #60	; 0x3c
    93ca:	7bfa      	ldrb	r2, [r7, #15]
    93cc:	701a      	strb	r2, [r3, #0]
    hpcd->IN_ep[i].tx_fifo_num = i;
    93ce:	7bfa      	ldrb	r2, [r7, #15]
    93d0:	7bfb      	ldrb	r3, [r7, #15]
    93d2:	b298      	uxth	r0, r3
    93d4:	6879      	ldr	r1, [r7, #4]
    93d6:	4613      	mov	r3, r2
    93d8:	00db      	lsls	r3, r3, #3
    93da:	1a9b      	subs	r3, r3, r2
    93dc:	009b      	lsls	r3, r3, #2
    93de:	440b      	add	r3, r1
    93e0:	3342      	adds	r3, #66	; 0x42
    93e2:	4602      	mov	r2, r0
    93e4:	801a      	strh	r2, [r3, #0]
    /* Control until ep is activated */
    hpcd->IN_ep[i].type = EP_TYPE_CTRL;
    93e6:	7bfa      	ldrb	r2, [r7, #15]
    93e8:	6879      	ldr	r1, [r7, #4]
    93ea:	4613      	mov	r3, r2
    93ec:	00db      	lsls	r3, r3, #3
    93ee:	1a9b      	subs	r3, r3, r2
    93f0:	009b      	lsls	r3, r3, #2
    93f2:	440b      	add	r3, r1
    93f4:	333f      	adds	r3, #63	; 0x3f
    93f6:	2200      	movs	r2, #0
    93f8:	701a      	strb	r2, [r3, #0]
    hpcd->IN_ep[i].maxpacket = 0U;
    93fa:	7bfa      	ldrb	r2, [r7, #15]
    93fc:	6879      	ldr	r1, [r7, #4]
    93fe:	4613      	mov	r3, r2
    9400:	00db      	lsls	r3, r3, #3
    9402:	1a9b      	subs	r3, r3, r2
    9404:	009b      	lsls	r3, r3, #2
    9406:	440b      	add	r3, r1
    9408:	3344      	adds	r3, #68	; 0x44
    940a:	2200      	movs	r2, #0
    940c:	601a      	str	r2, [r3, #0]
    hpcd->IN_ep[i].xfer_buff = 0U;
    940e:	7bfa      	ldrb	r2, [r7, #15]
    9410:	6879      	ldr	r1, [r7, #4]
    9412:	4613      	mov	r3, r2
    9414:	00db      	lsls	r3, r3, #3
    9416:	1a9b      	subs	r3, r3, r2
    9418:	009b      	lsls	r3, r3, #2
    941a:	440b      	add	r3, r1
    941c:	3348      	adds	r3, #72	; 0x48
    941e:	2200      	movs	r2, #0
    9420:	601a      	str	r2, [r3, #0]
    hpcd->IN_ep[i].xfer_len = 0U;
    9422:	7bfa      	ldrb	r2, [r7, #15]
    9424:	6879      	ldr	r1, [r7, #4]
    9426:	4613      	mov	r3, r2
    9428:	00db      	lsls	r3, r3, #3
    942a:	1a9b      	subs	r3, r3, r2
    942c:	009b      	lsls	r3, r3, #2
    942e:	440b      	add	r3, r1
    9430:	3350      	adds	r3, #80	; 0x50
    9432:	2200      	movs	r2, #0
    9434:	601a      	str	r2, [r3, #0]
  for (i = 0U; i < hpcd->Init.dev_endpoints; i++)
    9436:	7bfb      	ldrb	r3, [r7, #15]
    9438:	3301      	adds	r3, #1
    943a:	73fb      	strb	r3, [r7, #15]
    943c:	7bfa      	ldrb	r2, [r7, #15]
    943e:	687b      	ldr	r3, [r7, #4]
    9440:	685b      	ldr	r3, [r3, #4]
    9442:	429a      	cmp	r2, r3
    9444:	d3af      	bcc.n	93a6 <HAL_PCD_Init+0xa2>
  }

  for (i = 0U; i < hpcd->Init.dev_endpoints; i++)
    9446:	2300      	movs	r3, #0
    9448:	73fb      	strb	r3, [r7, #15]
    944a:	e044      	b.n	94d6 <HAL_PCD_Init+0x1d2>
  {
    hpcd->OUT_ep[i].is_in = 0U;
    944c:	7bfa      	ldrb	r2, [r7, #15]
    944e:	6879      	ldr	r1, [r7, #4]
    9450:	4613      	mov	r3, r2
    9452:	00db      	lsls	r3, r3, #3
    9454:	1a9b      	subs	r3, r3, r2
    9456:	009b      	lsls	r3, r3, #2
    9458:	440b      	add	r3, r1
    945a:	f203 13fd 	addw	r3, r3, #509	; 0x1fd
    945e:	2200      	movs	r2, #0
    9460:	701a      	strb	r2, [r3, #0]
    hpcd->OUT_ep[i].num = i;
    9462:	7bfa      	ldrb	r2, [r7, #15]
    9464:	6879      	ldr	r1, [r7, #4]
    9466:	4613      	mov	r3, r2
    9468:	00db      	lsls	r3, r3, #3
    946a:	1a9b      	subs	r3, r3, r2
    946c:	009b      	lsls	r3, r3, #2
    946e:	440b      	add	r3, r1
    9470:	f503 73fe 	add.w	r3, r3, #508	; 0x1fc
    9474:	7bfa      	ldrb	r2, [r7, #15]
    9476:	701a      	strb	r2, [r3, #0]
    /* Control until ep is activated */
    hpcd->OUT_ep[i].type = EP_TYPE_CTRL;
    9478:	7bfa      	ldrb	r2, [r7, #15]
    947a:	6879      	ldr	r1, [r7, #4]
    947c:	4613      	mov	r3, r2
    947e:	00db      	lsls	r3, r3, #3
    9480:	1a9b      	subs	r3, r3, r2
    9482:	009b      	lsls	r3, r3, #2
    9484:	440b      	add	r3, r1
    9486:	f203 13ff 	addw	r3, r3, #511	; 0x1ff
    948a:	2200      	movs	r2, #0
    948c:	701a      	strb	r2, [r3, #0]
    hpcd->OUT_ep[i].maxpacket = 0U;
    948e:	7bfa      	ldrb	r2, [r7, #15]
    9490:	6879      	ldr	r1, [r7, #4]
    9492:	4613      	mov	r3, r2
    9494:	00db      	lsls	r3, r3, #3
    9496:	1a9b      	subs	r3, r3, r2
    9498:	009b      	lsls	r3, r3, #2
    949a:	440b      	add	r3, r1
    949c:	f503 7301 	add.w	r3, r3, #516	; 0x204
    94a0:	2200      	movs	r2, #0
    94a2:	601a      	str	r2, [r3, #0]
    hpcd->OUT_ep[i].xfer_buff = 0U;
    94a4:	7bfa      	ldrb	r2, [r7, #15]
    94a6:	6879      	ldr	r1, [r7, #4]
    94a8:	4613      	mov	r3, r2
    94aa:	00db      	lsls	r3, r3, #3
    94ac:	1a9b      	subs	r3, r3, r2
    94ae:	009b      	lsls	r3, r3, #2
    94b0:	440b      	add	r3, r1
    94b2:	f503 7302 	add.w	r3, r3, #520	; 0x208
    94b6:	2200      	movs	r2, #0
    94b8:	601a      	str	r2, [r3, #0]
    hpcd->OUT_ep[i].xfer_len = 0U;
    94ba:	7bfa      	ldrb	r2, [r7, #15]
    94bc:	6879      	ldr	r1, [r7, #4]
    94be:	4613      	mov	r3, r2
    94c0:	00db      	lsls	r3, r3, #3
    94c2:	1a9b      	subs	r3, r3, r2
    94c4:	009b      	lsls	r3, r3, #2
    94c6:	440b      	add	r3, r1
    94c8:	f503 7304 	add.w	r3, r3, #528	; 0x210
    94cc:	2200      	movs	r2, #0
    94ce:	601a      	str	r2, [r3, #0]
  for (i = 0U; i < hpcd->Init.dev_endpoints; i++)
    94d0:	7bfb      	ldrb	r3, [r7, #15]
    94d2:	3301      	adds	r3, #1
    94d4:	73fb      	strb	r3, [r7, #15]
    94d6:	7bfa      	ldrb	r2, [r7, #15]
    94d8:	687b      	ldr	r3, [r7, #4]
    94da:	685b      	ldr	r3, [r3, #4]
    94dc:	429a      	cmp	r2, r3
    94de:	d3b5      	bcc.n	944c <HAL_PCD_Init+0x148>
  }

  /* Init Device */
  if (USB_DevInit(hpcd->Instance, hpcd->Init) != HAL_OK)
    94e0:	687b      	ldr	r3, [r7, #4]
    94e2:	681b      	ldr	r3, [r3, #0]
    94e4:	603b      	str	r3, [r7, #0]
    94e6:	687e      	ldr	r6, [r7, #4]
    94e8:	466d      	mov	r5, sp
    94ea:	f106 0410 	add.w	r4, r6, #16
    94ee:	cc0f      	ldmia	r4!, {r0, r1, r2, r3}
    94f0:	c50f      	stmia	r5!, {r0, r1, r2, r3}
    94f2:	cc0f      	ldmia	r4!, {r0, r1, r2, r3}
    94f4:	c50f      	stmia	r5!, {r0, r1, r2, r3}
    94f6:	e894 0003 	ldmia.w	r4, {r0, r1}
    94fa:	e885 0003 	stmia.w	r5, {r0, r1}
    94fe:	1d33      	adds	r3, r6, #4
    9500:	cb0e      	ldmia	r3, {r1, r2, r3}
    9502:	6838      	ldr	r0, [r7, #0]
    9504:	f001 f8d6 	bl	a6b4 <USB_DevInit>
    9508:	4603      	mov	r3, r0
    950a:	2b00      	cmp	r3, #0
    950c:	d005      	beq.n	951a <HAL_PCD_Init+0x216>
  {
    hpcd->State = HAL_PCD_STATE_ERROR;
    950e:	687b      	ldr	r3, [r7, #4]
    9510:	2202      	movs	r2, #2
    9512:	f883 23bd 	strb.w	r2, [r3, #957]	; 0x3bd
    return HAL_ERROR;
    9516:	2301      	movs	r3, #1
    9518:	e00d      	b.n	9536 <HAL_PCD_Init+0x232>
  }

  hpcd->USB_Address = 0U;
    951a:	687b      	ldr	r3, [r7, #4]
    951c:	2200      	movs	r2, #0
    951e:	f883 2038 	strb.w	r2, [r3, #56]	; 0x38
  hpcd->State = HAL_PCD_STATE_READY;
    9522:	687b      	ldr	r3, [r7, #4]
    9524:	2201      	movs	r2, #1
    9526:	f883 23bd 	strb.w	r2, [r3, #957]	; 0x3bd
  if (hpcd->Init.lpm_enable == 1U)
  {
    (void)HAL_PCDEx_ActivateLPM(hpcd);
  }
  #endif /* defined(STM32F446xx) || defined(STM32F469xx) || defined(STM32F479xx) || defined(STM32F412Zx) || defined(STM32F412Vx) || defined(STM32F412Rx) || defined(STM32F412Cx) || defined(STM32F413xx) || defined(STM32F423xx) */
  (void)USB_DevDisconnect(hpcd->Instance);
    952a:	687b      	ldr	r3, [r7, #4]
    952c:	681b      	ldr	r3, [r3, #0]
    952e:	4618      	mov	r0, r3
    9530:	f001 fff0 	bl	b514 <USB_DevDisconnect>

  return HAL_OK;
    9534:	2300      	movs	r3, #0
}
    9536:	4618      	mov	r0, r3
    9538:	3714      	adds	r7, #20
    953a:	46bd      	mov	sp, r7
    953c:	bdf0      	pop	{r4, r5, r6, r7, pc}

0000953e <HAL_PCD_Start>:
  * @brief  Start the USB device
  * @param  hpcd PCD handle
  * @retval HAL status
  */
HAL_StatusTypeDef HAL_PCD_Start(PCD_HandleTypeDef *hpcd)
{
    953e:	b580      	push	{r7, lr}
    9540:	b084      	sub	sp, #16
    9542:	af00      	add	r7, sp, #0
    9544:	6078      	str	r0, [r7, #4]
#if defined (USB_OTG_FS) || defined (USB_OTG_HS)
  USB_OTG_GlobalTypeDef *USBx = hpcd->Instance;
    9546:	687b      	ldr	r3, [r7, #4]
    9548:	681b      	ldr	r3, [r3, #0]
    954a:	60fb      	str	r3, [r7, #12]
#endif /* defined (USB_OTG_FS) || defined (USB_OTG_HS) */

  __HAL_LOCK(hpcd);
    954c:	687b      	ldr	r3, [r7, #4]
    954e:	f893 33bc 	ldrb.w	r3, [r3, #956]	; 0x3bc
    9552:	2b01      	cmp	r3, #1
    9554:	d101      	bne.n	955a <HAL_PCD_Start+0x1c>
    9556:	2302      	movs	r3, #2
    9558:	e020      	b.n	959c <HAL_PCD_Start+0x5e>
    955a:	687b      	ldr	r3, [r7, #4]
    955c:	2201      	movs	r2, #1
    955e:	f883 23bc 	strb.w	r2, [r3, #956]	; 0x3bc
#if defined (USB_OTG_FS) || defined (USB_OTG_HS)
  if ((hpcd->Init.battery_charging_enable == 1U) &&
    9562:	687b      	ldr	r3, [r7, #4]
    9564:	6a9b      	ldr	r3, [r3, #40]	; 0x28
    9566:	2b01      	cmp	r3, #1
    9568:	d109      	bne.n	957e <HAL_PCD_Start+0x40>
      (hpcd->Init.phy_itface != USB_OTG_ULPI_PHY))
    956a:	687b      	ldr	r3, [r7, #4]
    956c:	699b      	ldr	r3, [r3, #24]
  if ((hpcd->Init.battery_charging_enable == 1U) &&
    956e:	2b01      	cmp	r3, #1
    9570:	d005      	beq.n	957e <HAL_PCD_Start+0x40>
  {
    /* Enable USB Transceiver */
    USBx->GCCFG |= USB_OTG_GCCFG_PWRDWN;
    9572:	68fb      	ldr	r3, [r7, #12]
    9574:	6b9b      	ldr	r3, [r3, #56]	; 0x38
    9576:	f443 3280 	orr.w	r2, r3, #65536	; 0x10000
    957a:	68fb      	ldr	r3, [r7, #12]
    957c:	639a      	str	r2, [r3, #56]	; 0x38
  }
#endif /* defined (USB_OTG_FS) || defined (USB_OTG_HS) */
  (void)USB_DevConnect(hpcd->Instance);
    957e:	687b      	ldr	r3, [r7, #4]
    9580:	681b      	ldr	r3, [r3, #0]
    9582:	4618      	mov	r0, r3
    9584:	f001 ffae 	bl	b4e4 <USB_DevConnect>
  __HAL_PCD_ENABLE(hpcd);
    9588:	687b      	ldr	r3, [r7, #4]
    958a:	681b      	ldr	r3, [r3, #0]
    958c:	4618      	mov	r0, r3
    958e:	f001 f844 	bl	a61a <USB_EnableGlobalInt>
  __HAL_UNLOCK(hpcd);
    9592:	687b      	ldr	r3, [r7, #4]
    9594:	2200      	movs	r2, #0
    9596:	f883 23bc 	strb.w	r2, [r3, #956]	; 0x3bc
  return HAL_OK;
    959a:	2300      	movs	r3, #0
}
    959c:	4618      	mov	r0, r3
    959e:	3710      	adds	r7, #16
    95a0:	46bd      	mov	sp, r7
    95a2:	bd80      	pop	{r7, pc}

000095a4 <HAL_PCD_EP_Open>:
  * @param  ep_mps endpoint max packet size
  * @param  ep_type endpoint type
  * @retval HAL status
  */
HAL_StatusTypeDef HAL_PCD_EP_Open(PCD_HandleTypeDef *hpcd, uint8_t ep_addr, uint16_t ep_mps, uint8_t ep_type)
{
    95a4:	b580      	push	{r7, lr}
    95a6:	b084      	sub	sp, #16
    95a8:	af00      	add	r7, sp, #0
    95aa:	6078      	str	r0, [r7, #4]
    95ac:	4608      	mov	r0, r1
    95ae:	4611      	mov	r1, r2
    95b0:	461a      	mov	r2, r3
    95b2:	4603      	mov	r3, r0
    95b4:	70fb      	strb	r3, [r7, #3]
    95b6:	460b      	mov	r3, r1
    95b8:	803b      	strh	r3, [r7, #0]
    95ba:	4613      	mov	r3, r2
    95bc:	70bb      	strb	r3, [r7, #2]
  HAL_StatusTypeDef  ret = HAL_OK;
    95be:	2300      	movs	r3, #0
    95c0:	72fb      	strb	r3, [r7, #11]
  PCD_EPTypeDef *ep;

  if ((ep_addr & 0x80U) == 0x80U)
    95c2:	f997 3003 	ldrsb.w	r3, [r7, #3]
    95c6:	2b00      	cmp	r3, #0
    95c8:	da0f      	bge.n	95ea <HAL_PCD_EP_Open+0x46>
  {
    ep = &hpcd->IN_ep[ep_addr & EP_ADDR_MSK];
    95ca:	78fb      	ldrb	r3, [r7, #3]
    95cc:	f003 020f 	and.w	r2, r3, #15
    95d0:	4613      	mov	r3, r2
    95d2:	00db      	lsls	r3, r3, #3
    95d4:	1a9b      	subs	r3, r3, r2
    95d6:	009b      	lsls	r3, r3, #2
    95d8:	3338      	adds	r3, #56	; 0x38
    95da:	687a      	ldr	r2, [r7, #4]
    95dc:	4413      	add	r3, r2
    95de:	3304      	adds	r3, #4
    95e0:	60fb      	str	r3, [r7, #12]
    ep->is_in = 1U;
    95e2:	68fb      	ldr	r3, [r7, #12]
    95e4:	2201      	movs	r2, #1
    95e6:	705a      	strb	r2, [r3, #1]
    95e8:	e00f      	b.n	960a <HAL_PCD_EP_Open+0x66>
  }
  else
  {
    ep = &hpcd->OUT_ep[ep_addr & EP_ADDR_MSK];
    95ea:	78fb      	ldrb	r3, [r7, #3]
    95ec:	f003 020f 	and.w	r2, r3, #15
    95f0:	4613      	mov	r3, r2
    95f2:	00db      	lsls	r3, r3, #3
    95f4:	1a9b      	subs	r3, r3, r2
    95f6:	009b      	lsls	r3, r3, #2
    95f8:	f503 73fc 	add.w	r3, r3, #504	; 0x1f8
    95fc:	687a      	ldr	r2, [r7, #4]
    95fe:	4413      	add	r3, r2
    9600:	3304      	adds	r3, #4
    9602:	60fb      	str	r3, [r7, #12]
    ep->is_in = 0U;
    9604:	68fb      	ldr	r3, [r7, #12]
    9606:	2200      	movs	r2, #0
    9608:	705a      	strb	r2, [r3, #1]
  }

  ep->num = ep_addr & EP_ADDR_MSK;
    960a:	78fb      	ldrb	r3, [r7, #3]
    960c:	f003 030f 	and.w	r3, r3, #15
    9610:	b2da      	uxtb	r2, r3
    9612:	68fb      	ldr	r3, [r7, #12]
    9614:	701a      	strb	r2, [r3, #0]
  ep->maxpacket = ep_mps;
    9616:	883a      	ldrh	r2, [r7, #0]
    9618:	68fb      	ldr	r3, [r7, #12]
    961a:	609a      	str	r2, [r3, #8]
  ep->type = ep_type;
    961c:	68fb      	ldr	r3, [r7, #12]
    961e:	78ba      	ldrb	r2, [r7, #2]
    9620:	70da      	strb	r2, [r3, #3]

  if (ep->is_in != 0U)
    9622:	68fb      	ldr	r3, [r7, #12]
    9624:	785b      	ldrb	r3, [r3, #1]
    9626:	2b00      	cmp	r3, #0
    9628:	d004      	beq.n	9634 <HAL_PCD_EP_Open+0x90>
  {
    /* Assign a Tx FIFO */
    ep->tx_fifo_num = ep->num;
    962a:	68fb      	ldr	r3, [r7, #12]
    962c:	781b      	ldrb	r3, [r3, #0]
    962e:	b29a      	uxth	r2, r3
    9630:	68fb      	ldr	r3, [r7, #12]
    9632:	80da      	strh	r2, [r3, #6]
  }
  /* Set initial data PID. */
  if (ep_type == EP_TYPE_BULK)
    9634:	78bb      	ldrb	r3, [r7, #2]
    9636:	2b02      	cmp	r3, #2
    9638:	d102      	bne.n	9640 <HAL_PCD_EP_Open+0x9c>
  {
    ep->data_pid_start = 0U;
    963a:	68fb      	ldr	r3, [r7, #12]
    963c:	2200      	movs	r2, #0
    963e:	711a      	strb	r2, [r3, #4]
  }

  __HAL_LOCK(hpcd);
    9640:	687b      	ldr	r3, [r7, #4]
    9642:	f893 33bc 	ldrb.w	r3, [r3, #956]	; 0x3bc
    9646:	2b01      	cmp	r3, #1
    9648:	d101      	bne.n	964e <HAL_PCD_EP_Open+0xaa>
    964a:	2302      	movs	r3, #2
    964c:	e00e      	b.n	966c <HAL_PCD_EP_Open+0xc8>
    964e:	687b      	ldr	r3, [r7, #4]
    9650:	2201      	movs	r2, #1
    9652:	f883 23bc 	strb.w	r2, [r3, #956]	; 0x3bc
  (void)USB_ActivateEndpoint(hpcd->Instance, ep);
    9656:	687b      	ldr	r3, [r7, #4]
    9658:	681b      	ldr	r3, [r3, #0]
    965a:	68f9      	ldr	r1, [r7, #12]
    965c:	4618      	mov	r0, r3
    965e:	f001 f9fc 	bl	aa5a <USB_ActivateEndpoint>
  __HAL_UNLOCK(hpcd);
    9662:	687b      	ldr	r3, [r7, #4]
    9664:	2200      	movs	r2, #0
    9666:	f883 23bc 	strb.w	r2, [r3, #956]	; 0x3bc

  return ret;
    966a:	7afb      	ldrb	r3, [r7, #11]
}
    966c:	4618      	mov	r0, r3
    966e:	3710      	adds	r7, #16
    9670:	46bd      	mov	sp, r7
    9672:	bd80      	pop	{r7, pc}

00009674 <HAL_PCD_EP_Close>:
  * @param  hpcd PCD handle
  * @param  ep_addr endpoint address
  * @retval HAL status
  */
HAL_StatusTypeDef HAL_PCD_EP_Close(PCD_HandleTypeDef *hpcd, uint8_t ep_addr)
{
    9674:	b580      	push	{r7, lr}
    9676:	b084      	sub	sp, #16
    9678:	af00      	add	r7, sp, #0
    967a:	6078      	str	r0, [r7, #4]
    967c:	460b      	mov	r3, r1
    967e:	70fb      	strb	r3, [r7, #3]
  PCD_EPTypeDef *ep;

  if ((ep_addr & 0x80U) == 0x80U)
    9680:	f997 3003 	ldrsb.w	r3, [r7, #3]
    9684:	2b00      	cmp	r3, #0
    9686:	da0f      	bge.n	96a8 <HAL_PCD_EP_Close+0x34>
  {
    ep = &hpcd->IN_ep[ep_addr & EP_ADDR_MSK];
    9688:	78fb      	ldrb	r3, [r7, #3]
    968a:	f003 020f 	and.w	r2, r3, #15
    968e:	4613      	mov	r3, r2
    9690:	00db      	lsls	r3, r3, #3
    9692:	1a9b      	subs	r3, r3, r2
    9694:	009b      	lsls	r3, r3, #2
    9696:	3338      	adds	r3, #56	; 0x38
    9698:	687a      	ldr	r2, [r7, #4]
    969a:	4413      	add	r3, r2
    969c:	3304      	adds	r3, #4
    969e:	60fb      	str	r3, [r7, #12]
    ep->is_in = 1U;
    96a0:	68fb      	ldr	r3, [r7, #12]
    96a2:	2201      	movs	r2, #1
    96a4:	705a      	strb	r2, [r3, #1]
    96a6:	e00f      	b.n	96c8 <HAL_PCD_EP_Close+0x54>
  }
  else
  {
    ep = &hpcd->OUT_ep[ep_addr & EP_ADDR_MSK];
    96a8:	78fb      	ldrb	r3, [r7, #3]
    96aa:	f003 020f 	and.w	r2, r3, #15
    96ae:	4613      	mov	r3, r2
    96b0:	00db      	lsls	r3, r3, #3
    96b2:	1a9b      	subs	r3, r3, r2
    96b4:	009b      	lsls	r3, r3, #2
    96b6:	f503 73fc 	add.w	r3, r3, #504	; 0x1f8
    96ba:	687a      	ldr	r2, [r7, #4]
    96bc:	4413      	add	r3, r2
    96be:	3304      	adds	r3, #4
    96c0:	60fb      	str	r3, [r7, #12]
    ep->is_in = 0U;
    96c2:	68fb      	ldr	r3, [r7, #12]
    96c4:	2200      	movs	r2, #0
    96c6:	705a      	strb	r2, [r3, #1]
  }
  ep->num   = ep_addr & EP_ADDR_MSK;
    96c8:	78fb      	ldrb	r3, [r7, #3]
    96ca:	f003 030f 	and.w	r3, r3, #15
    96ce:	b2da      	uxtb	r2, r3
    96d0:	68fb      	ldr	r3, [r7, #12]
    96d2:	701a      	strb	r2, [r3, #0]

  __HAL_LOCK(hpcd);
    96d4:	687b      	ldr	r3, [r7, #4]
    96d6:	f893 33bc 	ldrb.w	r3, [r3, #956]	; 0x3bc
    96da:	2b01      	cmp	r3, #1
    96dc:	d101      	bne.n	96e2 <HAL_PCD_EP_Close+0x6e>
    96de:	2302      	movs	r3, #2
    96e0:	e00e      	b.n	9700 <HAL_PCD_EP_Close+0x8c>
    96e2:	687b      	ldr	r3, [r7, #4]
    96e4:	2201      	movs	r2, #1
    96e6:	f883 23bc 	strb.w	r2, [r3, #956]	; 0x3bc
  (void)USB_DeactivateEndpoint(hpcd->Instance, ep);
    96ea:	687b      	ldr	r3, [r7, #4]
    96ec:	681b      	ldr	r3, [r3, #0]
    96ee:	68f9      	ldr	r1, [r7, #12]
    96f0:	4618      	mov	r0, r3
    96f2:	f001 fa39 	bl	ab68 <USB_DeactivateEndpoint>
  __HAL_UNLOCK(hpcd);
    96f6:	687b      	ldr	r3, [r7, #4]
    96f8:	2200      	movs	r2, #0
    96fa:	f883 23bc 	strb.w	r2, [r3, #956]	; 0x3bc
  return HAL_OK;
    96fe:	2300      	movs	r3, #0
}
    9700:	4618      	mov	r0, r3
    9702:	3710      	adds	r7, #16
    9704:	46bd      	mov	sp, r7
    9706:	bd80      	pop	{r7, pc}

00009708 <HAL_PCD_EP_Receive>:
  * @param  pBuf pointer to the reception buffer
  * @param  len amount of data to be received
  * @retval HAL status
  */
HAL_StatusTypeDef HAL_PCD_EP_Receive(PCD_HandleTypeDef *hpcd, uint8_t ep_addr, uint8_t *pBuf, uint32_t len)
{
    9708:	b580      	push	{r7, lr}
    970a:	b086      	sub	sp, #24
    970c:	af00      	add	r7, sp, #0
    970e:	60f8      	str	r0, [r7, #12]
    9710:	607a      	str	r2, [r7, #4]
    9712:	603b      	str	r3, [r7, #0]
    9714:	460b      	mov	r3, r1
    9716:	72fb      	strb	r3, [r7, #11]
  PCD_EPTypeDef *ep;

  ep = &hpcd->OUT_ep[ep_addr & EP_ADDR_MSK];
    9718:	7afb      	ldrb	r3, [r7, #11]
    971a:	f003 020f 	and.w	r2, r3, #15
    971e:	4613      	mov	r3, r2
    9720:	00db      	lsls	r3, r3, #3
    9722:	1a9b      	subs	r3, r3, r2
    9724:	009b      	lsls	r3, r3, #2
    9726:	f503 73fc 	add.w	r3, r3, #504	; 0x1f8
    972a:	68fa      	ldr	r2, [r7, #12]
    972c:	4413      	add	r3, r2
    972e:	3304      	adds	r3, #4
    9730:	617b      	str	r3, [r7, #20]

  /*setup and start the Xfer */
  ep->xfer_buff = pBuf;
    9732:	697b      	ldr	r3, [r7, #20]
    9734:	687a      	ldr	r2, [r7, #4]
    9736:	60da      	str	r2, [r3, #12]
  ep->xfer_len = len;
    9738:	697b      	ldr	r3, [r7, #20]
    973a:	683a      	ldr	r2, [r7, #0]
    973c:	615a      	str	r2, [r3, #20]
  ep->xfer_count = 0U;
    973e:	697b      	ldr	r3, [r7, #20]
    9740:	2200      	movs	r2, #0
    9742:	619a      	str	r2, [r3, #24]
  ep->is_in = 0U;
    9744:	697b      	ldr	r3, [r7, #20]
    9746:	2200      	movs	r2, #0
    9748:	705a      	strb	r2, [r3, #1]
  ep->num = ep_addr & EP_ADDR_MSK;
    974a:	7afb      	ldrb	r3, [r7, #11]
    974c:	f003 030f 	and.w	r3, r3, #15
    9750:	b2da      	uxtb	r2, r3
    9752:	697b      	ldr	r3, [r7, #20]
    9754:	701a      	strb	r2, [r3, #0]

  if (hpcd->Init.dma_enable == 1U)
    9756:	68fb      	ldr	r3, [r7, #12]
    9758:	691b      	ldr	r3, [r3, #16]
    975a:	2b01      	cmp	r3, #1
    975c:	d102      	bne.n	9764 <HAL_PCD_EP_Receive+0x5c>
  {
    ep->dma_addr = (uint32_t)pBuf;
    975e:	687a      	ldr	r2, [r7, #4]
    9760:	697b      	ldr	r3, [r7, #20]
    9762:	611a      	str	r2, [r3, #16]
  }

  if ((ep_addr & EP_ADDR_MSK) == 0U)
    9764:	7afb      	ldrb	r3, [r7, #11]
    9766:	f003 030f 	and.w	r3, r3, #15
    976a:	2b00      	cmp	r3, #0
    976c:	d109      	bne.n	9782 <HAL_PCD_EP_Receive+0x7a>
  {
    (void)USB_EP0StartXfer(hpcd->Instance, ep, (uint8_t)hpcd->Init.dma_enable);
    976e:	68fb      	ldr	r3, [r7, #12]
    9770:	6818      	ldr	r0, [r3, #0]
    9772:	68fb      	ldr	r3, [r7, #12]
    9774:	691b      	ldr	r3, [r3, #16]
    9776:	b2db      	uxtb	r3, r3
    9778:	461a      	mov	r2, r3
    977a:	6979      	ldr	r1, [r7, #20]
    977c:	f001 fcbc 	bl	b0f8 <USB_EP0StartXfer>
    9780:	e008      	b.n	9794 <HAL_PCD_EP_Receive+0x8c>
  }
  else
  {
    (void)USB_EPStartXfer(hpcd->Instance, ep, (uint8_t)hpcd->Init.dma_enable);
    9782:	68fb      	ldr	r3, [r7, #12]
    9784:	6818      	ldr	r0, [r3, #0]
    9786:	68fb      	ldr	r3, [r7, #12]
    9788:	691b      	ldr	r3, [r3, #16]
    978a:	b2db      	uxtb	r3, r3
    978c:	461a      	mov	r2, r3
    978e:	6979      	ldr	r1, [r7, #20]
    9790:	f001 fa6e 	bl	ac70 <USB_EPStartXfer>
  }

  return HAL_OK;
    9794:	2300      	movs	r3, #0
}
    9796:	4618      	mov	r0, r3
    9798:	3718      	adds	r7, #24
    979a:	46bd      	mov	sp, r7
    979c:	bd80      	pop	{r7, pc}

0000979e <HAL_PCD_EP_GetRxCount>:
  * @param  hpcd PCD handle
  * @param  ep_addr endpoint address
  * @retval Data Size
  */
uint32_t HAL_PCD_EP_GetRxCount(PCD_HandleTypeDef *hpcd, uint8_t ep_addr)
{
    979e:	b480      	push	{r7}
    97a0:	b083      	sub	sp, #12
    97a2:	af00      	add	r7, sp, #0
    97a4:	6078      	str	r0, [r7, #4]
    97a6:	460b      	mov	r3, r1
    97a8:	70fb      	strb	r3, [r7, #3]
  return hpcd->OUT_ep[ep_addr & EP_ADDR_MSK].xfer_count;
    97aa:	78fb      	ldrb	r3, [r7, #3]
    97ac:	f003 020f 	and.w	r2, r3, #15
    97b0:	6879      	ldr	r1, [r7, #4]
    97b2:	4613      	mov	r3, r2
    97b4:	00db      	lsls	r3, r3, #3
    97b6:	1a9b      	subs	r3, r3, r2
    97b8:	009b      	lsls	r3, r3, #2
    97ba:	440b      	add	r3, r1
    97bc:	f503 7305 	add.w	r3, r3, #532	; 0x214
    97c0:	681b      	ldr	r3, [r3, #0]
}
    97c2:	4618      	mov	r0, r3
    97c4:	370c      	adds	r7, #12
    97c6:	46bd      	mov	sp, r7
    97c8:	f85d 7b04 	ldr.w	r7, [sp], #4
    97cc:	4770      	bx	lr

000097ce <HAL_PCD_EP_Transmit>:
  * @param  pBuf pointer to the transmission buffer
  * @param  len amount of data to be sent
  * @retval HAL status
  */
HAL_StatusTypeDef HAL_PCD_EP_Transmit(PCD_HandleTypeDef *hpcd, uint8_t ep_addr, uint8_t *pBuf, uint32_t len)
{
    97ce:	b580      	push	{r7, lr}
    97d0:	b086      	sub	sp, #24
    97d2:	af00      	add	r7, sp, #0
    97d4:	60f8      	str	r0, [r7, #12]
    97d6:	607a      	str	r2, [r7, #4]
    97d8:	603b      	str	r3, [r7, #0]
    97da:	460b      	mov	r3, r1
    97dc:	72fb      	strb	r3, [r7, #11]
  PCD_EPTypeDef *ep;

  ep = &hpcd->IN_ep[ep_addr & EP_ADDR_MSK];
    97de:	7afb      	ldrb	r3, [r7, #11]
    97e0:	f003 020f 	and.w	r2, r3, #15
    97e4:	4613      	mov	r3, r2
    97e6:	00db      	lsls	r3, r3, #3
    97e8:	1a9b      	subs	r3, r3, r2
    97ea:	009b      	lsls	r3, r3, #2
    97ec:	3338      	adds	r3, #56	; 0x38
    97ee:	68fa      	ldr	r2, [r7, #12]
    97f0:	4413      	add	r3, r2
    97f2:	3304      	adds	r3, #4
    97f4:	617b      	str	r3, [r7, #20]

  /*setup and start the Xfer */
  ep->xfer_buff = pBuf;
    97f6:	697b      	ldr	r3, [r7, #20]
    97f8:	687a      	ldr	r2, [r7, #4]
    97fa:	60da      	str	r2, [r3, #12]
  ep->xfer_len = len;
    97fc:	697b      	ldr	r3, [r7, #20]
    97fe:	683a      	ldr	r2, [r7, #0]
    9800:	615a      	str	r2, [r3, #20]
  ep->xfer_count = 0U;
    9802:	697b      	ldr	r3, [r7, #20]
    9804:	2200      	movs	r2, #0
    9806:	619a      	str	r2, [r3, #24]
  ep->is_in = 1U;
    9808:	697b      	ldr	r3, [r7, #20]
    980a:	2201      	movs	r2, #1
    980c:	705a      	strb	r2, [r3, #1]
  ep->num = ep_addr & EP_ADDR_MSK;
    980e:	7afb      	ldrb	r3, [r7, #11]
    9810:	f003 030f 	and.w	r3, r3, #15
    9814:	b2da      	uxtb	r2, r3
    9816:	697b      	ldr	r3, [r7, #20]
    9818:	701a      	strb	r2, [r3, #0]

  if (hpcd->Init.dma_enable == 1U)
    981a:	68fb      	ldr	r3, [r7, #12]
    981c:	691b      	ldr	r3, [r3, #16]
    981e:	2b01      	cmp	r3, #1
    9820:	d102      	bne.n	9828 <HAL_PCD_EP_Transmit+0x5a>
  {
    ep->dma_addr = (uint32_t)pBuf;
    9822:	687a      	ldr	r2, [r7, #4]
    9824:	697b      	ldr	r3, [r7, #20]
    9826:	611a      	str	r2, [r3, #16]
  }

  if ((ep_addr & EP_ADDR_MSK) == 0U)
    9828:	7afb      	ldrb	r3, [r7, #11]
    982a:	f003 030f 	and.w	r3, r3, #15
    982e:	2b00      	cmp	r3, #0
    9830:	d109      	bne.n	9846 <HAL_PCD_EP_Transmit+0x78>
  {
    (void)USB_EP0StartXfer(hpcd->Instance, ep, (uint8_t)hpcd->Init.dma_enable);
    9832:	68fb      	ldr	r3, [r7, #12]
    9834:	6818      	ldr	r0, [r3, #0]
    9836:	68fb      	ldr	r3, [r7, #12]
    9838:	691b      	ldr	r3, [r3, #16]
    983a:	b2db      	uxtb	r3, r3
    983c:	461a      	mov	r2, r3
    983e:	6979      	ldr	r1, [r7, #20]
    9840:	f001 fc5a 	bl	b0f8 <USB_EP0StartXfer>
    9844:	e008      	b.n	9858 <HAL_PCD_EP_Transmit+0x8a>
  }
  else
  {
    (void)USB_EPStartXfer(hpcd->Instance, ep, (uint8_t)hpcd->Init.dma_enable);
    9846:	68fb      	ldr	r3, [r7, #12]
    9848:	6818      	ldr	r0, [r3, #0]
    984a:	68fb      	ldr	r3, [r7, #12]
    984c:	691b      	ldr	r3, [r3, #16]
    984e:	b2db      	uxtb	r3, r3
    9850:	461a      	mov	r2, r3
    9852:	6979      	ldr	r1, [r7, #20]
    9854:	f001 fa0c 	bl	ac70 <USB_EPStartXfer>
  }

  return HAL_OK;
    9858:	2300      	movs	r3, #0
}
    985a:	4618      	mov	r0, r3
    985c:	3718      	adds	r7, #24
    985e:	46bd      	mov	sp, r7
    9860:	bd80      	pop	{r7, pc}

00009862 <HAL_PCD_EP_SetStall>:
  * @param  hpcd PCD handle
  * @param  ep_addr endpoint address
  * @retval HAL status
  */
HAL_StatusTypeDef HAL_PCD_EP_SetStall(PCD_HandleTypeDef *hpcd, uint8_t ep_addr)
{
    9862:	b580      	push	{r7, lr}
    9864:	b084      	sub	sp, #16
    9866:	af00      	add	r7, sp, #0
    9868:	6078      	str	r0, [r7, #4]
    986a:	460b      	mov	r3, r1
    986c:	70fb      	strb	r3, [r7, #3]
  PCD_EPTypeDef *ep;

  if (((uint32_t)ep_addr & EP_ADDR_MSK) > hpcd->Init.dev_endpoints)
    986e:	78fb      	ldrb	r3, [r7, #3]
    9870:	f003 020f 	and.w	r2, r3, #15
    9874:	687b      	ldr	r3, [r7, #4]
    9876:	685b      	ldr	r3, [r3, #4]
    9878:	429a      	cmp	r2, r3
    987a:	d901      	bls.n	9880 <HAL_PCD_EP_SetStall+0x1e>
  {
    return HAL_ERROR;
    987c:	2301      	movs	r3, #1
    987e:	e050      	b.n	9922 <HAL_PCD_EP_SetStall+0xc0>
  }

  if ((0x80U & ep_addr) == 0x80U)
    9880:	f997 3003 	ldrsb.w	r3, [r7, #3]
    9884:	2b00      	cmp	r3, #0
    9886:	da0f      	bge.n	98a8 <HAL_PCD_EP_SetStall+0x46>
  {
    ep = &hpcd->IN_ep[ep_addr & EP_ADDR_MSK];
    9888:	78fb      	ldrb	r3, [r7, #3]
    988a:	f003 020f 	and.w	r2, r3, #15
    988e:	4613      	mov	r3, r2
    9890:	00db      	lsls	r3, r3, #3
    9892:	1a9b      	subs	r3, r3, r2
    9894:	009b      	lsls	r3, r3, #2
    9896:	3338      	adds	r3, #56	; 0x38
    9898:	687a      	ldr	r2, [r7, #4]
    989a:	4413      	add	r3, r2
    989c:	3304      	adds	r3, #4
    989e:	60fb      	str	r3, [r7, #12]
    ep->is_in = 1U;
    98a0:	68fb      	ldr	r3, [r7, #12]
    98a2:	2201      	movs	r2, #1
    98a4:	705a      	strb	r2, [r3, #1]
    98a6:	e00d      	b.n	98c4 <HAL_PCD_EP_SetStall+0x62>
  }
  else
  {
    ep = &hpcd->OUT_ep[ep_addr];
    98a8:	78fa      	ldrb	r2, [r7, #3]
    98aa:	4613      	mov	r3, r2
    98ac:	00db      	lsls	r3, r3, #3
    98ae:	1a9b      	subs	r3, r3, r2
    98b0:	009b      	lsls	r3, r3, #2
    98b2:	f503 73fc 	add.w	r3, r3, #504	; 0x1f8
    98b6:	687a      	ldr	r2, [r7, #4]
    98b8:	4413      	add	r3, r2
    98ba:	3304      	adds	r3, #4
    98bc:	60fb      	str	r3, [r7, #12]
    ep->is_in = 0U;
    98be:	68fb      	ldr	r3, [r7, #12]
    98c0:	2200      	movs	r2, #0
    98c2:	705a      	strb	r2, [r3, #1]
  }

  ep->is_stall = 1U;
    98c4:	68fb      	ldr	r3, [r7, #12]
    98c6:	2201      	movs	r2, #1
    98c8:	709a      	strb	r2, [r3, #2]
  ep->num = ep_addr & EP_ADDR_MSK;
    98ca:	78fb      	ldrb	r3, [r7, #3]
    98cc:	f003 030f 	and.w	r3, r3, #15
    98d0:	b2da      	uxtb	r2, r3
    98d2:	68fb      	ldr	r3, [r7, #12]
    98d4:	701a      	strb	r2, [r3, #0]

  __HAL_LOCK(hpcd);
    98d6:	687b      	ldr	r3, [r7, #4]
    98d8:	f893 33bc 	ldrb.w	r3, [r3, #956]	; 0x3bc
    98dc:	2b01      	cmp	r3, #1
    98de:	d101      	bne.n	98e4 <HAL_PCD_EP_SetStall+0x82>
    98e0:	2302      	movs	r3, #2
    98e2:	e01e      	b.n	9922 <HAL_PCD_EP_SetStall+0xc0>
    98e4:	687b      	ldr	r3, [r7, #4]
    98e6:	2201      	movs	r2, #1
    98e8:	f883 23bc 	strb.w	r2, [r3, #956]	; 0x3bc

  (void)USB_EPSetStall(hpcd->Instance, ep);
    98ec:	687b      	ldr	r3, [r7, #4]
    98ee:	681b      	ldr	r3, [r3, #0]
    98f0:	68f9      	ldr	r1, [r7, #12]
    98f2:	4618      	mov	r0, r3
    98f4:	f001 fd88 	bl	b408 <USB_EPSetStall>
  if ((ep_addr & EP_ADDR_MSK) == 0U)
    98f8:	78fb      	ldrb	r3, [r7, #3]
    98fa:	f003 030f 	and.w	r3, r3, #15
    98fe:	2b00      	cmp	r3, #0
    9900:	d10a      	bne.n	9918 <HAL_PCD_EP_SetStall+0xb6>
  {
    (void)USB_EP0_OutStart(hpcd->Instance, (uint8_t)hpcd->Init.dma_enable, (uint8_t *)hpcd->Setup);
    9902:	687b      	ldr	r3, [r7, #4]
    9904:	6818      	ldr	r0, [r3, #0]
    9906:	687b      	ldr	r3, [r7, #4]
    9908:	691b      	ldr	r3, [r3, #16]
    990a:	b2d9      	uxtb	r1, r3
    990c:	687b      	ldr	r3, [r7, #4]
    990e:	f503 7371 	add.w	r3, r3, #964	; 0x3c4
    9912:	461a      	mov	r2, r3
    9914:	f001 fe16 	bl	b544 <USB_EP0_OutStart>
  }
  __HAL_UNLOCK(hpcd);
    9918:	687b      	ldr	r3, [r7, #4]
    991a:	2200      	movs	r2, #0
    991c:	f883 23bc 	strb.w	r2, [r3, #956]	; 0x3bc

  return HAL_OK;
    9920:	2300      	movs	r3, #0
}
    9922:	4618      	mov	r0, r3
    9924:	3710      	adds	r7, #16
    9926:	46bd      	mov	sp, r7
    9928:	bd80      	pop	{r7, pc}

0000992a <HAL_PCDEx_SetTxFiFo>:
  * @param  fifo The number of Tx fifo
  * @param  size Fifo size
  * @retval HAL status
  */
HAL_StatusTypeDef HAL_PCDEx_SetTxFiFo(PCD_HandleTypeDef *hpcd, uint8_t fifo, uint16_t size)
{
    992a:	b480      	push	{r7}
    992c:	b085      	sub	sp, #20
    992e:	af00      	add	r7, sp, #0
    9930:	6078      	str	r0, [r7, #4]
    9932:	460b      	mov	r3, r1
    9934:	70fb      	strb	r3, [r7, #3]
    9936:	4613      	mov	r3, r2
    9938:	803b      	strh	r3, [r7, #0]
         --> Txn should be configured with the minimum space of 16 words
     The FIFO is used optimally when used TxFIFOs are allocated in the top
         of the FIFO.Ex: use EP1 and EP2 as IN instead of EP1 and EP3 as IN ones.
     When DMA is used 3n * FIFO locations should be reserved for internal DMA registers */

  Tx_Offset = hpcd->Instance->GRXFSIZ;
    993a:	687b      	ldr	r3, [r7, #4]
    993c:	681b      	ldr	r3, [r3, #0]
    993e:	6a5b      	ldr	r3, [r3, #36]	; 0x24
    9940:	60bb      	str	r3, [r7, #8]

  if (fifo == 0U)
    9942:	78fb      	ldrb	r3, [r7, #3]
    9944:	2b00      	cmp	r3, #0
    9946:	d107      	bne.n	9958 <HAL_PCDEx_SetTxFiFo+0x2e>
  {
    hpcd->Instance->DIEPTXF0_HNPTXFSIZ = ((uint32_t)size << 16) | Tx_Offset;
    9948:	883b      	ldrh	r3, [r7, #0]
    994a:	0419      	lsls	r1, r3, #16
    994c:	687b      	ldr	r3, [r7, #4]
    994e:	681b      	ldr	r3, [r3, #0]
    9950:	68ba      	ldr	r2, [r7, #8]
    9952:	430a      	orrs	r2, r1
    9954:	629a      	str	r2, [r3, #40]	; 0x28
    9956:	e028      	b.n	99aa <HAL_PCDEx_SetTxFiFo+0x80>
  }
  else
  {
    Tx_Offset += (hpcd->Instance->DIEPTXF0_HNPTXFSIZ) >> 16;
    9958:	687b      	ldr	r3, [r7, #4]
    995a:	681b      	ldr	r3, [r3, #0]
    995c:	6a9b      	ldr	r3, [r3, #40]	; 0x28
    995e:	0c1b      	lsrs	r3, r3, #16
    9960:	68ba      	ldr	r2, [r7, #8]
    9962:	4413      	add	r3, r2
    9964:	60bb      	str	r3, [r7, #8]
    for (i = 0U; i < (fifo - 1U); i++)
    9966:	2300      	movs	r3, #0
    9968:	73fb      	strb	r3, [r7, #15]
    996a:	e00d      	b.n	9988 <HAL_PCDEx_SetTxFiFo+0x5e>
    {
      Tx_Offset += (hpcd->Instance->DIEPTXF[i] >> 16);
    996c:	687b      	ldr	r3, [r7, #4]
    996e:	681a      	ldr	r2, [r3, #0]
    9970:	7bfb      	ldrb	r3, [r7, #15]
    9972:	3340      	adds	r3, #64	; 0x40
    9974:	009b      	lsls	r3, r3, #2
    9976:	4413      	add	r3, r2
    9978:	685b      	ldr	r3, [r3, #4]
    997a:	0c1b      	lsrs	r3, r3, #16
    997c:	68ba      	ldr	r2, [r7, #8]
    997e:	4413      	add	r3, r2
    9980:	60bb      	str	r3, [r7, #8]
    for (i = 0U; i < (fifo - 1U); i++)
    9982:	7bfb      	ldrb	r3, [r7, #15]
    9984:	3301      	adds	r3, #1
    9986:	73fb      	strb	r3, [r7, #15]
    9988:	7bfa      	ldrb	r2, [r7, #15]
    998a:	78fb      	ldrb	r3, [r7, #3]
    998c:	3b01      	subs	r3, #1
    998e:	429a      	cmp	r2, r3
    9990:	d3ec      	bcc.n	996c <HAL_PCDEx_SetTxFiFo+0x42>
    }

    /* Multiply Tx_Size by 2 to get higher performance */
    hpcd->Instance->DIEPTXF[fifo - 1U] = ((uint32_t)size << 16) | Tx_Offset;
    9992:	883b      	ldrh	r3, [r7, #0]
    9994:	0418      	lsls	r0, r3, #16
    9996:	687b      	ldr	r3, [r7, #4]
    9998:	6819      	ldr	r1, [r3, #0]
    999a:	78fb      	ldrb	r3, [r7, #3]
    999c:	3b01      	subs	r3, #1
    999e:	68ba      	ldr	r2, [r7, #8]
    99a0:	4302      	orrs	r2, r0
    99a2:	3340      	adds	r3, #64	; 0x40
    99a4:	009b      	lsls	r3, r3, #2
    99a6:	440b      	add	r3, r1
    99a8:	605a      	str	r2, [r3, #4]
  }

  return HAL_OK;
    99aa:	2300      	movs	r3, #0
}
    99ac:	4618      	mov	r0, r3
    99ae:	3714      	adds	r7, #20
    99b0:	46bd      	mov	sp, r7
    99b2:	f85d 7b04 	ldr.w	r7, [sp], #4
    99b6:	4770      	bx	lr

000099b8 <HAL_PCDEx_SetRxFiFo>:
  * @param  hpcd PCD handle
  * @param  size Size of Rx fifo
  * @retval HAL status
  */
HAL_StatusTypeDef HAL_PCDEx_SetRxFiFo(PCD_HandleTypeDef *hpcd, uint16_t size)
{
    99b8:	b480      	push	{r7}
    99ba:	b083      	sub	sp, #12
    99bc:	af00      	add	r7, sp, #0
    99be:	6078      	str	r0, [r7, #4]
    99c0:	460b      	mov	r3, r1
    99c2:	807b      	strh	r3, [r7, #2]
  hpcd->Instance->GRXFSIZ = size;
    99c4:	687b      	ldr	r3, [r7, #4]
    99c6:	681b      	ldr	r3, [r3, #0]
    99c8:	887a      	ldrh	r2, [r7, #2]
    99ca:	625a      	str	r2, [r3, #36]	; 0x24

  return HAL_OK;
    99cc:	2300      	movs	r3, #0
}
    99ce:	4618      	mov	r0, r3
    99d0:	370c      	adds	r7, #12
    99d2:	46bd      	mov	sp, r7
    99d4:	f85d 7b04 	ldr.w	r7, [sp], #4
    99d8:	4770      	bx	lr
	...

000099dc <HAL_RCC_OscConfig>:
  *         supported by this API. User should request a transition to HSE Off
  *         first and then HSE On or HSE Bypass.
  * @retval HAL status
  */
__weak HAL_StatusTypeDef HAL_RCC_OscConfig(RCC_OscInitTypeDef  *RCC_OscInitStruct)
{
    99dc:	b580      	push	{r7, lr}
    99de:	b086      	sub	sp, #24
    99e0:	af00      	add	r7, sp, #0
    99e2:	6078      	str	r0, [r7, #4]
  uint32_t tickstart;

  /* Check Null pointer */
  if(RCC_OscInitStruct == NULL)
    99e4:	687b      	ldr	r3, [r7, #4]
    99e6:	2b00      	cmp	r3, #0
    99e8:	d101      	bne.n	99ee <HAL_RCC_OscConfig+0x12>
  {
    return HAL_ERROR;
    99ea:	2301      	movs	r3, #1
    99ec:	e22d      	b.n	9e4a <HAL_RCC_OscConfig+0x46e>
  }

  /* Check the parameters */
  assert_param(IS_RCC_OSCILLATORTYPE(RCC_OscInitStruct->OscillatorType));
  /*------------------------------- HSE Configuration ------------------------*/
  if(((RCC_OscInitStruct->OscillatorType) & RCC_OSCILLATORTYPE_HSE) == RCC_OSCILLATORTYPE_HSE)
    99ee:	687b      	ldr	r3, [r7, #4]
    99f0:	681b      	ldr	r3, [r3, #0]
    99f2:	f003 0301 	and.w	r3, r3, #1
    99f6:	2b00      	cmp	r3, #0
    99f8:	d075      	beq.n	9ae6 <HAL_RCC_OscConfig+0x10a>
  {
    /* Check the parameters */
    assert_param(IS_RCC_HSE(RCC_OscInitStruct->HSEState));
    /* When the HSE is used as system clock or clock source for PLL in these cases HSE will not disabled */
    if((__HAL_RCC_GET_SYSCLK_SOURCE() == RCC_CFGR_SWS_HSE) ||\
    99fa:	4ba3      	ldr	r3, [pc, #652]	; (9c88 <HAL_RCC_OscConfig+0x2ac>)
    99fc:	689b      	ldr	r3, [r3, #8]
    99fe:	f003 030c 	and.w	r3, r3, #12
    9a02:	2b04      	cmp	r3, #4
    9a04:	d00c      	beq.n	9a20 <HAL_RCC_OscConfig+0x44>
      ((__HAL_RCC_GET_SYSCLK_SOURCE() == RCC_CFGR_SWS_PLL) && ((RCC->PLLCFGR & RCC_PLLCFGR_PLLSRC) == RCC_PLLCFGR_PLLSRC_HSE)))
    9a06:	4ba0      	ldr	r3, [pc, #640]	; (9c88 <HAL_RCC_OscConfig+0x2ac>)
    9a08:	689b      	ldr	r3, [r3, #8]
    9a0a:	f003 030c 	and.w	r3, r3, #12
    if((__HAL_RCC_GET_SYSCLK_SOURCE() == RCC_CFGR_SWS_HSE) ||\
    9a0e:	2b08      	cmp	r3, #8
    9a10:	d112      	bne.n	9a38 <HAL_RCC_OscConfig+0x5c>
      ((__HAL_RCC_GET_SYSCLK_SOURCE() == RCC_CFGR_SWS_PLL) && ((RCC->PLLCFGR & RCC_PLLCFGR_PLLSRC) == RCC_PLLCFGR_PLLSRC_HSE)))
    9a12:	4b9d      	ldr	r3, [pc, #628]	; (9c88 <HAL_RCC_OscConfig+0x2ac>)
    9a14:	685b      	ldr	r3, [r3, #4]
    9a16:	f403 0380 	and.w	r3, r3, #4194304	; 0x400000
    9a1a:	f5b3 0f80 	cmp.w	r3, #4194304	; 0x400000
    9a1e:	d10b      	bne.n	9a38 <HAL_RCC_OscConfig+0x5c>
    {
      if((__HAL_RCC_GET_FLAG(RCC_FLAG_HSERDY) != RESET) && (RCC_OscInitStruct->HSEState == RCC_HSE_OFF))
    9a20:	4b99      	ldr	r3, [pc, #612]	; (9c88 <HAL_RCC_OscConfig+0x2ac>)
    9a22:	681b      	ldr	r3, [r3, #0]
    9a24:	f403 3300 	and.w	r3, r3, #131072	; 0x20000
    9a28:	2b00      	cmp	r3, #0
    9a2a:	d05b      	beq.n	9ae4 <HAL_RCC_OscConfig+0x108>
    9a2c:	687b      	ldr	r3, [r7, #4]
    9a2e:	685b      	ldr	r3, [r3, #4]
    9a30:	2b00      	cmp	r3, #0
    9a32:	d157      	bne.n	9ae4 <HAL_RCC_OscConfig+0x108>
      {
        return HAL_ERROR;
    9a34:	2301      	movs	r3, #1
    9a36:	e208      	b.n	9e4a <HAL_RCC_OscConfig+0x46e>
      }
    }
    else
    {
      /* Set the new HSE configuration ---------------------------------------*/
      __HAL_RCC_HSE_CONFIG(RCC_OscInitStruct->HSEState);
    9a38:	687b      	ldr	r3, [r7, #4]
    9a3a:	685b      	ldr	r3, [r3, #4]
    9a3c:	f5b3 3f80 	cmp.w	r3, #65536	; 0x10000
    9a40:	d106      	bne.n	9a50 <HAL_RCC_OscConfig+0x74>
    9a42:	4b91      	ldr	r3, [pc, #580]	; (9c88 <HAL_RCC_OscConfig+0x2ac>)
    9a44:	681b      	ldr	r3, [r3, #0]
    9a46:	4a90      	ldr	r2, [pc, #576]	; (9c88 <HAL_RCC_OscConfig+0x2ac>)
    9a48:	f443 3380 	orr.w	r3, r3, #65536	; 0x10000
    9a4c:	6013      	str	r3, [r2, #0]
    9a4e:	e01d      	b.n	9a8c <HAL_RCC_OscConfig+0xb0>
    9a50:	687b      	ldr	r3, [r7, #4]
    9a52:	685b      	ldr	r3, [r3, #4]
    9a54:	f5b3 2fa0 	cmp.w	r3, #327680	; 0x50000
    9a58:	d10c      	bne.n	9a74 <HAL_RCC_OscConfig+0x98>
    9a5a:	4b8b      	ldr	r3, [pc, #556]	; (9c88 <HAL_RCC_OscConfig+0x2ac>)
    9a5c:	681b      	ldr	r3, [r3, #0]
    9a5e:	4a8a      	ldr	r2, [pc, #552]	; (9c88 <HAL_RCC_OscConfig+0x2ac>)
    9a60:	f443 2380 	orr.w	r3, r3, #262144	; 0x40000
    9a64:	6013      	str	r3, [r2, #0]
    9a66:	4b88      	ldr	r3, [pc, #544]	; (9c88 <HAL_RCC_OscConfig+0x2ac>)
    9a68:	681b      	ldr	r3, [r3, #0]
    9a6a:	4a87      	ldr	r2, [pc, #540]	; (9c88 <HAL_RCC_OscConfig+0x2ac>)
    9a6c:	f443 3380 	orr.w	r3, r3, #65536	; 0x10000
    9a70:	6013      	str	r3, [r2, #0]
    9a72:	e00b      	b.n	9a8c <HAL_RCC_OscConfig+0xb0>
    9a74:	4b84      	ldr	r3, [pc, #528]	; (9c88 <HAL_RCC_OscConfig+0x2ac>)
    9a76:	681b      	ldr	r3, [r3, #0]
    9a78:	4a83      	ldr	r2, [pc, #524]	; (9c88 <HAL_RCC_OscConfig+0x2ac>)
    9a7a:	f423 3380 	bic.w	r3, r3, #65536	; 0x10000
    9a7e:	6013      	str	r3, [r2, #0]
    9a80:	4b81      	ldr	r3, [pc, #516]	; (9c88 <HAL_RCC_OscConfig+0x2ac>)
    9a82:	681b      	ldr	r3, [r3, #0]
    9a84:	4a80      	ldr	r2, [pc, #512]	; (9c88 <HAL_RCC_OscConfig+0x2ac>)
    9a86:	f423 2380 	bic.w	r3, r3, #262144	; 0x40000
    9a8a:	6013      	str	r3, [r2, #0]

      /* Check the HSE State */
      if((RCC_OscInitStruct->HSEState) != RCC_HSE_OFF)
    9a8c:	687b      	ldr	r3, [r7, #4]
    9a8e:	685b      	ldr	r3, [r3, #4]
    9a90:	2b00      	cmp	r3, #0
    9a92:	d013      	beq.n	9abc <HAL_RCC_OscConfig+0xe0>
      {
        /* Get Start Tick */
        tickstart = HAL_GetTick();
    9a94:	f7fe fb7a 	bl	818c <HAL_GetTick>
    9a98:	6138      	str	r0, [r7, #16]

        /* Wait till HSE is ready */
        while(__HAL_RCC_GET_FLAG(RCC_FLAG_HSERDY) == RESET)
    9a9a:	e008      	b.n	9aae <HAL_RCC_OscConfig+0xd2>
        {
          if((HAL_GetTick() - tickstart ) > HSE_TIMEOUT_VALUE)
    9a9c:	f7fe fb76 	bl	818c <HAL_GetTick>
    9aa0:	4602      	mov	r2, r0
    9aa2:	693b      	ldr	r3, [r7, #16]
    9aa4:	1ad3      	subs	r3, r2, r3
    9aa6:	2b64      	cmp	r3, #100	; 0x64
    9aa8:	d901      	bls.n	9aae <HAL_RCC_OscConfig+0xd2>
          {
            return HAL_TIMEOUT;
    9aaa:	2303      	movs	r3, #3
    9aac:	e1cd      	b.n	9e4a <HAL_RCC_OscConfig+0x46e>
        while(__HAL_RCC_GET_FLAG(RCC_FLAG_HSERDY) == RESET)
    9aae:	4b76      	ldr	r3, [pc, #472]	; (9c88 <HAL_RCC_OscConfig+0x2ac>)
    9ab0:	681b      	ldr	r3, [r3, #0]
    9ab2:	f403 3300 	and.w	r3, r3, #131072	; 0x20000
    9ab6:	2b00      	cmp	r3, #0
    9ab8:	d0f0      	beq.n	9a9c <HAL_RCC_OscConfig+0xc0>
    9aba:	e014      	b.n	9ae6 <HAL_RCC_OscConfig+0x10a>
        }
      }
      else
      {
        /* Get Start Tick */
        tickstart = HAL_GetTick();
    9abc:	f7fe fb66 	bl	818c <HAL_GetTick>
    9ac0:	6138      	str	r0, [r7, #16]

        /* Wait till HSE is bypassed or disabled */
        while(__HAL_RCC_GET_FLAG(RCC_FLAG_HSERDY) != RESET)
    9ac2:	e008      	b.n	9ad6 <HAL_RCC_OscConfig+0xfa>
        {
          if((HAL_GetTick() - tickstart ) > HSE_TIMEOUT_VALUE)
    9ac4:	f7fe fb62 	bl	818c <HAL_GetTick>
    9ac8:	4602      	mov	r2, r0
    9aca:	693b      	ldr	r3, [r7, #16]
    9acc:	1ad3      	subs	r3, r2, r3
    9ace:	2b64      	cmp	r3, #100	; 0x64
    9ad0:	d901      	bls.n	9ad6 <HAL_RCC_OscConfig+0xfa>
          {
            return HAL_TIMEOUT;
    9ad2:	2303      	movs	r3, #3
    9ad4:	e1b9      	b.n	9e4a <HAL_RCC_OscConfig+0x46e>
        while(__HAL_RCC_GET_FLAG(RCC_FLAG_HSERDY) != RESET)
    9ad6:	4b6c      	ldr	r3, [pc, #432]	; (9c88 <HAL_RCC_OscConfig+0x2ac>)
    9ad8:	681b      	ldr	r3, [r3, #0]
    9ada:	f403 3300 	and.w	r3, r3, #131072	; 0x20000
    9ade:	2b00      	cmp	r3, #0
    9ae0:	d1f0      	bne.n	9ac4 <HAL_RCC_OscConfig+0xe8>
    9ae2:	e000      	b.n	9ae6 <HAL_RCC_OscConfig+0x10a>
      if((__HAL_RCC_GET_FLAG(RCC_FLAG_HSERDY) != RESET) && (RCC_OscInitStruct->HSEState == RCC_HSE_OFF))
    9ae4:	bf00      	nop
        }
      }
    }
  }
  /*----------------------------- HSI Configuration --------------------------*/
  if(((RCC_OscInitStruct->OscillatorType) & RCC_OSCILLATORTYPE_HSI) == RCC_OSCILLATORTYPE_HSI)
    9ae6:	687b      	ldr	r3, [r7, #4]
    9ae8:	681b      	ldr	r3, [r3, #0]
    9aea:	f003 0302 	and.w	r3, r3, #2
    9aee:	2b00      	cmp	r3, #0
    9af0:	d063      	beq.n	9bba <HAL_RCC_OscConfig+0x1de>
    /* Check the parameters */
    assert_param(IS_RCC_HSI(RCC_OscInitStruct->HSIState));
    assert_param(IS_RCC_CALIBRATION_VALUE(RCC_OscInitStruct->HSICalibrationValue));

    /* Check if HSI is used as system clock or as PLL source when PLL is selected as system clock */
    if((__HAL_RCC_GET_SYSCLK_SOURCE() == RCC_CFGR_SWS_HSI) ||\
    9af2:	4b65      	ldr	r3, [pc, #404]	; (9c88 <HAL_RCC_OscConfig+0x2ac>)
    9af4:	689b      	ldr	r3, [r3, #8]
    9af6:	f003 030c 	and.w	r3, r3, #12
    9afa:	2b00      	cmp	r3, #0
    9afc:	d00b      	beq.n	9b16 <HAL_RCC_OscConfig+0x13a>
      ((__HAL_RCC_GET_SYSCLK_SOURCE() == RCC_CFGR_SWS_PLL) && ((RCC->PLLCFGR & RCC_PLLCFGR_PLLSRC) == RCC_PLLCFGR_PLLSRC_HSI)))
    9afe:	4b62      	ldr	r3, [pc, #392]	; (9c88 <HAL_RCC_OscConfig+0x2ac>)
    9b00:	689b      	ldr	r3, [r3, #8]
    9b02:	f003 030c 	and.w	r3, r3, #12
    if((__HAL_RCC_GET_SYSCLK_SOURCE() == RCC_CFGR_SWS_HSI) ||\
    9b06:	2b08      	cmp	r3, #8
    9b08:	d11c      	bne.n	9b44 <HAL_RCC_OscConfig+0x168>
      ((__HAL_RCC_GET_SYSCLK_SOURCE() == RCC_CFGR_SWS_PLL) && ((RCC->PLLCFGR & RCC_PLLCFGR_PLLSRC) == RCC_PLLCFGR_PLLSRC_HSI)))
    9b0a:	4b5f      	ldr	r3, [pc, #380]	; (9c88 <HAL_RCC_OscConfig+0x2ac>)
    9b0c:	685b      	ldr	r3, [r3, #4]
    9b0e:	f403 0380 	and.w	r3, r3, #4194304	; 0x400000
    9b12:	2b00      	cmp	r3, #0
    9b14:	d116      	bne.n	9b44 <HAL_RCC_OscConfig+0x168>
    {
      /* When HSI is used as system clock it will not disabled */
      if((__HAL_RCC_GET_FLAG(RCC_FLAG_HSIRDY) != RESET) && (RCC_OscInitStruct->HSIState != RCC_HSI_ON))
    9b16:	4b5c      	ldr	r3, [pc, #368]	; (9c88 <HAL_RCC_OscConfig+0x2ac>)
    9b18:	681b      	ldr	r3, [r3, #0]
    9b1a:	f003 0302 	and.w	r3, r3, #2
    9b1e:	2b00      	cmp	r3, #0
    9b20:	d005      	beq.n	9b2e <HAL_RCC_OscConfig+0x152>
    9b22:	687b      	ldr	r3, [r7, #4]
    9b24:	68db      	ldr	r3, [r3, #12]
    9b26:	2b01      	cmp	r3, #1
    9b28:	d001      	beq.n	9b2e <HAL_RCC_OscConfig+0x152>
      {
        return HAL_ERROR;
    9b2a:	2301      	movs	r3, #1
    9b2c:	e18d      	b.n	9e4a <HAL_RCC_OscConfig+0x46e>
      }
      /* Otherwise, just the calibration is allowed */
      else
      {
        /* Adjusts the Internal High Speed oscillator (HSI) calibration value.*/
        __HAL_RCC_HSI_CALIBRATIONVALUE_ADJUST(RCC_OscInitStruct->HSICalibrationValue);
    9b2e:	4b56      	ldr	r3, [pc, #344]	; (9c88 <HAL_RCC_OscConfig+0x2ac>)
    9b30:	681b      	ldr	r3, [r3, #0]
    9b32:	f023 02f8 	bic.w	r2, r3, #248	; 0xf8
    9b36:	687b      	ldr	r3, [r7, #4]
    9b38:	691b      	ldr	r3, [r3, #16]
    9b3a:	00db      	lsls	r3, r3, #3
    9b3c:	4952      	ldr	r1, [pc, #328]	; (9c88 <HAL_RCC_OscConfig+0x2ac>)
    9b3e:	4313      	orrs	r3, r2
    9b40:	600b      	str	r3, [r1, #0]
      if((__HAL_RCC_GET_FLAG(RCC_FLAG_HSIRDY) != RESET) && (RCC_OscInitStruct->HSIState != RCC_HSI_ON))
    9b42:	e03a      	b.n	9bba <HAL_RCC_OscConfig+0x1de>
      }
    }
    else
    {
      /* Check the HSI State */
      if((RCC_OscInitStruct->HSIState)!= RCC_HSI_OFF)
    9b44:	687b      	ldr	r3, [r7, #4]
    9b46:	68db      	ldr	r3, [r3, #12]
    9b48:	2b00      	cmp	r3, #0
    9b4a:	d020      	beq.n	9b8e <HAL_RCC_OscConfig+0x1b2>
      {
        /* Enable the Internal High Speed oscillator (HSI). */
        __HAL_RCC_HSI_ENABLE();
    9b4c:	4b4f      	ldr	r3, [pc, #316]	; (9c8c <HAL_RCC_OscConfig+0x2b0>)
    9b4e:	2201      	movs	r2, #1
    9b50:	601a      	str	r2, [r3, #0]

        /* Get Start Tick*/
        tickstart = HAL_GetTick();
    9b52:	f7fe fb1b 	bl	818c <HAL_GetTick>
    9b56:	6138      	str	r0, [r7, #16]

        /* Wait till HSI is ready */
        while(__HAL_RCC_GET_FLAG(RCC_FLAG_HSIRDY) == RESET)
    9b58:	e008      	b.n	9b6c <HAL_RCC_OscConfig+0x190>
        {
          if((HAL_GetTick() - tickstart ) > HSI_TIMEOUT_VALUE)
    9b5a:	f7fe fb17 	bl	818c <HAL_GetTick>
    9b5e:	4602      	mov	r2, r0
    9b60:	693b      	ldr	r3, [r7, #16]
    9b62:	1ad3      	subs	r3, r2, r3
    9b64:	2b02      	cmp	r3, #2
    9b66:	d901      	bls.n	9b6c <HAL_RCC_OscConfig+0x190>
          {
            return HAL_TIMEOUT;
    9b68:	2303      	movs	r3, #3
    9b6a:	e16e      	b.n	9e4a <HAL_RCC_OscConfig+0x46e>
        while(__HAL_RCC_GET_FLAG(RCC_FLAG_HSIRDY) == RESET)
    9b6c:	4b46      	ldr	r3, [pc, #280]	; (9c88 <HAL_RCC_OscConfig+0x2ac>)
    9b6e:	681b      	ldr	r3, [r3, #0]
    9b70:	f003 0302 	and.w	r3, r3, #2
    9b74:	2b00      	cmp	r3, #0
    9b76:	d0f0      	beq.n	9b5a <HAL_RCC_OscConfig+0x17e>
          }
        }

        /* Adjusts the Internal High Speed oscillator (HSI) calibration value. */
        __HAL_RCC_HSI_CALIBRATIONVALUE_ADJUST(RCC_OscInitStruct->HSICalibrationValue);
    9b78:	4b43      	ldr	r3, [pc, #268]	; (9c88 <HAL_RCC_OscConfig+0x2ac>)
    9b7a:	681b      	ldr	r3, [r3, #0]
    9b7c:	f023 02f8 	bic.w	r2, r3, #248	; 0xf8
    9b80:	687b      	ldr	r3, [r7, #4]
    9b82:	691b      	ldr	r3, [r3, #16]
    9b84:	00db      	lsls	r3, r3, #3
    9b86:	4940      	ldr	r1, [pc, #256]	; (9c88 <HAL_RCC_OscConfig+0x2ac>)
    9b88:	4313      	orrs	r3, r2
    9b8a:	600b      	str	r3, [r1, #0]
    9b8c:	e015      	b.n	9bba <HAL_RCC_OscConfig+0x1de>
      }
      else
      {
        /* Disable the Internal High Speed oscillator (HSI). */
        __HAL_RCC_HSI_DISABLE();
    9b8e:	4b3f      	ldr	r3, [pc, #252]	; (9c8c <HAL_RCC_OscConfig+0x2b0>)
    9b90:	2200      	movs	r2, #0
    9b92:	601a      	str	r2, [r3, #0]

        /* Get Start Tick*/
        tickstart = HAL_GetTick();
    9b94:	f7fe fafa 	bl	818c <HAL_GetTick>
    9b98:	6138      	str	r0, [r7, #16]

        /* Wait till HSI is ready */
        while(__HAL_RCC_GET_FLAG(RCC_FLAG_HSIRDY) != RESET)
    9b9a:	e008      	b.n	9bae <HAL_RCC_OscConfig+0x1d2>
        {
          if((HAL_GetTick() - tickstart ) > HSI_TIMEOUT_VALUE)
    9b9c:	f7fe faf6 	bl	818c <HAL_GetTick>
    9ba0:	4602      	mov	r2, r0
    9ba2:	693b      	ldr	r3, [r7, #16]
    9ba4:	1ad3      	subs	r3, r2, r3
    9ba6:	2b02      	cmp	r3, #2
    9ba8:	d901      	bls.n	9bae <HAL_RCC_OscConfig+0x1d2>
          {
            return HAL_TIMEOUT;
    9baa:	2303      	movs	r3, #3
    9bac:	e14d      	b.n	9e4a <HAL_RCC_OscConfig+0x46e>
        while(__HAL_RCC_GET_FLAG(RCC_FLAG_HSIRDY) != RESET)
    9bae:	4b36      	ldr	r3, [pc, #216]	; (9c88 <HAL_RCC_OscConfig+0x2ac>)
    9bb0:	681b      	ldr	r3, [r3, #0]
    9bb2:	f003 0302 	and.w	r3, r3, #2
    9bb6:	2b00      	cmp	r3, #0
    9bb8:	d1f0      	bne.n	9b9c <HAL_RCC_OscConfig+0x1c0>
        }
      }
    }
  }
  /*------------------------------ LSI Configuration -------------------------*/
  if(((RCC_OscInitStruct->OscillatorType) & RCC_OSCILLATORTYPE_LSI) == RCC_OSCILLATORTYPE_LSI)
    9bba:	687b      	ldr	r3, [r7, #4]
    9bbc:	681b      	ldr	r3, [r3, #0]
    9bbe:	f003 0308 	and.w	r3, r3, #8
    9bc2:	2b00      	cmp	r3, #0
    9bc4:	d030      	beq.n	9c28 <HAL_RCC_OscConfig+0x24c>
  {
    /* Check the parameters */
    assert_param(IS_RCC_LSI(RCC_OscInitStruct->LSIState));

    /* Check the LSI State */
    if((RCC_OscInitStruct->LSIState)!= RCC_LSI_OFF)
    9bc6:	687b      	ldr	r3, [r7, #4]
    9bc8:	695b      	ldr	r3, [r3, #20]
    9bca:	2b00      	cmp	r3, #0
    9bcc:	d016      	beq.n	9bfc <HAL_RCC_OscConfig+0x220>
    {
      /* Enable the Internal Low Speed oscillator (LSI). */
      __HAL_RCC_LSI_ENABLE();
    9bce:	4b30      	ldr	r3, [pc, #192]	; (9c90 <HAL_RCC_OscConfig+0x2b4>)
    9bd0:	2201      	movs	r2, #1
    9bd2:	601a      	str	r2, [r3, #0]

      /* Get Start Tick*/
      tickstart = HAL_GetTick();
    9bd4:	f7fe fada 	bl	818c <HAL_GetTick>
    9bd8:	6138      	str	r0, [r7, #16]

      /* Wait till LSI is ready */
      while(__HAL_RCC_GET_FLAG(RCC_FLAG_LSIRDY) == RESET)
    9bda:	e008      	b.n	9bee <HAL_RCC_OscConfig+0x212>
      {
        if((HAL_GetTick() - tickstart ) > LSI_TIMEOUT_VALUE)
    9bdc:	f7fe fad6 	bl	818c <HAL_GetTick>
    9be0:	4602      	mov	r2, r0
    9be2:	693b      	ldr	r3, [r7, #16]
    9be4:	1ad3      	subs	r3, r2, r3
    9be6:	2b02      	cmp	r3, #2
    9be8:	d901      	bls.n	9bee <HAL_RCC_OscConfig+0x212>
        {
          return HAL_TIMEOUT;
    9bea:	2303      	movs	r3, #3
    9bec:	e12d      	b.n	9e4a <HAL_RCC_OscConfig+0x46e>
      while(__HAL_RCC_GET_FLAG(RCC_FLAG_LSIRDY) == RESET)
    9bee:	4b26      	ldr	r3, [pc, #152]	; (9c88 <HAL_RCC_OscConfig+0x2ac>)
    9bf0:	6f5b      	ldr	r3, [r3, #116]	; 0x74
    9bf2:	f003 0302 	and.w	r3, r3, #2
    9bf6:	2b00      	cmp	r3, #0
    9bf8:	d0f0      	beq.n	9bdc <HAL_RCC_OscConfig+0x200>
    9bfa:	e015      	b.n	9c28 <HAL_RCC_OscConfig+0x24c>
      }
    }
    else
    {
      /* Disable the Internal Low Speed oscillator (LSI). */
      __HAL_RCC_LSI_DISABLE();
    9bfc:	4b24      	ldr	r3, [pc, #144]	; (9c90 <HAL_RCC_OscConfig+0x2b4>)
    9bfe:	2200      	movs	r2, #0
    9c00:	601a      	str	r2, [r3, #0]

      /* Get Start Tick */
      tickstart = HAL_GetTick();
    9c02:	f7fe fac3 	bl	818c <HAL_GetTick>
    9c06:	6138      	str	r0, [r7, #16]

      /* Wait till LSI is ready */
      while(__HAL_RCC_GET_FLAG(RCC_FLAG_LSIRDY) != RESET)
    9c08:	e008      	b.n	9c1c <HAL_RCC_OscConfig+0x240>
      {
        if((HAL_GetTick() - tickstart ) > LSI_TIMEOUT_VALUE)
    9c0a:	f7fe fabf 	bl	818c <HAL_GetTick>
    9c0e:	4602      	mov	r2, r0
    9c10:	693b      	ldr	r3, [r7, #16]
    9c12:	1ad3      	subs	r3, r2, r3
    9c14:	2b02      	cmp	r3, #2
    9c16:	d901      	bls.n	9c1c <HAL_RCC_OscConfig+0x240>
        {
          return HAL_TIMEOUT;
    9c18:	2303      	movs	r3, #3
    9c1a:	e116      	b.n	9e4a <HAL_RCC_OscConfig+0x46e>
      while(__HAL_RCC_GET_FLAG(RCC_FLAG_LSIRDY) != RESET)
    9c1c:	4b1a      	ldr	r3, [pc, #104]	; (9c88 <HAL_RCC_OscConfig+0x2ac>)
    9c1e:	6f5b      	ldr	r3, [r3, #116]	; 0x74
    9c20:	f003 0302 	and.w	r3, r3, #2
    9c24:	2b00      	cmp	r3, #0
    9c26:	d1f0      	bne.n	9c0a <HAL_RCC_OscConfig+0x22e>
        }
      }
    }
  }
  /*------------------------------ LSE Configuration -------------------------*/
  if(((RCC_OscInitStruct->OscillatorType) & RCC_OSCILLATORTYPE_LSE) == RCC_OSCILLATORTYPE_LSE)
    9c28:	687b      	ldr	r3, [r7, #4]
    9c2a:	681b      	ldr	r3, [r3, #0]
    9c2c:	f003 0304 	and.w	r3, r3, #4
    9c30:	2b00      	cmp	r3, #0
    9c32:	f000 80a0 	beq.w	9d76 <HAL_RCC_OscConfig+0x39a>
  {
    FlagStatus       pwrclkchanged = RESET;
    9c36:	2300      	movs	r3, #0
    9c38:	75fb      	strb	r3, [r7, #23]
    /* Check the parameters */
    assert_param(IS_RCC_LSE(RCC_OscInitStruct->LSEState));

    /* Update LSE configuration in Backup Domain control register    */
    /* Requires to enable write access to Backup Domain of necessary */
    if(__HAL_RCC_PWR_IS_CLK_DISABLED())
    9c3a:	4b13      	ldr	r3, [pc, #76]	; (9c88 <HAL_RCC_OscConfig+0x2ac>)
    9c3c:	6c1b      	ldr	r3, [r3, #64]	; 0x40
    9c3e:	f003 5380 	and.w	r3, r3, #268435456	; 0x10000000
    9c42:	2b00      	cmp	r3, #0
    9c44:	d10f      	bne.n	9c66 <HAL_RCC_OscConfig+0x28a>
    {
      __HAL_RCC_PWR_CLK_ENABLE();
    9c46:	2300      	movs	r3, #0
    9c48:	60fb      	str	r3, [r7, #12]
    9c4a:	4b0f      	ldr	r3, [pc, #60]	; (9c88 <HAL_RCC_OscConfig+0x2ac>)
    9c4c:	6c1b      	ldr	r3, [r3, #64]	; 0x40
    9c4e:	4a0e      	ldr	r2, [pc, #56]	; (9c88 <HAL_RCC_OscConfig+0x2ac>)
    9c50:	f043 5380 	orr.w	r3, r3, #268435456	; 0x10000000
    9c54:	6413      	str	r3, [r2, #64]	; 0x40
    9c56:	4b0c      	ldr	r3, [pc, #48]	; (9c88 <HAL_RCC_OscConfig+0x2ac>)
    9c58:	6c1b      	ldr	r3, [r3, #64]	; 0x40
    9c5a:	f003 5380 	and.w	r3, r3, #268435456	; 0x10000000
    9c5e:	60fb      	str	r3, [r7, #12]
    9c60:	68fb      	ldr	r3, [r7, #12]
      pwrclkchanged = SET;
    9c62:	2301      	movs	r3, #1
    9c64:	75fb      	strb	r3, [r7, #23]
    }

    if(HAL_IS_BIT_CLR(PWR->CR, PWR_CR_DBP))
    9c66:	4b0b      	ldr	r3, [pc, #44]	; (9c94 <HAL_RCC_OscConfig+0x2b8>)
    9c68:	681b      	ldr	r3, [r3, #0]
    9c6a:	f403 7380 	and.w	r3, r3, #256	; 0x100
    9c6e:	2b00      	cmp	r3, #0
    9c70:	d121      	bne.n	9cb6 <HAL_RCC_OscConfig+0x2da>
    {
      /* Enable write access to Backup domain */
      SET_BIT(PWR->CR, PWR_CR_DBP);
    9c72:	4b08      	ldr	r3, [pc, #32]	; (9c94 <HAL_RCC_OscConfig+0x2b8>)
    9c74:	681b      	ldr	r3, [r3, #0]
    9c76:	4a07      	ldr	r2, [pc, #28]	; (9c94 <HAL_RCC_OscConfig+0x2b8>)
    9c78:	f443 7380 	orr.w	r3, r3, #256	; 0x100
    9c7c:	6013      	str	r3, [r2, #0]

      /* Wait for Backup domain Write protection disable */
      tickstart = HAL_GetTick();
    9c7e:	f7fe fa85 	bl	818c <HAL_GetTick>
    9c82:	6138      	str	r0, [r7, #16]

      while(HAL_IS_BIT_CLR(PWR->CR, PWR_CR_DBP))
    9c84:	e011      	b.n	9caa <HAL_RCC_OscConfig+0x2ce>
    9c86:	bf00      	nop
    9c88:	40023800 	.word	0x40023800
    9c8c:	42470000 	.word	0x42470000
    9c90:	42470e80 	.word	0x42470e80
    9c94:	40007000 	.word	0x40007000
      {
        if((HAL_GetTick() - tickstart) > RCC_DBP_TIMEOUT_VALUE)
    9c98:	f7fe fa78 	bl	818c <HAL_GetTick>
    9c9c:	4602      	mov	r2, r0
    9c9e:	693b      	ldr	r3, [r7, #16]
    9ca0:	1ad3      	subs	r3, r2, r3
    9ca2:	2b02      	cmp	r3, #2
    9ca4:	d901      	bls.n	9caa <HAL_RCC_OscConfig+0x2ce>
        {
          return HAL_TIMEOUT;
    9ca6:	2303      	movs	r3, #3
    9ca8:	e0cf      	b.n	9e4a <HAL_RCC_OscConfig+0x46e>
      while(HAL_IS_BIT_CLR(PWR->CR, PWR_CR_DBP))
    9caa:	4b6a      	ldr	r3, [pc, #424]	; (9e54 <HAL_RCC_OscConfig+0x478>)
    9cac:	681b      	ldr	r3, [r3, #0]
    9cae:	f403 7380 	and.w	r3, r3, #256	; 0x100
    9cb2:	2b00      	cmp	r3, #0
    9cb4:	d0f0      	beq.n	9c98 <HAL_RCC_OscConfig+0x2bc>
        }
      }
    }

    /* Set the new LSE configuration -----------------------------------------*/
    __HAL_RCC_LSE_CONFIG(RCC_OscInitStruct->LSEState);
    9cb6:	687b      	ldr	r3, [r7, #4]
    9cb8:	689b      	ldr	r3, [r3, #8]
    9cba:	2b01      	cmp	r3, #1
    9cbc:	d106      	bne.n	9ccc <HAL_RCC_OscConfig+0x2f0>
    9cbe:	4b66      	ldr	r3, [pc, #408]	; (9e58 <HAL_RCC_OscConfig+0x47c>)
    9cc0:	6f1b      	ldr	r3, [r3, #112]	; 0x70
    9cc2:	4a65      	ldr	r2, [pc, #404]	; (9e58 <HAL_RCC_OscConfig+0x47c>)
    9cc4:	f043 0301 	orr.w	r3, r3, #1
    9cc8:	6713      	str	r3, [r2, #112]	; 0x70
    9cca:	e01c      	b.n	9d06 <HAL_RCC_OscConfig+0x32a>
    9ccc:	687b      	ldr	r3, [r7, #4]
    9cce:	689b      	ldr	r3, [r3, #8]
    9cd0:	2b05      	cmp	r3, #5
    9cd2:	d10c      	bne.n	9cee <HAL_RCC_OscConfig+0x312>
    9cd4:	4b60      	ldr	r3, [pc, #384]	; (9e58 <HAL_RCC_OscConfig+0x47c>)
    9cd6:	6f1b      	ldr	r3, [r3, #112]	; 0x70
    9cd8:	4a5f      	ldr	r2, [pc, #380]	; (9e58 <HAL_RCC_OscConfig+0x47c>)
    9cda:	f043 0304 	orr.w	r3, r3, #4
    9cde:	6713      	str	r3, [r2, #112]	; 0x70
    9ce0:	4b5d      	ldr	r3, [pc, #372]	; (9e58 <HAL_RCC_OscConfig+0x47c>)
    9ce2:	6f1b      	ldr	r3, [r3, #112]	; 0x70
    9ce4:	4a5c      	ldr	r2, [pc, #368]	; (9e58 <HAL_RCC_OscConfig+0x47c>)
    9ce6:	f043 0301 	orr.w	r3, r3, #1
    9cea:	6713      	str	r3, [r2, #112]	; 0x70
    9cec:	e00b      	b.n	9d06 <HAL_RCC_OscConfig+0x32a>
    9cee:	4b5a      	ldr	r3, [pc, #360]	; (9e58 <HAL_RCC_OscConfig+0x47c>)
    9cf0:	6f1b      	ldr	r3, [r3, #112]	; 0x70
    9cf2:	4a59      	ldr	r2, [pc, #356]	; (9e58 <HAL_RCC_OscConfig+0x47c>)
    9cf4:	f023 0301 	bic.w	r3, r3, #1
    9cf8:	6713      	str	r3, [r2, #112]	; 0x70
    9cfa:	4b57      	ldr	r3, [pc, #348]	; (9e58 <HAL_RCC_OscConfig+0x47c>)
    9cfc:	6f1b      	ldr	r3, [r3, #112]	; 0x70
    9cfe:	4a56      	ldr	r2, [pc, #344]	; (9e58 <HAL_RCC_OscConfig+0x47c>)
    9d00:	f023 0304 	bic.w	r3, r3, #4
    9d04:	6713      	str	r3, [r2, #112]	; 0x70
    /* Check the LSE State */
    if((RCC_OscInitStruct->LSEState) != RCC_LSE_OFF)
    9d06:	687b      	ldr	r3, [r7, #4]
    9d08:	689b      	ldr	r3, [r3, #8]
    9d0a:	2b00      	cmp	r3, #0
    9d0c:	d015      	beq.n	9d3a <HAL_RCC_OscConfig+0x35e>
    {
      /* Get Start Tick*/
      tickstart = HAL_GetTick();
    9d0e:	f7fe fa3d 	bl	818c <HAL_GetTick>
    9d12:	6138      	str	r0, [r7, #16]

      /* Wait till LSE is ready */
      while(__HAL_RCC_GET_FLAG(RCC_FLAG_LSERDY) == RESET)
    9d14:	e00a      	b.n	9d2c <HAL_RCC_OscConfig+0x350>
      {
        if((HAL_GetTick() - tickstart ) > RCC_LSE_TIMEOUT_VALUE)
    9d16:	f7fe fa39 	bl	818c <HAL_GetTick>
    9d1a:	4602      	mov	r2, r0
    9d1c:	693b      	ldr	r3, [r7, #16]
    9d1e:	1ad3      	subs	r3, r2, r3
    9d20:	f241 3288 	movw	r2, #5000	; 0x1388
    9d24:	4293      	cmp	r3, r2
    9d26:	d901      	bls.n	9d2c <HAL_RCC_OscConfig+0x350>
        {
          return HAL_TIMEOUT;
    9d28:	2303      	movs	r3, #3
    9d2a:	e08e      	b.n	9e4a <HAL_RCC_OscConfig+0x46e>
      while(__HAL_RCC_GET_FLAG(RCC_FLAG_LSERDY) == RESET)
    9d2c:	4b4a      	ldr	r3, [pc, #296]	; (9e58 <HAL_RCC_OscConfig+0x47c>)
    9d2e:	6f1b      	ldr	r3, [r3, #112]	; 0x70
    9d30:	f003 0302 	and.w	r3, r3, #2
    9d34:	2b00      	cmp	r3, #0
    9d36:	d0ee      	beq.n	9d16 <HAL_RCC_OscConfig+0x33a>
    9d38:	e014      	b.n	9d64 <HAL_RCC_OscConfig+0x388>
      }
    }
    else
    {
      /* Get Start Tick */
      tickstart = HAL_GetTick();
    9d3a:	f7fe fa27 	bl	818c <HAL_GetTick>
    9d3e:	6138      	str	r0, [r7, #16]

      /* Wait till LSE is ready */
      while(__HAL_RCC_GET_FLAG(RCC_FLAG_LSERDY) != RESET)
    9d40:	e00a      	b.n	9d58 <HAL_RCC_OscConfig+0x37c>
      {
        if((HAL_GetTick() - tickstart ) > RCC_LSE_TIMEOUT_VALUE)
    9d42:	f7fe fa23 	bl	818c <HAL_GetTick>
    9d46:	4602      	mov	r2, r0
    9d48:	693b      	ldr	r3, [r7, #16]
    9d4a:	1ad3      	subs	r3, r2, r3
    9d4c:	f241 3288 	movw	r2, #5000	; 0x1388
    9d50:	4293      	cmp	r3, r2
    9d52:	d901      	bls.n	9d58 <HAL_RCC_OscConfig+0x37c>
        {
          return HAL_TIMEOUT;
    9d54:	2303      	movs	r3, #3
    9d56:	e078      	b.n	9e4a <HAL_RCC_OscConfig+0x46e>
      while(__HAL_RCC_GET_FLAG(RCC_FLAG_LSERDY) != RESET)
    9d58:	4b3f      	ldr	r3, [pc, #252]	; (9e58 <HAL_RCC_OscConfig+0x47c>)
    9d5a:	6f1b      	ldr	r3, [r3, #112]	; 0x70
    9d5c:	f003 0302 	and.w	r3, r3, #2
    9d60:	2b00      	cmp	r3, #0
    9d62:	d1ee      	bne.n	9d42 <HAL_RCC_OscConfig+0x366>
        }
      }
    }

    /* Restore clock configuration if changed */
    if(pwrclkchanged == SET)
    9d64:	7dfb      	ldrb	r3, [r7, #23]
    9d66:	2b01      	cmp	r3, #1
    9d68:	d105      	bne.n	9d76 <HAL_RCC_OscConfig+0x39a>
    {
      __HAL_RCC_PWR_CLK_DISABLE();
    9d6a:	4b3b      	ldr	r3, [pc, #236]	; (9e58 <HAL_RCC_OscConfig+0x47c>)
    9d6c:	6c1b      	ldr	r3, [r3, #64]	; 0x40
    9d6e:	4a3a      	ldr	r2, [pc, #232]	; (9e58 <HAL_RCC_OscConfig+0x47c>)
    9d70:	f023 5380 	bic.w	r3, r3, #268435456	; 0x10000000
    9d74:	6413      	str	r3, [r2, #64]	; 0x40
    }
  }
  /*-------------------------------- PLL Configuration -----------------------*/
  /* Check the parameters */
  assert_param(IS_RCC_PLL(RCC_OscInitStruct->PLL.PLLState));
  if ((RCC_OscInitStruct->PLL.PLLState) != RCC_PLL_NONE)
    9d76:	687b      	ldr	r3, [r7, #4]
    9d78:	699b      	ldr	r3, [r3, #24]
    9d7a:	2b00      	cmp	r3, #0
    9d7c:	d064      	beq.n	9e48 <HAL_RCC_OscConfig+0x46c>
  {
    /* Check if the PLL is used as system clock or not */
    if(__HAL_RCC_GET_SYSCLK_SOURCE() != RCC_CFGR_SWS_PLL)
    9d7e:	4b36      	ldr	r3, [pc, #216]	; (9e58 <HAL_RCC_OscConfig+0x47c>)
    9d80:	689b      	ldr	r3, [r3, #8]
    9d82:	f003 030c 	and.w	r3, r3, #12
    9d86:	2b08      	cmp	r3, #8
    9d88:	d05c      	beq.n	9e44 <HAL_RCC_OscConfig+0x468>
    {
      if((RCC_OscInitStruct->PLL.PLLState) == RCC_PLL_ON)
    9d8a:	687b      	ldr	r3, [r7, #4]
    9d8c:	699b      	ldr	r3, [r3, #24]
    9d8e:	2b02      	cmp	r3, #2
    9d90:	d141      	bne.n	9e16 <HAL_RCC_OscConfig+0x43a>
        assert_param(IS_RCC_PLLN_VALUE(RCC_OscInitStruct->PLL.PLLN));
        assert_param(IS_RCC_PLLP_VALUE(RCC_OscInitStruct->PLL.PLLP));
        assert_param(IS_RCC_PLLQ_VALUE(RCC_OscInitStruct->PLL.PLLQ));

        /* Disable the main PLL. */
        __HAL_RCC_PLL_DISABLE();
    9d92:	4b32      	ldr	r3, [pc, #200]	; (9e5c <HAL_RCC_OscConfig+0x480>)
    9d94:	2200      	movs	r2, #0
    9d96:	601a      	str	r2, [r3, #0]

        /* Get Start Tick */
        tickstart = HAL_GetTick();
    9d98:	f7fe f9f8 	bl	818c <HAL_GetTick>
    9d9c:	6138      	str	r0, [r7, #16]

        /* Wait till PLL is ready */
        while(__HAL_RCC_GET_FLAG(RCC_FLAG_PLLRDY) != RESET)
    9d9e:	e008      	b.n	9db2 <HAL_RCC_OscConfig+0x3d6>
        {
          if((HAL_GetTick() - tickstart ) > PLL_TIMEOUT_VALUE)
    9da0:	f7fe f9f4 	bl	818c <HAL_GetTick>
    9da4:	4602      	mov	r2, r0
    9da6:	693b      	ldr	r3, [r7, #16]
    9da8:	1ad3      	subs	r3, r2, r3
    9daa:	2b02      	cmp	r3, #2
    9dac:	d901      	bls.n	9db2 <HAL_RCC_OscConfig+0x3d6>
          {
            return HAL_TIMEOUT;
    9dae:	2303      	movs	r3, #3
    9db0:	e04b      	b.n	9e4a <HAL_RCC_OscConfig+0x46e>
        while(__HAL_RCC_GET_FLAG(RCC_FLAG_PLLRDY) != RESET)
    9db2:	4b29      	ldr	r3, [pc, #164]	; (9e58 <HAL_RCC_OscConfig+0x47c>)
    9db4:	681b      	ldr	r3, [r3, #0]
    9db6:	f003 7300 	and.w	r3, r3, #33554432	; 0x2000000
    9dba:	2b00      	cmp	r3, #0
    9dbc:	d1f0      	bne.n	9da0 <HAL_RCC_OscConfig+0x3c4>
          }
        }

        /* Configure the main PLL clock source, multiplication and division factors. */
        WRITE_REG(RCC->PLLCFGR, (RCC_OscInitStruct->PLL.PLLSource                                            | \
    9dbe:	687b      	ldr	r3, [r7, #4]
    9dc0:	69da      	ldr	r2, [r3, #28]
    9dc2:	687b      	ldr	r3, [r7, #4]
    9dc4:	6a1b      	ldr	r3, [r3, #32]
    9dc6:	431a      	orrs	r2, r3
    9dc8:	687b      	ldr	r3, [r7, #4]
    9dca:	6a5b      	ldr	r3, [r3, #36]	; 0x24
    9dcc:	019b      	lsls	r3, r3, #6
    9dce:	431a      	orrs	r2, r3
    9dd0:	687b      	ldr	r3, [r7, #4]
    9dd2:	6a9b      	ldr	r3, [r3, #40]	; 0x28
    9dd4:	085b      	lsrs	r3, r3, #1
    9dd6:	3b01      	subs	r3, #1
    9dd8:	041b      	lsls	r3, r3, #16
    9dda:	431a      	orrs	r2, r3
    9ddc:	687b      	ldr	r3, [r7, #4]
    9dde:	6adb      	ldr	r3, [r3, #44]	; 0x2c
    9de0:	061b      	lsls	r3, r3, #24
    9de2:	491d      	ldr	r1, [pc, #116]	; (9e58 <HAL_RCC_OscConfig+0x47c>)
    9de4:	4313      	orrs	r3, r2
    9de6:	604b      	str	r3, [r1, #4]
                                 RCC_OscInitStruct->PLL.PLLM                                                 | \
                                 (RCC_OscInitStruct->PLL.PLLN << RCC_PLLCFGR_PLLN_Pos)             | \
                                 (((RCC_OscInitStruct->PLL.PLLP >> 1U) - 1U) << RCC_PLLCFGR_PLLP_Pos) | \
                                 (RCC_OscInitStruct->PLL.PLLQ << RCC_PLLCFGR_PLLQ_Pos)));
        /* Enable the main PLL. */
        __HAL_RCC_PLL_ENABLE();
    9de8:	4b1c      	ldr	r3, [pc, #112]	; (9e5c <HAL_RCC_OscConfig+0x480>)
    9dea:	2201      	movs	r2, #1
    9dec:	601a      	str	r2, [r3, #0]

        /* Get Start Tick */
        tickstart = HAL_GetTick();
    9dee:	f7fe f9cd 	bl	818c <HAL_GetTick>
    9df2:	6138      	str	r0, [r7, #16]

        /* Wait till PLL is ready */
        while(__HAL_RCC_GET_FLAG(RCC_FLAG_PLLRDY) == RESET)
    9df4:	e008      	b.n	9e08 <HAL_RCC_OscConfig+0x42c>
        {
          if((HAL_GetTick() - tickstart ) > PLL_TIMEOUT_VALUE)
    9df6:	f7fe f9c9 	bl	818c <HAL_GetTick>
    9dfa:	4602      	mov	r2, r0
    9dfc:	693b      	ldr	r3, [r7, #16]
    9dfe:	1ad3      	subs	r3, r2, r3
    9e00:	2b02      	cmp	r3, #2
    9e02:	d901      	bls.n	9e08 <HAL_RCC_OscConfig+0x42c>
          {
            return HAL_TIMEOUT;
    9e04:	2303      	movs	r3, #3
    9e06:	e020      	b.n	9e4a <HAL_RCC_OscConfig+0x46e>
        while(__HAL_RCC_GET_FLAG(RCC_FLAG_PLLRDY) == RESET)
    9e08:	4b13      	ldr	r3, [pc, #76]	; (9e58 <HAL_RCC_OscConfig+0x47c>)
    9e0a:	681b      	ldr	r3, [r3, #0]
    9e0c:	f003 7300 	and.w	r3, r3, #33554432	; 0x2000000
    9e10:	2b00      	cmp	r3, #0
    9e12:	d0f0      	beq.n	9df6 <HAL_RCC_OscConfig+0x41a>
    9e14:	e018      	b.n	9e48 <HAL_RCC_OscConfig+0x46c>
        }
      }
      else
      {
        /* Disable the main PLL. */
        __HAL_RCC_PLL_DISABLE();
    9e16:	4b11      	ldr	r3, [pc, #68]	; (9e5c <HAL_RCC_OscConfig+0x480>)
    9e18:	2200      	movs	r2, #0
    9e1a:	601a      	str	r2, [r3, #0]

        /* Get Start Tick */
        tickstart = HAL_GetTick();
    9e1c:	f7fe f9b6 	bl	818c <HAL_GetTick>
    9e20:	6138      	str	r0, [r7, #16]

        /* Wait till PLL is ready */
        while(__HAL_RCC_GET_FLAG(RCC_FLAG_PLLRDY) != RESET)
    9e22:	e008      	b.n	9e36 <HAL_RCC_OscConfig+0x45a>
        {
          if((HAL_GetTick() - tickstart ) > PLL_TIMEOUT_VALUE)
    9e24:	f7fe f9b2 	bl	818c <HAL_GetTick>
    9e28:	4602      	mov	r2, r0
    9e2a:	693b      	ldr	r3, [r7, #16]
    9e2c:	1ad3      	subs	r3, r2, r3
    9e2e:	2b02      	cmp	r3, #2
    9e30:	d901      	bls.n	9e36 <HAL_RCC_OscConfig+0x45a>
          {
            return HAL_TIMEOUT;
    9e32:	2303      	movs	r3, #3
    9e34:	e009      	b.n	9e4a <HAL_RCC_OscConfig+0x46e>
        while(__HAL_RCC_GET_FLAG(RCC_FLAG_PLLRDY) != RESET)
    9e36:	4b08      	ldr	r3, [pc, #32]	; (9e58 <HAL_RCC_OscConfig+0x47c>)
    9e38:	681b      	ldr	r3, [r3, #0]
    9e3a:	f003 7300 	and.w	r3, r3, #33554432	; 0x2000000
    9e3e:	2b00      	cmp	r3, #0
    9e40:	d1f0      	bne.n	9e24 <HAL_RCC_OscConfig+0x448>
    9e42:	e001      	b.n	9e48 <HAL_RCC_OscConfig+0x46c>
        }
      }
    }
    else
    {
      return HAL_ERROR;
    9e44:	2301      	movs	r3, #1
    9e46:	e000      	b.n	9e4a <HAL_RCC_OscConfig+0x46e>
    }
  }
  return HAL_OK;
